:020000040800F2
:100000000000011091E60308797C0308E19A0008DA
:1000100095E7030895E7030895E70308000000004B
:10002000000000000000000000000000C182030882
:10003000BD82030800000000B9820308D9AD0008A2
:1000400095E7030895E7030895E7030895E7030894
:1000500095E7030895E70308F5AB010821AD010812
:10006000E5AC0108A9AC01086DAC0108FDD7030897
:10007000EDD70308DDD70308CDD70308BDD70308A4
:10008000A9D7030895D7030895E7030895E7030860
:1000900095E7030895E7030895E7030831AC0108E5
:1000A00095E7030819A7000895E7030829A70008A2
:1000B00009A70008F9A6000895E7030895E70308D3
:1000C00095E7030895E7030895E7030895E7030814
:1000D00095E7030845B00008A5AF000895E70308B9
:1000E000B9AB010895E70308B585030895E7030850
:1000F00095E7030895E7030895E7030881D7030808
:1001000095E7030895E7030895E7030895E70308D3
:1001100005AF000865AE00084D60030831600308B4
:100120006DD7030859D7030845D7030831D703080B
:100130001DD7030895E7030895E7030895E703082B
:1001400095E7030895E7030895E703087D7C030816
:1001500009D70308F5D60308E1D6030895E7030895
:1001600095E7030895E7030895E7030895E7030873
:1001700095E7030895E7030895E7030895E7030863
:0801800095E7030895E7030869
:0801880028E203000100000061
:1001900016000800802400209424002000000000A5
:1001A000040600082700040050270020B82700207C
:1001B000000000000C060008010104005028002087
:1001C000103E0020000000000000000008020900AE
:1001D000A63D0020143E0020000000004B9D0108B9
:1001E00002000C00EC3D0020203E0020000000003A
:1001F00000000000F7010600A03D00202C3E00207A
:100200000000000010060008FF010100753E0020FC
:1002100054410020000000001806000803123300BB
:1002200017410020E4400020000000001A060008EA
:1002300025005A00304000208A40002000000000C5
:1002400000000000F6110C0024400020184000209F
:10025000000000005006000815007000383F002024
:10026000A83F002000000000000000002A006000FD
:10027000783E0020D83E00200000000091C2020815
:100280000300010050430020544300200000000000
:10029000000000002C001000A04800209048002022
:1002A00000000000452F02082B002400D448002045
:1002B000B048002000000000152F0208290050005F
:1002C000C8470020F848002000000000000000009F
:1002D00010000300284B0020344B002000000000D9
:1002E0005C06000828001000184B0020384B002046
:1002F00000000000697D020823001000084B002068
:10030000484B002000000000817D02081900050014
:10031000004B0020584B0020000000006006000841
:10032000F8110100FC4A0020604B00200000000092
:100330006606000800010400F84A0020644B002013
:1003400000000000680600081F000E001C4C002082
:10035000584C0020000000006C0600080502010057
:10036000044C0020684C0020000000007A060008C1
:1003700003010A00F84B00206C4C00200000000034
:100380007C06000814000200CC4D0020885100209B
:1003900000000000860600080C0024001E55002006
:1003A000F055002000000000ADC001080E20EA005A
:1003B00012540020145600200000000005C302085B
:1003C000130004005C5500200057002000000000CE
:1003D0008806000802010300FD5300200457002096
:1003E00000000000D5C0010801020500975300205D
:1003F0000857002000000000E59802080400800073
:100400006C6D0020F06D0020000000000000000076
:10041000F9010400B05A0020706E002000000000B6
:100420003D9D0108FD011E00905A0020746E0020C1
:100430000000000025960008060016001057002056
:10044000946E00200000000025C30208012008006F
:100450008C740020AC740020000000008C060008A2
:100460001A00080074740020B4740020000000001A
:100470009406000826000E004C7900203C790020EC
:1004800000000000A1EA02080B20100020770020E5
:100490005C790020000000009C0600081E0004009B
:1004A0001C7B0020047D002000000000AC0600083A
:1004B00022000C009C7A0020087D00200000000033
:1004C000B00600081B00F4000C7E0020B08C002059
:1004D00000000000D50A03080E020200087E00207A
:1004E000A48D002000000000BC0600082F001100B1
:1004F000388C0020A88D002000000000BE060008F7
:1005000005100600888C0020BC8D00200000000033
:10051000D0060008F5216C00807D0020C48D0020ED
:10052000000000000D3103080A020A00D48E0020EA
:10053000E48E002000000000D606000818102C00F1
:10054000049500205C95002000000000253602087C
:100550000D002C0030950020889500200000000040
:1005600019C1010802020300088F0020B495002081
:1005700000000000000000000C020100F88E0020C6
:10058000B895002000000000E0060008FB01010013
:1005900084B2002048B300200000000089940008C5
:1005A000FC01090050B100204CB300200000000005
:1005B0004D9400080A10120048A9002058B30020EA
:1005C00000000000E206000834001000F0A6002041
:1005D0006CB3002000000000B9C2020812200C0019
:1005E000E0A600207CB3002000000000F406000814
:1005F000FE0109009CB30020F0B3002000000000C1
:04060000D194000889
:10060400C409000019012828200300002401000067
:1006140000000000000000000000000000000000D6
:1006240000000000000000000000000000000000C6
:1006340000000000000000000000000000000000B6
:1006440000000000000000000100000000000000A5
:100654000000000000000000000105000000280167
:10066400000004008C0000000000000000000100F5
:100674000000000500000000040101006C160000E9
:100684000000030008040400E8036400040A0001F5
:100694007E05EA05B40532002B21231E6401010006
:1006A400000001000A01290000000100C800141E16
:1006B400010064002C01280000000000000000007C
:1006C4000000000000000000000000002000020103
:1006D400000000004A01B400D6010000010000300F
:1006E4000100005A0000000090012C01C8006400C1
:0C06F4000000000100054D4C54590000AE
:100700000100000001010000A82C04084C6004084E
:100710000000000000000000B82C0408C02C0408F1
:100720000000000001200000C42C0408CC2C0408A8
:100730000000000001400000D02C04080050040814
:100740000000000001200000DC2C0408E82C040854
:100750000000000004000000EC2C0408746304088E
:100760000000000004000000F82C0408DC3B040832
:1007700000000000010000000201FF000000803FB7
:100780000000803FFFFFFFFF0101D601E9280208BA
:100790000000000000000000C80000200508030061
:1007A00000000000541D0408301D0408241D040826
:1007B000000000000100000000000000010203042E
:1007C0000102030406070809756A0208716A020833
:1007D0006D6A0208956C0208716C02086B6A020867
:1007E000696A0208556A0208456A02083D6A0208F9
:1007F000416A0208000101010100E00120700020AF
:10080000702D72000800000000600240106002407D
:1008100000000000000B00000000200000000000AD
:10082000000000000060024028600240000000005C
:10083000060C000000002000000000000000000086
:10084000006002404060024000000000100D000007
:1008500000002000000000000000000000600240D6
:100860005860024000000000160E0000000020004A
:1008700000000000000000000060024070600240C4
:1008800000000000200F0000000020000000000019
:10089000000000000060024088600240000000008C
:1008A00026100000000020000000000000000000F2
:1008B00000600240A0600240000000003011000013
:1008C0000000200000000000000000000060024066
:1008D000B860024000000000362F00000000200039
:1008E00000000000000000000064024010640240AC
:1008F0000000000000380000000040000000000080
:100900000000000000640240286402400000000073
:100910000639000000004000000000000000000058
:10092000006402404064024000000000103A0000F1
:1009300000004000000000000000000000640240D1
:100940005864024000000000163B00000000400018
:1009500000000000000000000064024070640240DB
:1009600000000000203C00000000400000000000EB
:1009700000000000006402408864024000000000A3
:1009800026440000000040000000000000000000BD
:1009900000640240A06402400000000030450000F6
:1009A0000000400000000000000000000064024061
:1009B000B86402400000000036460000000040001D
:1009C00000000000000000000000803F0000803FA9
:1009D0000000000000000000000000000000803F58
:1009E0000000000000000000000000000000000007
:1009F00000000000000000000000000000000000F7
:100A0000000000000000803F000000000000000027
:100A100000000000D83204080000000000000000C0
:100A2000E9C00108A08601000400000000000000E9
:100A300000000000000000000000000000000000B6
:100A40000000000000000000EC660408385A0408AA
:100A500000000000192901087D00000006000000C8
:100A60000000000000000000000000000000000086
:100A7000000000000000000000000000AC6004085E
:100A8000000000000000000029250108E803000024
:100A90000300000000000000000000000000000053
:100AA0000000000000000000000000000000000046
:100AB000B4600408000000000000000059C40208EF
:100AC00010270000030000000000000000000000EC
:100AD0000000000000000000000000000000000016
:100AE00000000000C060040800000000992D02080A
:100AF0001DFE0008204E0000050000000000000060
:100B000000000000000000000000000000000000E5
:100B10000000000000000000703404080000000025
:100B2000000000005DB10008102700000100000077
:100B300000000000000000000000000000000000B5
:100B4000000000000000000000000000C460040875
:100B5000000000000000000019940008E8030000F5
:100B60000500000000000000000000000000000080
:100B70000000000000000000000000000000000075
:100B8000D06004080000000000000000D5C3010888
:100B9000204E0000030000000000000000000000E4
:100BA0000000000000000000000000000000000045
:100BB00000000000E06004080000000000000000E9
:100BC000DDC10108204E000003000000000000000D
:100BD0000000000000000000000000000000000015
:100BE0000000000000000000F060040800000000A9
:100BF0000000000055960008400D030003000000AF
:100C000000000000000000000000000000000000E4
:100C1000000000000000000000000000A4330408F1
:100C2000000000000000000029C103081027000098
:100C300001000000000000000000000000000000B3
:100C400000000000000000000000000000000000A4
:100C5000783404080000000000000000A59D020890
:100C6000102700000300000000000000000000004A
:100C70000000000000000000000000000000000074
:100C800000000000843404080000000000000000A0
:100C900011B80008A00F00000100000000000000D3
:100CA0000000000000000000000000000000000044
:100CB00000000000000000000061040800000000C7
:100CC00000000000D104030810270000010000000C
:100CD0000000000000000000000000000000000014
:100CE000000000000000000000000000AC33040819
:100CF0000000000000000000913F03081A410000BE
:100D000001000000000000000000000000000000E2
:100D100000000000000000000000000000000000D3
:100D2000E83404080000000000000000996A02088E
:100D3000102700000100000000000000000000007B
:100D400000000000000000000000000000000000A3
:100D5000000000000C61040800000000000000001A
:100D6000358903081A41000001000000000000005E
:100D70000000000000000000000000000000000073
:100D800000000000000000001061040800000000E6
:100D900000000000C5780108400D030000000000BD
:100DA0000000000000000000000000000000000043
:100DB00000000000000000000000000018610408AE
:100DC000000000000000000075780108400D0300DD
:100DD0000000000000000000000000000000000013
:100DE0000000000000000000000000000000000003
:100DF00020610408000000000000000055A6020861
:100E0000A0860100030000000000000000000000B8
:100E100000000000000000000000000000000000D2
:100E20000000000000000101FFFF00000902430074
:100E3000020100C032090400000102020100052481
:100E4000001001052401000104240202052406000B
:100E500001070582030800FF09040100020A0000DF
:100E60000007050102400000070581024000000064
:100E7000FF00000001000000FFFFFFFF0000803FB7
:100E8000000000000000000000000000080000005A
:100E90009D21030855210308453003080000000088
:100EA000451D0308A9200308292103081120030870
:100EB0000000000000000000391D0308C578030889
:100EC000C1780308BD780308B1780308AD7803083A
:100ED000B9780308B5780308397903082D79030830
:100EE0000579030819790308F1780308DD78030808
:100EF000C978030804030904120100020202004039
:100F00008304405700020102030100001573020828
:100F100085220308C16D0208891D030831220308D8
:100F2000991D0308B51D0308791D0308691D0308F1
:100F300000000000000000000000000000000000B1
:100F4000601A0020FFFFFFFFFA0000000100000010
:100F500001000000DC630408E4630408588C0020EE
:100F60000100C40900000000568C00200100C409E3
:100F700000000000548C00200100C40900000000A3
:100F8000528C00200100C409000000004E8C00209B
:100F90000100C40900000000508C00200100C409B9
:100FA000000000004C8C00200100C409000000007B
:100FB0004A8C00200100C40900000000A853002052
:100FC0000100C80001000000A65300203200307567
:100FD00032000000A5530020055A0500A053002050
:100FE00000FF0100A453002001000000540800206D
:100FF000A253002002000000C82704089F530020CD
:1010000000FF0100A353002001000000540800204D
:10101000A153002002000000C827040896530020B6
:1010200001000000281D040895530020010801005C
:101030009453002004000000EC27040856550020BB
:101040000100FF7F01000000555500200200000054
:10105000002804080654002003000000102804089B
:101060000554002003000000102804080455002047
:101070000000F40101000000025500200000F4010E
:1010800001000000005500200000F40101000000F4
:10109000FE5400200000F40101000000FC54002078
:1010A00000FF01001C550020E803D0070A000000E3
:1010B0001A550020006401000A00000016550020A7
:1010C0000064010015550020006401001B5500203C
:1010D000006401000A0000001455002000640100B3
:1010E0000A00000019550020006401000A000000F9
:1010F00018550020006401000A0000001755002068
:10110000006401000A0000001355002000FF0100E8
:101110000A0000001255002000FF01000A00000034
:101120000E5400200000F401010000000C540020C7
:101130000000F401010000000A5400200000F40146
:1011400001000000085400200000F401010000002C
:101150000E5500201400E803010000000C5500208B
:10116000E8033075010000000B55002000C80100A5
:101170000A55002000C801000955002000C80100E0
:1011800008550020006401000A00000007550020F7
:1011900000FF01000A0000004B55002000C80100BC
:1011A0004A55002000C801004955002000C8010030
:1011B0004855002000C801004755002000C8010024
:1011C0004655002000C801004555002000C8010018
:1011D0004455002000C801004355002000C801000C
:1011E000F46304080000000000000000000000009C
:1011F0000000000004640408090000000000000072
:10120000B0080020040000000C640408090000007D
:1012100000000000A40800200400000090690408F9
:1012200009000000000000009808002004000000F1
:10123000042E040809000000000000008C080020B3
:10124000040000001464040809000000000000000D
:1012500080080020040000001C640408090000004D
:10126000000000007408002004000000246404084A
:1012700009000000000000006808002004000000D1
:101280002C64040809000000000000005C08002035
:1012900004000000346404080100000000000000A5
:1012A0000000000000000000000000000E00000030
:1012B0000000000000000000000000004865040875
:1012C000000000000000000000000000000000001E
:1012D0008C3204080700000000000000D408002041
:1012E000000000005865040808000000000000002D
:1012F000C808002000000000646504080800000021
:1013000000000000BC080020000000003464040855
:1013100001000000000000000000000000000000CC
:10132000000000000E0000000000000000000000AF
:10133000000000006C6504080000000000000000D0
:1013400000000000000000007C6504080D000000A3
:10135000000000001009002000000000846504085F
:101360000D00000000000000040900200000000043
:101370008C6504080700000000000000FC08002045
:1013800000000000946504080D000000000000004B
:10139000F0080020000000009C6504080D0000001B
:1013A00000000000E408002000000000A46504081C
:1013B0000700000000000000DC0800200000000022
:1013C0003464040801000000000000000000000078
:1013D00000000000000000000E00000000000000FF
:1013E0000000000000000000AC65040800000000E0
:1013F0000000000000000000000000008C32040823
:101400000C00000000000000AA53002000000000B3
:10141000C06504080C00000000000000AC53002070
:1014200000000000D06504080C000000000000006F
:10143000E253002000000000E06504080C000000FA
:1014400000000000D653002000000000F4650408EE
:101450000C00000000000000AE530020000000005F
:10146000006604080C00000000000000B0530020DB
:1014700000000000086604080C00000000000000E6
:10148000B2530020000000001C6604080C0000009D
:1014900000000000B453002000000000246604088F
:1014A0000C00000000000000B65300200000000007
:1014B0002C6604080C00000000000000F45300201B
:1014C00000000000446604080C000000000000005A
:1014D000B853002000000000506604080C00000013
:1014E00000000000BA530020000000001C63040844
:1014F0000C00000000000000BC53002000000000B1
:10150000586604080C00000000000000BE530020D4
:1015100000000000646604080C00000000000000E9
:10152000C053002000000000706604080C0000009A
:1015300000000000C2530020000000007C66040888
:101540000C00000000000000C45300200000000058
:10155000886604080C00000000000000C65300204C
:1015600000000000946604080C0000000000000069
:10157000DA530020000000009C6604080C00000004
:1015800000000000D853002000000000A4660408FA
:101590000C00000000000000E653002000000000E6
:1015A000B06604080C00000000000000E8530020B2
:1015B00000000000BC6604080C00000000000000F1
:1015C000EE53002000000000E06404080C0000005E
:1015D00000000000C853002000000000C866040896
:1015E0000C00000000000000D053002000000000AC
:1015F000D06604080C00000000000000CA53002060
:1016000000000000DC6604080C0000000000000080
:10161000CC53002000000000E86604080C00000025
:1016200000000000CE53002000000000F066040817
:101630000C00000000000000D25300200000000059
:10164000AC3204080C00000000000000DC53002055
:1016500000000000FC6604080C0000000000000010
:10166000D453002000000000086704080C000000AC
:1016700000000000E453002000000000146704088C
:101680000C00000000000000DE53002000000000FD
:101690001C6704080C00000000000000E05300205C
:1016A00000000000246704080C0000000000000097
:1016B000EA530020000000002C6704080C00000022
:1016C00000000000EC530020000000003464040817
:1016D0000100000000000000000000000000000009
:1016E000000000000E0000000000000000000000EC
:1016F0000000000034670408000000000000000043
:10170000000000000000000044670408050000001D
:1017100000000000045400200000000034640408AD
:1017200001000000000000000000000000000000B8
:10173000000000000E00000000000000000000009B
:10174000000000004C6704080000000000000000DA
:101750000000000000000000EC5E04080D00000026
:101760000000000030090020000000005867040855
:101770000700000000000000280900200000000011
:10178000C86604080D000000000000001C090020CD
:1017900000000000346404080100000000000000A4
:1017A0000000000000000000000000000E0000002B
:1017B0000000000000000000000000006067040856
:1017C0000000000000000000000000000000000019
:1017D000706704080D0000000000000048090020A8
:1017E00000000000786704080A0000000000000004
:1017F0006255002000000000846704080A00000011
:10180000000000006A550020000000008C670408FA
:101810000A000000000000007255002000000000D7
:101820009467040808000000000000003C09002044
:101830000000000034640408010000000000000003
:101840000000000000000000000000000E0000008A
:101850000000000000000000000000009C67040879
:101860000000000000000000000000000000000078
:10187000B06704080D0000000000000060090020AF
:1018800000000000C067040804000000DDA2020898
:101890000000000000000000C86704080D00000000
:1018A000000000005409002000000000DC6704086C
:1018B00004000000B9A202080000000000000000BF
:1018C0003464040801000000000000000000000073
:1018D00000000000000000000E00000000000000FA
:1018E0000000000000000000E467040800000000A1
:1018F000000000000000000000000000F86704087D
:1019000007000000000000009C090020000000000B
:10191000046804080800000000000000900900208E
:10192000000000001068040808000000000000002B
:1019300084090020000000001C6804080800000062
:10194000000000007809002000000000286804085A
:1019500008000000000000006C09002000000000EA
:1019600034640408010000000000000000000000D2
:1019700000000000000000000E0000000000000059
:1019800000000000000000003468040800000000AF
:1019900000000000FF00002000000000302D0408BF
:1019A0000B00000000000000140A002000000000EE
:1019B000406804080B00000000000000080A002036
:1019C000000000004C6804080B000000000000004C
:1019D000FC09002000000000586804080B0000000B
:1019E00000000000F0090020000000006468040806
:1019F0000B00000000000000E409002000000000CF
:101A0000382D04080B00000000000000D809002059
:101A100000000000706804080B00000000000000D7
:101A2000CC090020000000007C68040807000000CA
:101A300000000000C40900200000000084680408C1
:101A40000700000000000000BC09002000000000AA
:101A5000906804080B00000000000000B00900209E
:101A6000000000009C68040808000000000000005E
:101A7000A4090020000000003464040801000000F4
:101A80000000000000000000000000000000000056
:101A90000E00000000000000000000000000000038
:101AA000A86804080000000000000000000000001A
:101AB00000000000BC6804080800000000000000EE
:101AC000440A002000000000C86804080800000064
:101AD00000000000380A002000000000D46804085C
:101AE00008000000000000002C0A00200000000098
:101AF000E06804080800000000000000200A002040
:101B00000000000034640408010000000000000030
:101B10000000000000000000000000000E000000B7
:101B2000000000000000000000000000E868040859
:101B30000000000000000000FC0000200000000089
:101B4000F86804080B000000000000008C0A002068
:101B500000000000046904080B0000000000000001
:101B6000800A00200000000010690408070000003F
:101B700000000000780A0020000000001C69040832
:101B80000700000000000000700A002000000000B4
:101B9000286904080700000000000000680A00200F
:101BA0000000000034690408080000000000000084
:101BB0005C0A0020000000003C69040808000000E6
:101BC00000000000500A00200000000034640408F7
:101BD0000100000000000000000000000000000004
:101BE000000000000E0000000000000000000000E7
:101BF000000000004469040800000000000000002C
:101C0000FC000020000000005069040807000000EC
:101C100000000000D80A00200000000058690408F5
:101C20000700000000000000D00A002000000000B3
:101C3000606904080700000000000000C80A0020D6
:101C400000000000CC2D0408070000000000000088
:101C5000C00A002000000000D42D04080700000086
:101C600000000000B80A002000000000DC2D04087D
:101C70000700000000000000B00A00200000000083
:101C8000686904080700000000000000A80A00209E
:101C90000000000070690408070000000000000058
:101CA000A00A002000000000786904080700000076
:101CB00000000000980A00200000000034640408BE
:101CC0000100000000000000000000000000000013
:101CD000000000000E0000000000000000000000F6
:101CE0000000000000000000FD9A0208E00A002049
:101CF000025400201B00000020280408015400208A
:101D00000A3201000054002001FA0100FC530020B7
:101D100000C80100FA530020E803D00701000000CA
:101D20004D4C545950484634000000009E5300204A
:101D3000000301009D530020000301001D9A0208CA
:101D4000F5990208BC0B0020B199020865990208B8
:101D5000340C00205D9A0208459A0208E80C002025
:101D6000139B020851A00208F40F0020F598020806
:101D700085A2020844100020E1A30208799D020810
:101D8000BC100020399B0208000000005C110020FC
:101D9000DD9B0208AD9B0208E8110020699C020847
:101DA000AD9C02088812002010550020010301009C
:101DB000799B02084D9B0208A01300200D9C02088D
:101DC00001A302082C140020D99C02085DA302087C
:101DD000F414002006550020010301008069040866
:101DE00000000000000000000000000000000000F3
:101DF0008C69040808000000000000001416002090
:101E000000000000946904080700000000000000C2
:101E10000C16002000000000A46904080700000060
:101E2000000000000416002000000000B069040853
:101E30000700000000000000FC150020000000006A
:101E4000BC6904080D00000000000000F01500202F
:101E500000000000C869040803000000CD870308E3
:101E6000E4150020000000003464040801000000B4
:101E70000000000000000000000000000000000062
:101E80000E00000000000000000000000000000044
:101E9000D0690408000000000000000000000000FD
:101EA00000000000E06904080A00000000000000D3
:101EB000042D040800000000E86904080A0000007E
:101EC00000000000882C040800000000F0690408ED
:101ED0000A000000000000004C5500200000000037
:101EE000F86904080A000000000000002016002025
:101EF000000000003464040801000000000000003D
:101F00000000000000000000000000000E000000C3
:101F1000000000000000000000000000006A04084B
:101F200000000000000000000000000000000000B1
:101F30000C6A040803000000CD8703085416002033
:101F400000000000186A040803000000CD870308A1
:101F50004816002000000000206A0408030000006A
:101F6000CD8703083C16002000000000286A040802
:101F700005000000000000009C530020000000004D
:101F8000306A04080700000000000000341600203A
:101F9000000000003C6A0408070000000000000088
:101FA0002C1600200000000034640408010000002A
:101FB0000000000000000000000000000000000021
:101FC0000E00000000000000000000000000000003
:101FD000486A040800000000000000000000000043
:101FE000000000005C6A040803000000CD870308BD
:101FF0007816002000000000DC3304080300000015
:10200000CD8703086C16002000000000686A0408F1
:1020100003000000CD8703086016002000000000C8
:10202000346404080100000000000000000000000B
:1020300000000000000000000E0000000000000092
:102040000000000000000000746A040800000000A6
:10205000000000000000000000000000806A04088A
:1020600007000000A9A30208D41600200000000009
:10207000EC66040803000000CD870308C8160020A2
:10208000000000008C6A040803000000CD870308EC
:10209000BC16002000000000946A04080300000041
:1020A000CD870308B0160020000000009C6A0408D9
:1020B000070000008DA30208A81600200000000001
:1020C000602D040803000000CD8703089C16002043
:1020D00000000000A86A040803000000CD87030880
:1020E0009016002000000000B46A040803000000FD
:1020F000CD87030884160020000000003464040823
:1021000001000000000000000000000000000000CE
:10211000000000000E0000000000000000000000B1
:1021200000000000B99A0208759A0208DC16002027
:10213000459D020800000000901700204199020808
:102140001D9902081C18002000000000000000007B
:10215000D01800201D9D0208C5A3020848190020C0
:10216000C06A040800000000000000000000000039
:1021700000000000CC6A040803000000CD870308BB
:10218000541A002000000000D46A04080300000074
:10219000CD870308481A002000000000AC33040873
:1021A00003000000CD8703083C1A00200000000057
:1021B000E06A040803000000CD870308301A0020FD
:1021C00000000000EC6A040803000000CD8703084B
:1021D000241A002000000000F46A04080200000035
:1021E000E58603080000000000000000FC6A040807
:1021F00002000000E5860308010000000000000066
:10220000086B040802000000E586030802000000D5
:1022100000000000000000000E00000000000000B0
:10222000000000000000000001010000500100005B
:1022300007000000020000003C1B0020000000001E
:10224000000000000000000000000000000000008E
:10225000000000000000000000000000000000007E
:10226000000000000000000000000000000000006E
:10227000000000000000000000000000000000005E
:10228000000000000000000000000000000000004E
:1022900000000000000000000000000043000000FB
:1022A000000000000000000000000000000000002E
:1022B00000000000000000000000000043000000DB
:1022C000000000000000000000000000000000000E
:1022D00000000000000000000000000043000000BB
:1022E00000000000000000000000000000000000EE
:1022F000000000000000000000000000430000009B
:1023000000000000000000000000000000000000CD
:10231000000000000000000000000000430000007A
:1023200000000000000000000000000000000000AD
:10233000000000000000000000000000430000005A
:10234000000000000000000000000000000000008D
:10235000000000000000000000000000430000003A
:10236000000000000000000000000000000000006D
:1023700000000000000000000000000033EA030835
:102380000FEA0308000000009F6C0408CD630408F6
:102390009B6004089B6004089B6004089B60040821
:1023A0009B6004089B6004089B6004089B60040811
:1023B0009B600408FFFFFFFFFFFFFFFFFFFFFFFF22
:1023C000FFFF0000010041534349490000000000A5
:1023D00000000000000000000000000000000000FD
:1023E0000000000000004153434949000000000084
:1023F00000000000000000000000000000000000DD
:0C240000000000000000000001000000CF
:108000004FF48053838270472DE9F0472A4F2B4D60
:108010002B4C82463868894612F096FD012002F00A
:108020003DFE0026A8464AFA06F3DA0720683DD549
:1080300012F090FD286812F08DFD012002F02EFE56
:10804000286812F081FD0136012002F027FE042E7F
:10805000E9D1206812F07EFD286812F07BFD012036
:1080600002F01CFE286812F06FFD012002F016FEDF
:10807000002529FA05F3DB0720681AD512F06AFDFE
:10808000D8F8000012F066FD012002F007FED8F8D3
:10809000000012F059FD0135012002F0FFFD142D02
:1080A000E7D13868BDE8F04712F054BD12F04CFD3E
:1080B000C0E712F049FDE3E7E43D0020E83D002081
:1080C000E03D0020A849A948A94A2DE9F84F01231D
:1080D00003700B88128823F040031B041B0C0B80D9
:1080E0000B8823F038031B0452084FEA13430BD0CC
:1080F00042F48072002A92FAA2F1B1FA81F208BF2A
:108100004FF0FF32013AD2001343974A9BB21380DB
:1081100013889BB243F040031380964B1B6813B146
:108120001A689B885383904940F2E93302E0002BA0
:1081300000F09E810A89013B12F0020F9BB2F6D03B
:1081400005238B8140F2E933874902E0002B00F0E0
:108150008F810A89013B12F0010F9BB2F6D08B8907
:10816000814940F2E93302E0002B00F0A5810A8941
:10817000013B12F0020F9BB2F6D000238B8140F23C
:10818000E933794902E0002B00F096810A89013B2E
:1081900012F0010F9BB2F6D08B89734940F2E9339C
:1081A00002E0002B00F084810A89013B12F0020FEB
:1081B0009BB2F6D006238B8140F2E9336A4902E094
:1081C000002B00F075810A89013B12F0010F9BB270
:1081D000F6D08B89644940F2E93302E0002B00F0CD
:1081E00063810A89013B12F0020F9BB2F6D0002393
:1081F0008B8140F2E9335C4902E0002B00F05481AE
:108200000A89013B12F0010F9BB2F6D08B89DFF88F
:108210006CA155499AF8004040F2E93344F001045A
:1082200002E0002B00F03C810A89013B12F0020FB2
:108230009BB2F6D004238B8140F2E9334A4902E035
:10824000002B00F02D810A89013B12F0010F9BB237
:10825000F6D08B89444940F2E93302E0002B00F06C
:108260001B810A89013B12F0020F9BB2F6D0A4B227
:108270008C8140F2E9333C4902E0002B00F00C8194
:108280000A89013B12F0010F9BB2F6D08B893A4F5D
:108290003B88002B47D0DFF8E890DFF8E880324CCD
:1082A0004FF0000B072699F8015040F2E93302E045
:1082B000002B00F0D5802089013B10F0020F9BB20B
:1082C000F6D0A68140F2E93302E0002B00F0C8802E
:1082D0002089013B10F0010F9BB2F6D0A38940F238
:1082E000E93302E0002B00F0BF802089013B10F051
:1082F000020F9BB2F6D0ADB2A58140F2E93302E0A5
:10830000002B00F0B1802089013B10F0010F9BB2DF
:10831000F6D0A3893B8819F8010F08F8010F0BF17B
:10832000010B9B45BFDB104840F2E93302E0002B14
:1083300000F0AE800289013B12F0020F9BB2F6D032
:1083400007238381084940F2E93302E0002B00F063
:108350009F800A89013B12F0010F9BB2F6D08B89F6
:10836000014840F2E93311E0003C00406055002034
:108370008C070020F08E0020FA000020101D002045
:108380008B510020131D0020002B7DD00289013B62
:1083900012F0020F9BB2F7D0FF238381484940F2CD
:1083A000E93301E0002B6FD00A89013B12F0010F85
:1083B0009BB2F7D08B899AF80040414840F2E933EC
:1083C00001E0002B5CD00289013B12F0020F9BB24E
:1083D000F7D0042383813A4940F2E93301E0002BCE
:1083E0004ED00A89013B12F0010F9BB2F7D08B8966
:1083F000334840F2E93301E0002B3DD00289013BD4
:1084000012F0020F9BB2F7D0A4B22D49848140F242
:10841000E93301E0002B2FD00A89013B12F0010F54
:108420009BB2F7D08B89274B1B6813B11A689B88C6
:108430001383234A138823F040031B041B0C13806F
:10844000138823F038031B041B0C138013889BB282
:1084500043F0400313801C4B00211970BDE8F88FD6
:10846000204612F0DFFC3AE7204612F0DBFC51E731
:10847000134812F0D7FC73E6114812F0D3FCD2E790
:108480000F4812F0CFFCB3E70D4812F0CBFC92E797
:108490000B4812F0C7FC63E7094812F0C3FCF6E68C
:1084A000074812F0BFFCD5E6054812F0BBFCAEE66B
:1084B000034812F0B7FC8DE6014812F0B3FC6CE6FD
:1084C000003C0040F08E002060550020AA490A8838
:1084D00022F040022DE9F0471204A84F120C3B880D
:1084E0000A800A8822F0380212045B084FEA12421E
:1084F00000F00D8243F4807090FAA0F10028B1FAE8
:1085000081F108BF4FF0FF310139C9000A439A4990
:108510009B4D92B20A800A8892B242F040020A80D1
:10852000296811B10A6888885083964A1278012A0E
:1085300000F05482C0F00D82022A40F0D481924EA5
:10854000082232704FF4C372DFF844828A48A8F8D8
:108550000020028822F040021204120C02800288DD
:1085600022F038021204120C5BB143F4807090FACE
:10857000A0F30028B3FA83F308BF4FF0FF33013BA9
:10858000DB0013437C4A9BB2138013889BB243F0F9
:108590004003138011B10B688A885A83764C4FF0E0
:1085A00010094FF0010A40F2E93302E0002B00F01D
:1085B000A4812289013B12F0020F9BB2F6D01FFA70
:1085C00089F3A38140F2E93302E0002B00F09581AA
:1085D0002289013B12F0010F9BB2F6D0A38940F231
:1085E000E93302E0002B00F08C812289013B12F07C
:1085F000020F9BB2F6D0A4F80CA040F2E93302E0DF
:10860000002B00F07E812289013B12F0010F9BB20A
:10861000F6D0A38909F10109B9F1200FC3D1296866
:1086200011B10B688A881A83534B1A8822F04002D2
:108630001204120C1A801A8822F038021204120C4A
:108640001A801A8892B242F040021A8018883A883A
:1086500020F040000004000C18801B8823F0380331
:108660001B0452084FEA13430BD042F48072002AD5
:1086700092FAA2F0B0FA80F208BF4FF0FF32013A4E
:10868000D20013433C4A9BB2138013889BB243F041
:108690004003138011B10B688A885A8334783649B5
:1086A00040F2E93302E0002B00F04B810A89013BE4
:1086B00012F0020F9BB2F6D000238B8140F2E93317
:1086C0002D4902E0002B00F03C810A89013B12F0A9
:1086D000010F9BB2F6D08B89274940F2E93302E0C3
:1086E000002B00F032810A89013B12F0020F9BB28D
:1086F000F6D0A4B28C8140F2E9331F4902E0002B8E
:1087000000F023810A89013B12F0010F9BB2F6D0E1
:108710008B891E4B18491C7840F2E93302E0002B8C
:1087200000F0F7800A89013B12F0020F9BB2F6D0ED
:1087300002238B8140F2E9330F4902E0002B00F065
:10874000E8800A89013B12F0010F9BB2F6D08B89B9
:10875000094940F2E93302E0002B00F0DE800A898B
:10876000013B12F0020F9BB2F6D0A4B28C8140F212
:10877000E933014911E000BF003C00408C070020B4
:10878000F08E0020048F0020040100200B8F0020B9
:10879000FA000020002B00F0C0800A89013B12F093
:1087A000010F9BB2F6D08B899A4B9B481C7840F204
:1087B000E93302E0002B00F0B4800289013B12F0A3
:1087C000020F9BB2F6D003238381934940F2E93331
:1087D00002E0002B00F0A5800A89013B12F0010F96
:1087E0009BB2F6D08B898C4840F2E93302E0002B33
:1087F00000F09B800289013B12F0020F9BB2F6D081
:10880000A4B28549848140F2E93302E0002B00F0F4
:108810008C800A89013B12F0010F9BB2F6D08B8944
:108820007E4B7D481C7840F2E93344F0040401E0BB
:10883000002B7ED00289013B12F0020F9BB2F7D0D1
:1088400004238381744940F2E93301E0002B70D0A6
:108850000A89013B12F0010F9BB2F7D08B896E4859
:1088600040F2E93301E0002B67D00289013B12F0AE
:10887000020F9BB2F7D0A4B26749848140F2E9337A
:1088800001E0002B59D00A89013B12F0010F9BB285
:10889000F7D08B892B6813B11A689B8813835E4AC3
:1088A0005F4C13885F4823F040031B041B0C1380AC
:1088B000138823F038031B041B0C138013889BB20E
:1088C00043F040031380B8F80020002137F061F92D
:1088D0002378D3B1544B1B78002B00F08580002304
:1088E0002370BDE8F087514E327812F0400F0CBF74
:1088F0004FF4C3724FF4F07226E6204612F092FA5B
:108900006DE6204612F08EFA84E6BDE8F08719463F
:10891000FCE5414812F086FA1AE73F4812F082FA65
:1089200042E73D4812F07EFA5DE73B4812F07AFAE2
:1089300076E7394812F076FA91E7374812F072FA82
:10894000A8E7354812F06EFAC6E6334812F06AFA24
:10895000DFE6314940F2E93301E0002B55D00A89C6
:10896000013B12F0020F9BB2F7D0A0238B8140F2A3
:10897000E933294901E0002B47D00A89013B12F075
:10898000010F9BB2F7D08B89234940F2E93301E014
:10899000002B35D00A89013B12F0020F9BB2F7D0B1
:1089A00000238B8140F2E9331B4900E043B30A897D
:1089B000013B12F0010F9BB2F8D08B89D8B200F0C6
:1089C0000603022B194E03D000F00503012B11D032
:1089D0003B882968082232705B08B3E5134E4822B1
:1089E00032704FF4F072AFE5FFF76CFB0023237099
:1089F000BDE8F0873B882968482232705B08F0E7C1
:108A0000054812F00FFAC0B2D9E7034812F00AFA8B
:108A1000BAE700BF0C8F0020003C0040101D002072
:108A200000000020141D00206055002004010020DB
:108A300089498A4A2DE9F84F012313700B88884A27
:108A400023F040031B041B0C12880B800B8823F0BF
:108A500038031B0452084FEA13430BD042F48072D0
:108A6000002A92FAA2F1B1FA81F208BF4FF0FF3268
:108A7000013AD2001343784A9BB2138013889BB209
:108A800043F040031380774B1B6813B11A689B882F
:108A90005383714940F2E93302E0002B00F0458135
:108AA0000A89013B12F0020F9BB2F6D080238B8122
:108AB00040F2E933684902E0002B00F036810A8970
:108AC000013B12F0010F9BB2F6D08B89624940F254
:108AD000E93302E0002B00F02C810A89013B12F0FF
:108AE000020F9BB2F6D000238B8140F2E9335A4942
:108AF00002E0002B00F01D810A89013B12F0010FFA
:108B00009BB2F6D08889C0B2564B1B6813B11A6865
:108B10009B881383504A544C1388544D23F04003D0
:108B20001B041B0C1380138823F038031B041B0C3D
:108B3000138013889BB243F04003138023782F687F
:108B400083423ED0FFF7C2FC494E4A4BB6F8EE21B5
:108B5000DFF828C1B3F8008000210B464FF0050B69
:108B60004FF0060A4FF00709B5181CF802402879A3
:108B7000A04202F1010703F1050012D006EB000E3E
:108B8000F0182C71150A80F8F0B180F8F2A180F885
:108B9000F32180F8F49180F8F151013106338EF819
:108BA000F041BAB2424501F101016BD26329DBDD2C
:108BB000A6F8EE21002B6AD1284A00231370BDE8E5
:108BC000F88F2D4B2A4E1B78002BBED1D6F8E431FE
:108BD000FB1AB3F57A7FB8D9214B1046198834F0C7
:108BE0006DFC204B1B6813B11A689B885383A0212E
:108BF000194834F015FC0021174834F011FC194BCA
:108C00001B68814613B11A689B881383DFF8708054
:108C10001148042134F052FC98F80030182B00F071
:108C2000918019F0040F40F0898009F00503012BB1
:108C300000F0968063B923785B0609D5D6F8E82161
:108C40002B68002A00F091809B1A642B00F2908020
:108C5000C6F8E47179E700BF003C00406055002091
:108C60008C070020F08E002004010020E8B30020D3
:108C7000101D0020FA000020048F00208C510020DD
:108C8000F98E00200022A6F8EE21002B94D0404857
:108C9000404A0188128821F040010904090C018032
:108CA000018821F03801090452084FEA11410BD024
:108CB00042F48072002A92FAA2F0B0FA80F208BF61
:108CC0004FF0FF32013AD2000A43314992B20A8092
:108CD0000A8892B242F040020A802F4A126812B10A
:108CE000116892884A8300222C49294834F068FB95
:108CF000294B1B6813B11A689B881383244A138875
:108D000023F040031B041B0C1380138823F038034B
:108D10001B041B0C138013889BB243F04003138089
:108D20001F4A00231370BDE8F88F194812F07AF833
:108D3000CCE6174812F076F8C0B2E5E60023C6F894
:108D4000E83185E72378174A03F04003002B09F048
:108D500007010CBF0D20102013805180D08060E7E8
:108D600023785A067FF56AAF72E7C6F8E8316FE7F5
:108D7000FFF7ACFB98F80030182B7FF469AFB6F81A
:108D8000EC31084A01339BB2A6F8EC3193805FE7DF
:108D9000003C00408C070020F08E0020001F0020C7
:108DA00060550020FC8E00202DE9F84FA94F3B783C
:108DB00003B1FEE7A84CA94A01233B70238812881F
:108DC00023F040031B041B0C2380238823F038036B
:108DD0001B0452084FEA13430BD042F48072002A5E
:108DE00092FAA2F4B4FA84F208BF4FF0FF32013ACB
:108DF000D2001343984ADFF870829BB21380138825
:108E00009BB243F040031380D8F8003013B11A68C6
:108E10009B885383924B01220D461A7004468E495B
:108E200040F2E93302E0002B00F0A3810A89013B04
:108E300012F0020F9BB2F6D000238B8140F2E9338F
:108E4000854902E0002B00F094810A89013B12F071
:108E5000010F9BB2F6D08B897F4940F2E93302E0E3
:108E6000002B00F09A810A89013B12F0020F9BB29D
:108E7000F6D000238B8140F2E933774902E0002BE2
:108E800000F08B810A89013B12F0010F9BB2F6D0F2
:108E90008B89714940F2E93302E0002B00F07981BF
:108EA0000A89013B12F0020F9BB2F6D009238B8195
:108EB00040F2E933684902E0002B00F06A810A8938
:108EC000013B12F0010F9BB2F6D08B89624940F250
:108ED000E93302E0002B00F058810A89013B12F0CF
:108EE000020F9BB2F6D0A4B28C8140F2E9335A490A
:108EF00002E0002B00F049810A89013B12F0010FCA
:108F00009BB2F6D08B89574E534C013D4FF0000A6F
:108F10004FF00A0B40F2E93302E0002B00F0108121
:108F20002289013B12F0020F9BB2F6D0A4F80CB0DC
:108F300040F2E93302E0002B00F002812289013B7C
:108F400012F0010F9BB2F6D0A38940F2E93302E0A0
:108F5000002B00F0F9802289013B12F0020F9BB236
:108F6000F6D01FFA8AF3A38140F2E93302E0002B26
:108F700000F0EA802289013B12F0010F9BB2F6D08B
:108F8000A38915F8019F40F2E93302E0002B00F0BD
:108F9000DF802289013B12F0020F9BB2F6D00B2337
:108FA000A38140F2E93302E0002B00F0D180228956
:108FB000013B12F0010F9BB2F6D0A38940F2E933D6
:108FC00002E0002B00F0C8802289013B12F0020F62
:108FD0009BB2F6D01FFA89F9A4F80C9040F2E9335D
:108FE00002E0002B00F0B8802289013B12F0010F53
:108FF0009BB2F6D0A389336833B11A689B88516954
:109000000B4214BF538313830AF1010ABAF1360FDE
:1090100080D140F2E933104802E0002B00F0B1802B
:109020000289013B12F0020F9BB2F6D00823838124
:10903000094940F2E93302E0002B00F0A2800A89DE
:10904000013B12F0010F9BB2F6D08B89024840F22F
:10905000E9330EE060550020003C00408C07002002
:1090600061550020B4B30020F08E0020002B00F0EA
:1090700084800289013B12F0020F9BB2F6D0A0233C
:109080008381484940F2E93301E0002B75D00A8919
:10909000013B12F0010F9BB2F7D08B89414CA02508
:1090A00040F2E93301E0002B5AD02289013B12F053
:1090B000020F9BB2F7D0A58140F2E93301E0002B0B
:1090C0004ED02289013B12F0010F9BB2F7D0A38949
:1090D00040F2E93301E0002B46D02289013B12F037
:1090E000020F9BB2F7D00023A38140F2E93301E0E5
:1090F000002B39D02289013B12F0010F9BB2F7D02F
:10910000A089C0B28306CBD4D8F8003013B11A6856
:109110009B881383234A138823F040031B041B0CF2
:109120001380138823F038031B041B0C138013884F
:109130009BB243F04003002113803970BDE8F88FE3
:10914000204611F06FFE00E7204611F06BFE18E795
:10915000204611F067FE31E7204611F063FE4AE732
:10916000204611F05FFEB3E7204611F05BFEC0B26F
:10917000C8E70C4811F056FE6EE60A4811F052FEA0
:109180008CE7084811F04EFE60E7064811F04AFEF1
:10919000B9E6044811F046FE98E6024811F042FE96
:1091A00077E600BF003C004030B4147874B11E2351
:1091B000074D13FB01012944801A83181D2BD8BFCA
:1091C0000C7012F8014F0131002CF6D130BC704701
:1091D0008C510020F8B5434C434A2388128823F071
:1091E00040031B041B0C23802388C1F1030123F0DF
:1091F000380341EA80071B045208FFB24FEA1343C9
:109200000BD042F48072002A92FAA2F1B1FA81F2F4
:1092100008BF4FF0FF32013AD2001343314A334DB9
:109220009BB2138013889BB243F0400313802B68DA
:1092300013B11A689B8853832A4CBFB2102640F2A0
:10924000E93301E0002B45D02289013B12F0020FE7
:109250009BB2F7D0B3B2A38140F2E93301E0002B17
:1092600038D02289013B12F0010F9BB2F7D0A389BD
:1092700040F2E93301E0002B30D02289013B12F0AB
:10928000020F9BB2F7D0A78140F2E93300E02BB385
:109290002289013B12F0010F9BB2F8D0A38901365D
:1092A000202ECCD12B6813B11A689B8813830D4AEA
:1092B000138823F040031B041B0C1380138823F036
:1092C00038031B041B0C138013889BB243F040032C
:1092D0001380F8BD204611F0A5FDC9E7204611F026
:1092E000A1FDDCE7003C00408C070020F08E002050
:1092F00038B5454B1D7800287BD105F0F70543496B
:109300001D700B88424A23F040031B041B0C12887B
:109310000B800B8823F038031B0452084FEA1343D9
:109320000BD042F48072002A92FAA2F1B1FA81F2D3
:1093300008BF4FF0FF32013AD2001343334A354C95
:109340009BB2138013889BB243F0400313802368C1
:1093500013B11A689B88538340F2E9332B4901E02B
:10936000002B49D00A89013B12F0020F9BB2F7D0C3
:1093700004238B8140F2E933244901E0002B3BD0E8
:109380000A89013B12F0010F9BB2F7D08B891F496C
:1093900040F2E93301E0002B32D00A89013B12F0A0
:1093A000020F9BB2F7D0ADB28D8140F2E93317497D
:1093B00000E02BB30A89013B12F0010F9BB2F8D0F9
:1093C0008B89236813B11A689B8813830F4A13880B
:1093D00023F040031B041B0C1380138823F0380375
:1093E0001B041B0C138013889BB243F040031380B3
:1093F00038BD45F0080582E7044811F013FDC6E7C3
:10940000024811F00FFDDCE7101D0020003C004079
:109410008C070020F08E002038B50B4C23688BB1F0
:109420005A68821A002A054604DA0CE05A68AA1A19
:10943000002A07DB9A68226018461A68904723685A
:10944000002BF3D138BD38BD644700200D4B0421FB
:109450000022890710B4027203F1600402D5197961
:10946000815401329C4203F1180308D0072A06DC1C
:1094700099798907F3D49C4203F11803F6D15DF87A
:10948000044B70477029040810B4104C0423214683
:1094900013F001034FF0000201F1180108D101326D
:1094A000052A0ED08B7913F0010301F11801F6D0D3
:1094B00002EB420204EBC2025DF8044B1379037025
:1094C000704703705DF8044B704700BF70290408B3
:1094D0000123302131224170427103720370037104
:1094E000704700BF436A8269D154436A0169826B45
:1094F00001338B4228BF00234362002A2FD0EFF3B1
:109500001182502383F31288836B1968C9072CD406
:1095100070B45E686EB9456A816A8D4217D08469FD
:109520000C44DC600ED9691A59608562002180F80C
:109530005C10196841F00101D2B2196082F3118800
:1095400070BC70470469611A59608662EEE70123B6
:1095500080F85C30D2B282F3118870BC7047826DA3
:10956000D36843F08003D3607047D2B282F311888E
:10957000704700BF426B10B462B1C36CC2684469EB
:10958000D11A013B615C5DF8044B08BF1346C3640C
:10959000C8B27047016A4369C4685B5C0131A1428B
:1095A00028BF114601625DF8044BD8B2704700BF76
:1095B000836B13B190F85C007047836A406A181A95
:1095C000B0FA80F040097047416A836A99420AD331
:1095D000CB1A816B026961B14968501E0B4483420A
:1095E0000AD2C01A704702691144CB1A816B002954
:1095F000F2D1501EC01A704700207047436B43B130
:10960000C26C5B6893422FBF981AC0689B1AC0183F
:109610007047C269036A9A422FBFD01AC068801887
:10962000C01A70470A4B30B503F1100493F90020BB
:109630005D78072AC8BF143A811804338D7213F875
:10964000025C855413F8012C0A75A342EED130BD9B
:1096500070FC03082DE9F0478C4B1B78DB070746AD
:1096600044D58B4B8B4D1C788B4E012C59D01CD381
:10967000022C07D189498A4A09881288914201D966
:1096800001241C70EB7AE3B12B89D3B1854B1B7895
:10969000BBB112F0B1FF002800F09B802B7B83420E
:1096A0002CBF0121002131700CE07C497E4A0988E1
:1096B00010886A7B801A8842E2DAEB7A0024002B59
:1096C000E2D131782A79632A06D8022C774E00F04D
:1096D000BA803378002B5DD1754AAB7A8C4238BFA3
:1096E0000C461470002B4CD1BDE8F0876B4B694DD4
:1096F00019885B88E878CB1A83EAE3728142A2EB8F
:10970000E3721DD32B788B421AD3614B1C78E01E79
:10971000012861D96749097802294FD0012C5E4E92
:10972000A5D15F4A5D491288687B0988121A914267
:1097300039DD5D4A12888A42A4D200241C70A1E758
:10974000B1EB400FE1DC524B1C78E11E012940F2E5
:109750009480022ADEDC57494F4E0878DFF84481B6
:10976000DFF844C1DFF838E1002103240228347017
:109770001C7088F80010ACF80010AEF8001081D111
:109780001FE0012C71D0022C0BD10720BDE8F0475F
:1097900032F084BC7068381A474B984258DD7270BA
:1097A0009AE7BDE8F08702241C706BE7022AD2DD3D
:1097B0004049097802294FF0040464D13949364EF2
:1097C00009783E48022ACCBF00220122C280818053
:1097D0004BE70221317075E7022A9BDC95F800C047
:1097E00091FBFCFC0CF1010CBCF1080FDFF8B4A0FC
:1097F000304EA87895F801E096F800802A4CDFF802
:10980000A090254EA8BF4FF0080C8AF800C01FFAA0
:109810008CFA10FB0AF01EFB0AFE80B2DFF88CA067
:109820002080A9F800E000244FF0640EB8F1020F88
:1098300034701C70CAF804408AF801E07FF439AF34
:109840000FFA8CF1BDE73078A0B90123776033704F
:10985000C2F164021A4B00FB02F083FB0023C01725
:10986000A0EBA3506430707036E70820BDE8F047E5
:1098700032F014BC7368F81A8EE7032C96D10D49A8
:10988000097802299AD0044EFCE600BFF04B002074
:10989000B828002020770020C8280020144C002081
:1098A000BC2800202A4C0020BA280020C028002014
:1098B000EC7D0020F98E00207F969800FC8E002021
:1098C0006BCA5F6B038A2DE9F0478589ADB21D40F5
:1098D00029D00F4606464FF000484FF00009B5FA70
:1098E00085F328FA03F2D24391B21B3B1540318233
:1098F000042B16D8DFE803F03129211903007B6A15
:10990000002B32D003F1FF3A1FFA8AFAC7F82490ED
:109910003C6A34B123682046514698476468002C5D
:10992000F8D1002DDBD1BDE8F0873868716B036892
:1099300089B29847002DD2D1F5E77868B16B0368FA
:1099400089B29847002DCAD1EDE7B868F16B03687A
:1099500089B29847002DC2D1E5E7F868316C0368F9
:1099600089B29847002DBAD1DDE7F36A1FFA83FA6E
:10997000CEE700BF30B50446806D61718389A2686F
:1099800023F400531B041B0C838185B0A379009240
:1099900013F004022ED04FF4805213F00203ADF8FE
:1099A00004203CD1ADF806304FF480630022ADF8BE
:1099B000083011F00103ADF80C2026D1ADF80A30C3
:1099C00008238A07694648BFADF80A301DF0EEFD4E
:1099D000A379A26D13F0080F938A1BD123F008031B
:1099E0001B041B0C938293899BB243F40053938115
:1099F00005B030BD13F00203ADF8042012D04FF4CF
:109A000000551346ADF80650D0E70423ADF80A30F0
:109A10000C23D6E79BB243F008039382E3E74FF4AD
:109A20000053BFE7ADF80630C0E700BF10B50446ED
:109A3000806DA160838923F400531B041B0C838178
:109A4000A37984B013F00402009133D04FF4805214
:109A500013F00203ADF804203CD1ADF806304FF40A
:109A600080636279ADF80830D1074FF00003ADF89C
:109A70000A30ADF80C3045BF0423ADF80A30082396
:109A80000C236946920748BFADF80A301DF08EFDE1
:109A9000A379A26D13F0080F938A16D123F008035F
:109AA0001B041B0C938293899BB243F40053938154
:109AB00004B010BD13F00203ADF804200DD04FF434
:109AC00000511346ADF80610CBE79BB243F00803F4
:109AD0009382E8E74FF40053BFE7ADF80630C0E7E4
:109AE00008B50121022011F043F8094B1B7803F05F
:109AF0000503052B08D00021012011F039F80021C1
:109B0000084611F035F8FEE724F0A0F8F3E700BFAF
:109B1000843D0020022828BF022010B4084C094BC5
:109B2000207000EB8002C0EBC20207495DF8044BD5
:109B3000013003EB4203C0B20B6032F0D5BB00BF73
:109B4000E0A60020125400208877002008B51AF003
:109B5000FBF811F09DFABDE808401AF0DDB800BF2F
:109B600038B5484B5A899989914224BF00225A81BD
:109B7000198ADA89914224BF0022DA81DA78CAB1DF
:109B8000072A41496AD091F85300404D0124002131
:109B90000A282C709C70D9715DD00C2807D0002A3F
:109BA0006CD0DFED3B7A072A0ED00A2862D0DFEDB9
:109BB000397A09E0344A92F853000A2856D00C2822
:109BC0005BD1D979DFED347A344C9FED350AA27838
:109BD000002918BFF0EE407A062A04D8314901EB7B
:109BE000820191ED040A217979B1013A032A0BD857
:109BF000F7EE007A87EE800A35F00EF82388984257
:109C000028BF1846208038BD38BD9B781F4A07EE14
:109C1000103A1178B8EEC77A67EE277A07EE101A75
:109C2000B8EEC77A27EE277AB4EEC70AF1EE10FA3B
:109C3000EADD80EE277AFDEEC77A17EE903A102B18
:109C4000A8BF1023012BB8BF0123DBB28B4238BF62
:109C50000B46137038BDDFED147AA4E791F853007A
:109C60000A2803D00C28ACD0D9799AE7D979DFED4E
:109C70000E7AA9E7DFED0D7AA6E7D979DFED047A50
:109C8000A2E700BF48A900205CA90020FC4A0020F0
:109C90006F1203396F12833A0AD7A3391057002085
:109CA0006F12033870FC03085304E9380F506E3A02
:109CB0002DE9F047AC4FAD4E1AF046F8BE421ED229
:109CC000DFF82483DFF824934446258862197DB1A8
:109CD0004A450DD2052D0BD933886188C3F30B0398
:109CE000994200F0E380144625886219002DEFD1D7
:109CF00071683046143611F057F9BE42E4D39C4ADD
:109D00001378A3F1170102290FD99A4911F83300EA
:109D1000002840F0FA80D8000144497829B19649DA
:109D200011F833300BB918231370944B5A78022A68
:109D300000F2DC809249934802EB420201EB82017F
:109D40001A780160022A00F2DA8002EB82018E4B5F
:109D5000C2EBC10203EB4203998C5A8C8B4C9142AB
:109D6000236001D300225A84894B9A78042A00F098
:109D7000ED8032B91A88B2F5F07F84BF4FF4F072EB
:109D80001A80844DFFF7ECFE2B68834A1A40002AA4
:109D900000F0E580D80700F1D480590400F1CC80B0
:109DA0001A0700F1BB809B0400F1BF802DF066FA1A
:109DB00010B97A4812F0B0F9402011F02BF94FF4A5
:109DC000007011F027F94FF4003011F023F94FF42F
:109DD000001011F01FF94FF0007011F01BF94FF057
:109DE000806011F017F924F005FC002130226C4846
:109DF00035F0CFFE206823F05FFB6A4B256803F146
:109E0000500102E0043399427DD01A78002AF9D13A
:109E10009C78D8788442F5D26349644B0A7028460E
:109E20001D6020F0C1FD624A62491079624A634BAD
:109E30001160C822642111FB0021002259609A6040
:109E4000DA601A615A619A61DA6183F8202083F836
:109E500021201FF09BFA5A4B9FED5A5A1B885A4AF1
:109E60009FED5A6A50795A4906EE903AF8EEE66A42
:109E70001388C5EE265A07EE103A53881279C1EDC1
:109E8000005A07EE903AB8EEC77A524BF8EEE77AEE
:109E900018725A7227EE067A67EE867ABDE8F047A6
:109EA00083ED017AC3ED007A19F036BF63799B0721
:109EB0007FF419AF716894F804A0304611F074F87B
:109EC0003388BAEB133F04D01436BE42FFF4FCAE25
:109ED00015E773887068AA1FC3F30B039A4204F155
:109EE0000601A8BF1A4634F0C1FCEDE700225A7003
:109EF0001A78244822490160022A7FF626AF002200
:109F00001A70214B28E7012286E7D8000C186468F4
:109F1000002C7FF401AF17241470FDE62E4811F0D9
:109F200079F82B689B047FF541AF2C4811F072F84B
:109F3000402011F06FF839E7294811F06BF82B68D1
:109F40002EE7284811F066F82B6826E79A8AB2F5C2
:109F50007A7FBFF416AF4FF47A729A8211E743F01A
:109F600008032B6016E700BF0406000890010008F4
:109F7000CC4D0020F81F040830060408E0A600209D
:109F80001E5500208C770020125400208877002076
:109F9000105700205C550020096000023095002019
:109FA0003C250020C8470020291B002070250020E8
:109FB0008C7400200E4B0020842500208C7900201A
:109FC00050270020C0C9FB488024002017B7D13893
:109FD00054270020F46E00200160000209400002B6
:109FE000092000020860000202400008008000080A
:109FF00008B519F0A9FE11F04BF819F08DFEFFF726
:10A0000057FE0120BDE8084032F06EB970B50F4C24
:10A010000F4DAC4206D261682046143410F0C4FFE4
:10A02000AC42F8D30B4B0C4D0C4C0D4A0D4E1E6040
:10A03000002301260C492E70A371137053700B4836
:10A040000860BDE8704026F093BD00BF9001000895
:10A050000406000888770020753E00201C4C002074
:10A06000E0A60020125400208C7700201E5500200E
:10A0700008B5FFF7CBFF19F067FE11F009F8BDE84E
:10A08000084019F049BE00BFF0B50C2934D8DFE80C
:10A0900001F0893333335E333333343333330700E2
:10A0A000048C9689B2F802E01788734D24F480542A
:10A0B0002404240C0484038C8488818B23F40053AF
:10A0C00021F4E6411B0409041B0C46EA0E06090CA8
:10A0D00043EA063341EA0721A8429BB2A4B289B2FF
:10A0E00000F09E8005F58065A84200F09980926896
:10A0F0008480818302640384F0BD048C9589B2F866
:10A1000002C0B2F800E05C4F24F480742404240CF4
:10A110000484038C8688818B23F400731B0421F054
:10A1200073011B0C45EA0C04090443EA0423090CDF
:10A13000B8429BB2B6B241EA0E015CD04F4CA0428D
:10A1400059D0926886808183C2630384F0BD048CF9
:10A150009589B2F802C0B2F800E0474E24F010042E
:10A160002404240C0484038C8788018B23F02003AF
:10A1700021F4E6411B0409041B0C45EA0C04090CFC
:10A1800043EA041341EA0E21B0429BB2BFB289B246
:10A190005DD03A4CA0425AD0926887800183826396
:10A1A0000384F0BD048C9789B2F802E01688324D22
:10A1B00024F001042404240C0484038C8488018B7F
:10A1C00023F002031B0421F073011B0C47EA0E0766
:10A1D00009043B43090CA8429BB2A4B241EA060120
:10A1E00025D005F58065A84221D09268848001833E
:10A1F00042630384F0BDD589148A578A23F400632F
:10A2000043EA05254FF6FF332B40958826F4405648
:10A210003C4343EA052346EA04169BB2B6B290E7F4
:10A22000158A24F4804444EA8514A4B25FE7D689F1
:10A23000158A578A23F00803334324F44074968820
:10A240003D4323F004032C433343A4B2CDE7D48928
:10A25000158A568A23F0800343EA04134FF6BF742D
:10A260001C40938827F44067354344EA031347EAC8
:10A2700085079BB2BFB28FE7000001400004014098
:10A280002DE9F04F7822002183B0C248C24CDFF89C
:10A290002493C24DC24EC34FDFF81C8335F079FCC6
:10A2A000C148C249DFF814E3DFF814C30022A35801
:10A2B000834200F0D481B3F1804F00F0D281AB42F1
:10A2C00000F0D181B34200F0D081BB4200F0CF81D9
:10A2D000734500F0CE81634500F0CD81434500F029
:10A2E000CC81DFF8E0A2534500F0C9810AF5806A0D
:10A2F000534500F0C6810AF5806A534500F0C381DA
:10A30000AAF5983A534500F0C0810AF5806A534592
:10A3100000F084810AF5806A534508BF0D2300F0E0
:10A320007E811832782AC2D1252010F0C3F9002886
:10A330003FD001689E4C01F13F4303F57E039A0A2A
:10A340000123A25C02F01F045209032A03FA04F35A
:10A3500000F09D81042A00F0B881022A03D1934ABB
:10A36000546C2343536483880093B3FA83F3C3F19B
:10A370001F039BB2DA0801EB820203F00703106AA5
:10A380009B000F249C4020EA04001062106A022403
:10A3900004FA03F3034313620846002369468DF869
:10A3A00004408DF805308DF806308DF807301DF02B
:10A3B00049FA202010F07EF900283FD001687C4C3B
:10A3C00001F13F4303F57E039A0A0123A25C02F0E8
:10A3D0001F045209032A03FA04F300F06C81042AD3
:10A3E00000F07D81022A03D1704A546C23435364E8
:10A3F00083880093B3FA83F3C3F11F039BB2DA0897
:10A4000001EB820203F00703106A9B000F249C40BB
:10A4100020EA04001062106A022404FA03F30343E2
:10A4200013620846002369468DF804408DF8053014
:10A430008DF806308DF807301DF004FA232010F057
:10A4400039F9002840D00168594C01F13F4303F528
:10A450007E039A0A0123A25C02F01F045209032A18
:10A4600003FA04F300F02281042A00F03D81022A5D
:10A4700003D14E4A546C2343536483880093B3FA48
:10A4800083F3C3F11F039BB2DA0801EB820203F0EE
:10A490000703106A9B000F249C4020EA040010620E
:10A4A000146A012000FA03F32343136208460023D1
:10A4B000022269468DF804208DF805308DF80630AB
:10A4C0008DF807301DF0BEF9212010F0F3F80028B8
:10A4D0003FD00168364C01F13F4303F57E039A0AF1
:10A4E0000123A25C02F01F045209032A03FA04F3B9
:10A4F00000F0D780042A00F0ED80022A03D12B4A15
:10A50000546C2343536483880093B3FA83F3C3F1F9
:10A510001F039BB2DA0801EB820203F00703106A03
:10A520009B000F249C4020EA04001062106A022461
:10A5300004FA03F3034313620846002369468DF8C7
:10A5400004408DF805308DF806308DF807301DF089
:10A5500079F9182010F0AEF800285CD0046814498E
:10A5600004F13F4303F57E039A0A01238A5C02F05B
:10A570001F015209032A03FA01F300F08D80042A17
:10A5800000F09E80022A1FD1084A516C0B4353648D
:10A590001AE000BF348E0020702904080004004037
:10A5A00000080040000C004000000140003802405C
:10A5B00038290408902804080004014000100040D5
:10A5C000001400400040014083880093B3FA83F3F5
:10A5D000C3F11F039BB2DA0804EB820203F0070306
:10A5E000116A9B000F20984021EA00011162106A55
:10A5F000012101FA03F303431362204600230222E0
:10A6000069468DF804208DF805308DF806308DF8F8
:10A6100007301DF017F903B0BDE8F08F0C2309EBEC
:10A62000C3034FF0010A1B7903F01F0B5B09032BD7
:10A630000AFA0BFA0ED0042B07D0022B7FF471AE6E
:10A640004B6C4AEA03034B646BE60B6B4AEA030369
:10A650000B6366E60B6C4AEA03030B6461E60023B6
:10A66000DDE70123DBE70223D9E70323D7E7042350
:10A67000D5E70523D3E70623D1E70723CFE7082350
:10A68000CDE70923CBE70A23C9E70B23C7E7194A1C
:10A69000146C2343136466E6164A116C0B4313646F
:10A6A00092E7144A146C234313642CE7114A146C88
:10A6B00023431364E1E60F4A146C2343136497E6C3
:10A6C0000C4A116B0B4313637EE70A4A146B234356
:10A6D000136348E6074A146B2343136313E7054AE1
:10A6E000146B2343136383E6024A146B23431363FF
:10A6F000C3E600BF0038024001490248FFF7E2B854
:10A70000848E00200004004002494FF08040FFF793
:10A71000D9B800BF5C8E002001490248FFF7D2B8CB
:10A72000348E00200000014001490248FFF7CAB8FA
:10A73000348E002000000140F0B504683F4DA30AAC
:10A74000AB425CD03F35AB4255D0B3F5801F00D053
:10A75000F0BD4FF0480E01264779B0004FEA970C44
:10A76000002956D063460227A5899F4083190CEB28
:10A7700043032F4303F1040C314DBFB245F82310BE
:10A7800045F82C20A781EFF31181502282F3128823
:10A79000821905EBC202136953B3136204338219A1
:10A7A00005EBC202576917B11F6053690433821960
:10A7B00005EBC202976917B11F60936904338219D0
:10A7C00005EBC202D76917B11F60D36904330027B4
:10A7D000CAB21F6082F31188304405EBC000036ADF
:10A7E0008BB9A38923F001031B041B0CA381F0BDCB
:10A7F00005EB0E03D3E74FF0200E0026ACE74FF039
:10A80000700E0226A8E7A3899BB243F00103A3813F
:10A81000F0BD0223BF0803FA07F7A389084D9BB2D6
:10A8200023EA070387190CEB470CA3810CF10403FF
:10A8300045F82C1045F82320A5E700BF01001000C3
:10A84000348E00202B4B98423CD0B0F1804F3BD04F
:10A85000A3F57C43984239D003F58063984237D002
:10A8600003F58063984235D003F58063984233D076
:10A8700003F58063984231D003F5704398422FD09E
:10A8800003F5705398422DD003F5806398422BD086
:10A8900003F58063984229D0A3F59833984227D0D6
:10A8A00003F58063984207D003F58063984208BFA0
:10A8B0000D2202D0002070470C220F4B03EBC20385
:10A8C000187970470022F8E70122F6E70222F4E740
:10A8D0000322F2E70422F0E70522EEE70622ECE786
:10A8E0000722EAE70822E8E70922E6E70A22E4E786
:10A8F0000B22E2E700000140902804082DE9F04F08
:10A90000013085B0C3B203930B4602918B4C8C4E41
:10A91000002B00F09A8032208A4D8B4FDFF82C926A
:10A9200031F01EFA4FF4FA7A4FF0100C4FF47A70AF
:10A93000D9F80430C3F30803002B40F0DE80EFF3B6
:10A940001183002B40F0D9802968A26800BF2B68D2
:10A950009942F9D1D7F800E000FB0EF39B1AB3FB44
:10A96000FEF300FB01314FF0010E0191D9F80430E4
:10A97000C3F30803002B40F08780EFF31183002B13
:10A9800040F082802B68A16800BF2A689342F9D109
:10A99000D7F800B000FB0BF2521AB2FBFBF200FB3F
:10A9A0000323019A9B1AB3F57A7FDFD3BAF1010A28
:10A9B000BED1039B002B40F0BD804FF47A7ADFF8C4
:10A9C0008C9150464FF0100CD9F80430C3F30803B3
:10A9D000002B75D1EFF31183002B71D12968A26888
:10A9E00000BF2B689942F9D1D7F800E000FB0EF3C5
:10A9F0009B1AB3FBFEF300FB01314FF0010E0191F6
:10AA0000D9F80430C3F3080313BBEFF31183FBB988
:10AA10002B68A16800BF2A689342F9D1D7F800B02B
:10AA200000FB0BF2521AB2FBFBF200FB0323019A6C
:10AA30009B1AB3F57A7FE3D3BAF1010AC4D1029B22
:10AA4000013B0293002B7FF466AF05B0BDE8F08FA9
:10AA5000EFF311888CF31288A1682368DB0344BFED
:10AA6000C6F800E0A1682B6832685FFA88F888F3BE
:10AA70001188D7F800801A4400FB08F35B1AB3FB77
:10AA8000F8F300FB0233D2E7EFF311888CF312885E
:10AA9000A1682368DB0344BFC6F800E0A1682B6807
:10AAA00032685FFA88F888F31188D7F800801A4472
:10AAB00000FB08F35B1AB3FBF8F300FB023370E70B
:10AAC000EFF311828CF31288D4F808E02368D903DD
:10AAD00003D501233360D4F808E02B683168D2B283
:10AAE00082F311883A68194400FB02F3A3EB0E03CA
:10AAF000B3FBF2F300FB01317FE7EFF311828CF33C
:10AB00001288D4F808E02368D90303D50123336001
:10AB1000D4F808E02B683168D2B282F311883A6821
:10AB2000194400FB02F3A3EB0E03B3FBF2F300FBAB
:10AB3000013118E7184630F095FF3EE710E000E0DD
:10AB4000E4B30020E8B30020ECB3002000ED00E007
:10AB5000204B5B68C3F3080330B4BBB9EFF3118338
:10AB6000A3B91D4B1D4C1868A16800BF1A6890421C
:10AB7000F9D11B4B1C684FF47A7202FB04F3591A8B
:10AB8000B1FBF4F130BC02FB00107047EFF311820F
:10AB9000102383F3128811498C680B6813F4803FEB
:10ABA000104B02D0012018608C680B49D2B20D689E
:10ABB000186882F311880A4B19684FF47A72284496
:10ABC00002FB01F31B1B30BCB3FBF1F302FB0030B3
:10ABD000704700BF00ED00E0E8B3002010E000E0A7
:10ABE000ECB30020E4B300202DE9F84F8046FFF7D6
:10ABF000AFFF254E2549DFF8A0E0254A254D8446C4
:10AC000010274FF47A740120DEF80430C3F30803F0
:10AC1000D3B9EFF31183BBB90B68D2F808A000BF1A
:10AC2000D1F800904B45F7D1D6F800B004FB0BF9F2
:10AC3000A9EB0A09B9FBFBF904FB0393A3EB0C0393
:10AC40004345E1D3BDE8F88FEFF3118A87F312880B
:10AC5000D2F808B01368DB0344BF2860D2F808B00C
:10AC60000B68D5F800905FFA8AFA8AF31188D6F853
:10AC700000A0994404FB0AF3A3EB0B03B3FBFAF324
:10AC800004FB0933DAE700BFECB30020E8B300208F
:10AC900010E000E0E4B3002000ED00E02DE9F04F0B
:10ACA000DFF830C1474A4849484E494D8046102791
:10ACB00018F1FF38C0F08480DCF80430C3F30803D7
:10ACC000002B5CD1EFF31183002B58D10B689468F3
:10ACD00000BF08688342F9D1D6F800904FF47A702B
:10ACE00000FB09FEAEEB040EBEFBF9FE00FB03EE1B
:10ACF000DCF80430C3F308034FF47A740120FBB985
:10AD0000EFF31183E3B90B68D2F808A000BFD1F8C4
:10AD100000904B45F7D1D6F800B004FB0BF9A9EB36
:10AD20000A09B9FBFBF904FB0393A3EB0E03B3F58C
:10AD30007A7FBDD2DCF80430C3F30803002BDFD0E8
:10AD4000EFF3118A87F31288D2F808B01368DB0397
:10AD500044BF2860D2F808B00B68D5F800905FFABD
:10AD60008AFA8AF31188D6F800A0994404FB0AF302
:10AD7000A3EB0B03B3FBFAF304FB0933D5E7EFF3C3
:10AD8000118487F31288D2F808901368D80303D58A
:10AD900001232B60D2F808900B682868E4B284F392
:10ADA0001188D6F800A04FF47A7400EB030E04FB70
:10ADB0000AF3A3EB0903B3FBFAF304FB0E3E97E798
:10ADC000BDE8F08F10E000E0E8B30020ECB3002015
:10ADD000E4B3002000ED00E030B4EFF31183102263
:10ADE00082F312880649074C0A6807480132002599
:10ADF0000A602560DBB2026883F3118830BC7047BB
:10AE0000E8B30020E4B3002010E000E00F4B1B8803
:10AE1000014643B90E4B0F4A1B7810680BB981F0FD
:10AE200001010FF09DBE0C4B5A691AB118B91A688E
:10AE3000106058747047094A18681188084A92FBD4
:10AE4000F1F2012102605974704700BFC0B30020C5
:10AE5000C2B30020C4B30020C8B30020E0B3002078
:10AE600020A1070038B5264B1C69636B73B1A36D35
:10AE7000A26BD2B1998A1A88C90592B201D5D207BC
:10AE800000D438BD4FF6F7721A8038BDA36D99898A
:10AE90001A88890692B2EBD59206E9D5E26AD2B158
:10AEA0009888216B80B29047E1E799891A880D064E
:10AEB00092B2DFD51006DDD5A26A616A8A4219D046
:10AEC000A1692569885C98800132B2FBF5F105FB28
:10AED0001122A262CEE79B88E2696169DBB28B54E2
:10AEE000E269E068A36D0132B2FBF0F100FB1122D0
:10AEF000E261BDE7DA6822F08002DA60BAE700BFFB
:10AF0000883D002038B5264BDC68636B73B1A36DB8
:10AF1000A26BD2B1998A1A88C90592B201D5D2071B
:10AF200000D438BD4FF6F7721A8038BDA36D9989E9
:10AF30001A88890692B2EBD59206E9D5E26AD2B1B7
:10AF40009888216B80B29047E1E799891A880D06AD
:10AF500092B2DFD51006DDD5A26A616A8A4219D0A5
:10AF6000A1692569885C98800132B2FBF5F105FB87
:10AF70001122A262CEE79B88E2696169DBB28B5441
:10AF8000E269E068A36D0132B2FBF0F100FB11222F
:10AF9000E261BDE7DA6822F08002DA60BAE700BF5A
:10AFA000883D002038B5264B5C68636B73B1A36D98
:10AFB000A26BD2B1998A1A88C90592B201D5D2077B
:10AFC00000D438BD4FF6F7721A8038BDA36D998949
:10AFD0001A88890692B2EBD59206E9D5E26AD2B117
:10AFE0009888216B80B29047E1E799891A880D060D
:10AFF00092B2DFD51006DDD5A26A616A8A4219D005
:10B00000A1692569885C98800132B2FBF5F105FBE6
:10B010001122A262CEE79B88E2696169DBB28B54A0
:10B02000E269E068A36D0132B2FBF0F100FB11228E
:10B03000E261BDE7DA6822F08002DA60BAE700BFB9
:10B04000883D002038B5264B1C68636B73B1A36D37
:10B05000A26BD2B1998A1A88C90592B201D5D207DA
:10B0600000D438BD4FF6F7721A8038BDA36D9989A8
:10B070001A88890692B2EBD59206E9D5E26AD2B176
:10B080009888216B80B29047E1E799891A880D066C
:10B0900092B2DFD51006DDD5A26A616A8A4219D064
:10B0A000A1692569885C98800132B2FBF5F105FB46
:10B0B0001122A262CEE79B88E2696169DBB28B5400
:10B0C000E269E068A36D0132B2FBF0F100FB1122EE
:10B0D000E261BDE7DA6822F08002DA60BAE700BF19
:10B0E000883D002070B4EFF31186502383F312885B
:10B0F000836B1A68D20720D45D686DB9446A826A8E
:10B10000944217D081691144D9600ED9A21A5A60AD
:10B110008462002280F85C201A6842F00102F1B2D9
:10B120001A6081F3118870BC704701698A1A5A60ED
:10B130008562EEE7012380F85C30F3B283F3118877
:10B1400070BC704703685B6A03B11847704700BF63
:10B1500003681B6A03B11847704700BF2DE9F04F21
:10B16000BB4B1E788FB0002E7ED1BA4BBA4C1D78E7
:10B17000DFF8088305F00105A4F10A0B54F80A0C66
:10B18000B0B1CC2707FB06B70FF0E4F880B154F854
:10B190000A0C0FF0DBF814F8023C024683B92428AD
:10B1A0003BD075B354F80A0C0FF0D4F80028EED158
:10B1B0000136032E04F1CC04E0D10FB0BDE8F08FCE
:10B1C000012B2ED0022B33D0032B40D0042B00F0C8
:10B1D0006881052B00F05681062BE3D114F8019C01
:10B1E000B9F1000F00F0DA81B9F1010F00F013821C
:10B1F00001360023032E04F8023C04F1CC04BDD137
:10B20000DBE7232A54F80A0C00F08181934B93F872
:10B210002A309342B8D132F047FA012304F8023CB5
:10B22000C0E74D2800F06681002304F8023CB9E72E
:10B2300000233C2804F8023C00F056813E28B1D19E
:10B240000122032304F8012C04F8023CAAE7C028D9
:10B25000EAD80021042304F8050C04F8040C04F8CF
:10B26000061C04F8023C9DE77D4B18680028A4D01A
:10B270000FF0FAFDDFF808A27A4DDFF8F891DAF85E
:10B2800000000FF067F8002897D0DAF800000FF000
:10B290005DF809281BD03F2819D02B68002B67D1F7
:10B2A000042800F0B0810C2800F0CA807F28E6D086
:10B2B000A0F12002D2B25E2AE1D80BB92028DED05C
:10B2C0005A1C09F803002A6014F0F6F8D7E72C6836
:10B2D000002C5AD1644FA34607F51878BBF1000F34
:10B2E00008BFBB4610374745F8D1BBF1000F00F04F
:10B2F0005081103FDBF800003A68065D135D9E4206
:10B30000204402EB040140F04281661E4E44224676
:10B310000BB9FD2A5CD906F8013F01322A6010F80A
:10B32000013F11F801EF9E45F2D00AB15F4512D0FE
:10B330004E4814F0C9F85F4508D35BF8100B14F0C1
:10B34000C3F8092014F0B8F8BB45F6D9484814F002
:10B35000BBF82A680024944291D2661E4E4416F827
:10B36000010F14F0A9F82B6801349C42F7D386E74B
:10B370000C2865D00A2834D00D2832D07F2800F060
:10B38000BD80FF2B3FF67BAF92E7374E002706F5D7
:10B390001878BB4602E0103646450DD0224631688B
:10B3A000484610F0C1F80028F5D1B346002FF2D17D
:10B3B000374610364645F1D13B465F469B46002B4B
:10B3C00098D1002F3FF45BAF284814F07DF8B4E724
:10B3D000511C202009F80200296009F801300A46B2
:10B3E000A4E714F0F2F82321224834F0E9FB002806
:10B3F00000F00781A0EB0900286090B1431E19F806
:10B400000310202940F0058109EB030243B112F833
:10B41000011D202903F1FF304ED10346002BF6D148
:10B420002B604FF480720021484634F0B2FB084B89
:10B430001B78002B3FF4C1AE0D4814F045F81EE711
:10B440000D4814F041F80A4814F03EF817E700BF21
:10B450008C440020F04B002036290020309500203D
:10B46000504100208844002020010408F82B0408E3
:10B47000002C040888430020082C040858210020D0
:10B480008443002014F8063C14F8051C994273D834
:10B4900014F8043C83427FF4C7AE062304F8023C50
:10B4A0009CE614F8043C04F8030C5A40052304F805
:10B4B000042C04F8023C75E62B60C44C002204F511
:10B4C000187809F8032002E01034444550D0216870
:10B4D000484617F083F80028F6D0444548D2E36880
:10B4E000984700232B609CE7032204F8013C04F8F2
:10B4F000022C57E6022304F8023C53E6013B0022EB
:10B50000B3482B6009F8032013F0DEFFB7E6B14B18
:10B51000B149DB78B14ADFF8F4E21060003318BFBC
:10B5200001230B70AE4BAF4ACEF80030AE4BC8F8DB
:10B5300004204FF0400E012188F80CE0C8F800000C
:10B54000C8F8080088F80D50A848197014F088FC55
:10B55000A74813F0B9FF4FF400600DF0B5FBA54B01
:10B5600093F82A30232B3FF456AE14F8023C33E60E
:10B57000A14813F0A9FFB4E714F8041CF8185140CF
:10B58000013304F8041C04F8063C82720AE62246E1
:10B59000CBE69A48103F13F097FFCEE6984B14F88D
:10B5A00003CC0A940FCB0DF1380E06AF87E80F00DD
:10B5B0004EF82C9D14F8053CADF8329039462344E2
:10B5C000012772460AA80B93ADF830C08DF834708D
:10B5D00002F06CFE00283BD1039F002304F8023CDC
:10B5E000002F3FF4E5AD54F80A0C11F035FA01369E
:10B5F00054F80A0CB847032E04F1CC047FF4BEAD16
:10B60000DBE52868F9E67F4815F0B4FF0FB0BDE828
:10B61000F08F034651E714F8053C14F8032C0A9404
:10B6200023440B936E2A4FF000030C930D93ADF857
:10B6300030207FF4DDAD0AA80FF0F8FF0AA80FF064
:10B64000E9FF0AA80FF0E6FF0AA80FF0E3FFCFE535
:10B65000069A6D4B54F80A0C07920693FFF778FD93
:10B66000069A079FBDF92230CDF81490BF1AFF2F1C
:10B670004FF0240239468DF81020A8BFFF214D223B
:10B6800001338DF8112000F09F809DF82430002BAD
:10B6900014BF3C233E23BDF820208DF81230FE2F2E
:10B6A0008DF813108DF8142040F38A803B128DF82A
:10B6B00015708DF816304FF00309072204A954F8CD
:10B6C0000A0C0EF017FE09F101099DF813309DF8E0
:10B6D0001420B9F1020F83EA02030AD09DF8152065
:10B6E000B9F1040F83EA020303D19DF816205340F9
:10B6F000DBB2002F8DF80B3056DD3A46069954F830
:10B700000A0C0EF0F7FDA7F1040E4FEA9E0E791E0B
:10B710000EF1010E06294FEA8E099DF80B30069AAC
:10B720001FDD4FF0000C6046924601935AF8043B2F
:10B730000CF1010CE64580EA0300F7D8019BC0F349
:10B74000072E80EA0E0E83EA0E03C0F3074E83EA4B
:10B750000E0383EA1063B9454A44A1EB0901DBB249
:10B7600020D01078002983EA00031BDD50780129DE
:10B7700083EA0003DBB215DD9078022983EA000337
:10B7800010DDD078032983EA00030BDD107904294A
:10B7900083EA000306DD5079052983EA000301DD11
:10B7A000927953408DF80B3054F80A0C01220DF1B8
:10B7B0000B010EF09FFD54F80A0CFFF7C3FC0BE7DA
:10B7C0004FF00109052279E7212364E720010408ED
:10B7D000302C0408E0A60020242900208443002007
:10B7E0005C210020FD9C01088C440020342C0408BE
:10B7F000002C040830950020142C0408F82B0408B1
:10B800009CFC03088843002014B400205041002011
:10B810002DE9F04F2DED028B93B0054624F08CF806
:10B82000994B1E7826B113B0BDEC028BBDE8F08FAA
:10B83000964B1B685805F6D5DFF89C82D8F8002097
:10B84000002A00F01E81924CD4F8283103F5F4331D
:10B8500048339D42C0F015818E4F94F82C313968E1
:10B86000C4F828510133DBB2890784F82C3101F187
:10B87000ED8513F0070901F02B85282B864B0293E9
:10B8800001F026875E209047844B1B78002B6BD0FD
:10B890007F4C834AD4F83431EB1A934201F2D683B9
:10B8A000DFF838A29AF80080B8F1000F33D1DFF842
:10B8B0000092D9F800000EF04DFDC0B201280ED95B
:10B8C0000228784F41F0C4873B78002B42F01D815D
:10B8D000D4F83C31EB1AB3F57A6F82F07B81724871
:10B8E0000768002F40D09AF80030BBB96F4BD9F8E9
:10B8F00000001B689B781E3B012B4FF0020142F2B7
:10B900001481043023F0D0FE012200238AF80020A5
:10B9100084F8483126E0644807682FB3D4F84431EE
:10B9200040F6B732EB1A93421ED994F84031002BFF
:10B9300001F08487013BDBB284F84031002B01F039
:10B94000F28517F8011B94F84821076094F84931F3
:10B9500057480A440133006884F8482184F8493183
:10B960000EF0FCFCC4F84451524A029B12781B684A
:10B97000012A03F101030A9301F092824E4B1B78D6
:10B980007BB1DFF85C81D8F8003053B1029B404CAA
:10B99000D3F800B0D4F85C31ABEB0303632B01F2B6
:10B9A000BC81DFF8408198F800A0BAF1020F01F0E5
:10B9B00096853C4F97F87430032B01F050843F4B31
:10B9C0001B7873B13E4E33685BB1314CFFF7C0F862
:10B9D000D4F86831039044F61F62C31A934200F210
:10B9E0002581384B1B78002B7ED1374B1B7843B118
:10B9F000274CD4F8B83203F50043E8339D4281F078
:10BA0000C582324B1B78002B3FF40DAF204E304CDB
:10BA1000304D06F2C12720680EF09CFC00283FF450
:10BA200002AF20680EF092FC2B7880465A1E33B18C
:10BA300020682A700EF08EFC0028F2D1F3E6032273
:10BA40003946781E34F08BF896F8C03296F8C12249
:10BA500086F8C38283F47F4383F0FF039B1A1FFAA7
:10BA600088F89BB2B8EB132FD5D196F8C222DBB27F
:10BA70009A42D0D1781E1CF049F82B7818442870CF
:10BA8000C9E7054B0293FFE68C44002048B1002033
:10BA9000A821002030770020E8B300203A78002069
:10BAA0003F0D030004000020A07700209C770020B9
:10BAB000987700203B7800204878002050780020BC
:10BAC00054780020C0780020D17800205A780020D7
:10BAD0006078002064780020A8770020A4770020F8
:10BAE000187700204E470020444C2278002A41F06D
:10BAF000CE81DFF8349199F80040002C72D1404E8D
:10BB00003078002841F08C873E4C3F4ED4F8B0226C
:10BB100031783E4B93FBF1F313449D42FFF465AF44
:10BB200094F8B4323A4AC4F8B052D75CFB0702F139
:10BB30006781B80702F1B080790702F16D803A079A
:10BB400045D5344B344F0B930DF14809A3F13D0219
:10BB500049F8202D0021A3F1400203F8401C0223E4
:10BB6000112151709370484639680FF06FFD4846B7
:10BB700079680FF06BFDFB89284903EBC3039B0039
:10BB8000053381FB0321DB17C3EBA10189B24846D2
:10BB90000FF074FD3B8A03EB8303590089B24846DA
:10BBA0000FF06CFD1E4B1B789B0743BF398901F5D5
:10BBB0007A7189B24FF47A7148460FF05FFD0A9BA3
:10BBC0003A7D591C0A9148461A7023F05BFE94F89E
:10BBD000B4323178013393FBF1F201FB123384F874
:10BBE000B43202E70F4E376E002F41F02585054B2A
:10BBF00089F80070C3F8B052F7E600BF2C78002037
:10BC0000C8780020A8210020D0780020A08601005C
:10BC1000CC780020EC770020B85A00206766666672
:10BC200086770020D8780020C978002094F86E31FB
:10BC3000002B41F08084DF4B1B6803F00802002AD0
:10BC400048F603414AF60B404BF60F4249F60747C8
:10BC500004BF02460F4613F0040F4FF0190118BF3E
:10BC600017469B0684F86E1103D547F4804747F0CA
:10BC7000200710F0B3FCC7F30909002842F0C78180
:10BC8000CD4B9B79002B42F04F82984664204FF0B9
:10BC9000FF3A4FF0000C0A970B97ADF834C0CDF87F
:10BCA0003AC0CDF83EC0CDF842C0CDF83090ADF8E6
:10BCB0003680ADF838A08DF846000AAF0FCFDFF818
:10BCC00008E384F805C0AEE80F0097E80F00AEE87F
:10BCD00007002EF8023B71464FF0010C1B0CFE27AB
:10BCE0001F20C82201F81E39A770A27184F807C06E
:10BCF000E07094F87E01207180F0F10383EA031371
:10BD0000DAB2130983F0E70343EA022383EAC203AA
:10BD10001BB283EA0312D2B2C3F3072383EA1213DE
:10BD200043EA022383EAC2031BB283F0C80282EA19
:10BD30000212D2B2C3F3072383EA121343EA0223A7
:10BD400083EAC2031BB283EA0C0787EA0717FFB234
:10BD5000C3F3072282EA171242EA072200EB0C0320
:10BD600082EAC7070EEB0C0084F87E31278011F8B9
:10BD7000013B7B4083EA0313DBB21A0982EA1722F4
:10BD800042EA032282EAC3031BB29FB281422780A8
:10BD9000EDD183F07C0383EA0313DBB24FEA131E79
:10BDA0008EEA172E8EEA032E8EEAC30E0FFA8EFE4F
:10BDB0001FFA8EF9DFF814C2A4F800905FFA8EFE25
:10BDC0004FEA192984F8289084F827E00CF5D378F5
:10BDD00004F1220ADCF80000DCF80410DCF808208A
:10BDE000DCF80C3047460FC70CF1100CD445B846B0
:10BDF000F0D1DCF800003860704F9CF8043088F80F
:10BE0000043007F1270884F8CDE184F8CE9117F8C3
:10BE1000011F30680EF0A2FAB845F8D194F86F21EE
:10BE2000002A41F0F4836649029B08781B680A21C6
:10BE300084F86F11002801F02C85DFF894E10128C7
:10BE4000BEF80010059142F2FE810228BEF8028081
:10BE500002F0F580BEF804100491032802F00E826F
:10BE60000428BEF806A002F004820528BEF8087077
:10BE700002F0FB810628BEF80AC002F0F381072811
:10BE8000BEF80C1001D0BEF80E2094F87EB10A93D3
:10BE90008BF0300383EA0313DBB24FEA131E4948E9
:10BEA00084F804B08EF07A0E4EEA032E00888EEAF3
:10BEB000C303DFF820E1C0EB00208EFB009E864428
:10BEC000C0171BB2C0EB6E200690C3F3072E83EAA7
:10BED0000310059BC0B24FF0000963F30F098EEA0F
:10BEE000101305934FF0000E049B68F31F4967F38E
:10BEF0000F0E4FF00008002763F30F0861F30F07E0
:10BF0000059BCDF82C906CF31F4E62F31F474FF04A
:10BF1000000C9DF81820CDF834E06AF31F48CDF8E6
:10BF200030800E978DF83CC08DF83D2043EA002309
:10BF30000DF1280883EAC007B8E80F003FB287F088
:10BF4000C80989EA0919DFF880E084F805C05FFABA
:10BF500089F9C7F30727AEE80F0087EA191747EA00
:10BF6000092398E8030083EAC9031BB283F023077F
:10BF70004EF8040B87EA0717FFB2C3F3072282EAE1
:10BF80001712704642EA072282EAC70720F81419FE
:10BF90000BF1010B4FF0230CFE211622C82384F86D
:10BFA0007EB1278084F807C00EF1020EA170E27006
:10BFB000A37111E030770020207700204F2300206C
:10BFC00010460020348C0020B0210020AA2100203F
:10BFD0004A8C00200308208010F8013B7B4083EA54
:10BFE0000313DBB21A0982EA172242EA032282EA29
:10BFF000C3031BB29FB270452780EDD183F0F403D9
:10C0000083EA0313DBB24FEA131E8EEA172E8EEA81
:10C01000032E8EEAC30E0FFA8EFE1FFA8EFCCA4F55
:10C02000A4F800C04FEA1C295FFA8EFE84F81EE0D7
:10C0300084F81F907968BA683868FB6807F5D37C84
:10C04000ACE80F0038697969BA6904F2C518ACE840
:10C05000070004F2A71784F8C59184F8C4E117F823
:10C06000011F30680EF07AF9B845F8D194F87231B2
:10C07000002B41F0DC82B54B1B681922980684F82E
:10C08000722140F1F482B24BB24F1B78990741F113
:10C0900047863B7D042B8CBF4FF003084FF002080E
:10C0A000FEF756FD3B8A3A890A9003EB83035B0057
:10C0B000ADF842304FF47A703B680C93B7F80EE05D
:10C0C000397D7B688DF8448000FB02F24FF0000C54
:10C0D0004FF0FF300DF12809ADF840E0CDF82CC04D
:10C0E0000E920D938DF845100F90C846B8E80F00DA
:10C0F000DFF86CE2AEE80F0098E80F00AEE807004A
:10C100007246182122F81C39E17194F87E1184F8E6
:10C1100005C081F0780383EA0313D8B2030983F0E2
:10C12000F60343EA002383EAC0031BB283EA031049
:10C13000C0B2C3F3072383EA101343EA002383EA60
:10C14000C0031BB283F0C80080EA001C5FFA8CFCBD
:10C15000C3F3072080EA1C1040EA0C2080EACC00E0
:10C1600000B280F0180383EA031C5FFA8CFCC0F372
:10C17000072383EA1C1343EA0C2383EACC03C82079
:10C1800001F1010A4FF0FE084FF01E0CA0710EF1F4
:10C19000020E217184F87EA1238084F8028084F845
:10C1A00003C0184612F8011B414081EA0111C9B2CF
:10C1B0000B0983EA102343EA012383EAC10109B290
:10C1C00088B272452080EDD181F0180181EA011119
:10C1D000C9B24FEA111B8BEA102B8BEA012B8BEAB9
:10C1E000C10B0FFA8BFB1FFA8BF3574A23805FFAC0
:10C1F0008BFB1B0A0492059384F8273084F826B041
:10C20000964602F5D37A04F12208DEF80000DEF843
:10C210000410DEF80820DEF80C30D446ACE80F003D
:10C220000EF1100EC645E246EFD1DEF80000CCF864
:10C230000000DFF830819DF8143084F8CCB108F1AB
:10C24000260A84F8CD31C3461BF8011F30680EF072
:10C2500085F8DA45F8D1FEF77BFC3F4B3F4AB3F94E
:10C260000410B7F808E03B680B930A907B680C93C6
:10C2700082FB01274FF47A70C9174FF0000C00FBC6
:10C280000EF0C1EBA701ADF83CC0ADF83EC0ADF873
:10C2900040C0ADF842100D900E90CE46BEE80F00A3
:10C2A0002F4F84F805C00FC79EE807004FF0210C00
:10C2B00087E807001C23C8224FF0FE0EE370A2712E
:10C2C00084F807C084F802E094F87E11217181F0AF
:10C2D0006A0383EA0313DAB2130983F0D50343EA4E
:10C2E000022383EAC2031BB283EA0312D2B2C3F36E
:10C2F000072383EA121343EA022383EAC2031BB231
:10C3000083F0C80282EA0212D2B2C3F3072383EA9F
:10C31000121343EA022383EAC2031BB283EA0C022C
:10C3200082EA0210C0B2C3F3072282EA101242EA84
:10C330000022013182EAC0020C3784F87E1122808B
:10C34000A7F11C0110460FE0AA2100203077002041
:10C3500086770020B85A002034770020676666662A
:10C36000B02100204F23002011F8013B434083EA15
:10C370000313DBB21A0982EA102242EA032282EA9C
:10C38000C3031BB298B2B9422080EDD183F0680399
:10C3900083EA0313DBB24FEA131B8BEA102282EA13
:10C3A000032B8BEAC30B0FFA8BFB1FFA8BF3DA4FCD
:10C3B00023804FEA132C5FFA8BFB04F1220384F8ED
:10C3C00025C084F824B007F5D37A0593FB68386854
:10C3D0007968BA68D646AEE80F00059B10379F42D1
:10C3E000F246F3D13B88CD4FAEF80030C24684F818
:10C3F000CAB184F8CBC11AF8011F30680DF0AEFF46
:10C400005745F8D194F87EC1C54A84F804C08CF031
:10C41000EB0383EA0313D9B20B0983F0C50343EAA4
:10C42000012383EAC1031BB283EA0310C0B2C3F342
:10C43000072181EA101141EA002181EAC00109B215
:10C440000CCA81F0C80787EA0717FFB24FF0000E49
:10C45000C1F307210B93CDF830E081EA17130A925C
:10C4600099E8070043EA072383EAC7030FFA83F931
:10C47000AC4B84F805E089F0310783E8070087EAD0
:10C480000717FFB2C9F3072383EA171343EA072309
:10C4900083EAC703277A607AA27AE17A94F80CE0FB
:10C4A00094F811901BB25F4087EA0717FFB2C3F3FD
:10C4B000072383EA171343EA072383EAC7031BB260
:10C4C000584080EA0010C0B2C3F3072383EA101378
:10C4D00043EA002383EAC0031BB25A4082EA0210F7
:10C4E000C0B2C3F3072282EA101242EA002282EAB3
:10C4F000C00212B2514081EA0111C9B2C2F307234E
:10C5000083EA111343EA012383EAC1031BB28EEAD3
:10C51000030E8EEA0E1E5FFA8EFEC3F3072383EA34
:10C520001E1343EA0E23677BA07BE17B227C83EA18
:10C53000CE031BB25F4087EA0717FFB2C3F307239E
:10C5400083EA171343EA072383EAC7031BB2584061
:10C5500080EA0010C0B2C3F3072383EA101343EA52
:10C56000002383EAC0031BB2594081EA0111C9B21A
:10C57000C3F3072383EA111343EA012383EAC103C8
:10C580001BB25A4082EA0212D2B2C3F3072383EAF3
:10C59000121343EA022383EAC2031BB289EA0309A6
:10C5A00089EA09195FFA89F9C3F3072383EA1913A2
:10C5B00043EA092383EAC903A17CE27CDFF8709196
:10C5C0001BB2594081EA0111C9B2C3F3072383EAC0
:10C5D000111343EA012383EAC1031BB25A4082EAE2
:10C5E0000212D2B2C3F3072383EA121343EA0223EF
:10C5F00083EAC2031BB283F0270787EA0712D2B28D
:10C60000C3F3072787EA121747EA022787EAC20718
:10C610003FB20CF10103BAB25FFA87FA4FF0310C66
:10C62000FE200C2184F87E31C8234FEA122E22808E
:10C6300084F807C0A070E170A37184F814A0049F6F
:10C6400084F815E07968BA68FB683868B7F810C0F4
:10C65000A9E80F0029F803CB84F8BBE184F8BAA15C
:10C6600018F8011F30680DF079FEC145F8D194F833
:10C670007671002F40F0D6872B4B94F87E81B3F96A
:10C680000010B3F90220B3F904309FED286ADFF8F7
:10C690009490677107EE103A029B1B680A9388F02A
:10C6A0006A0383EA031306EE901AD9B20B0983F0EA
:10C6B000D50343EA012383EAC1031BB283EA0311D2
:10C6C0005242C9B207EE902AC3F3072383EA11133B
:10C6D00043EA0123F8EEE77AF8EEE66AB8EEC77AA5
:10C6E00083EAC1031BB267EE867A66EE866A27EE9E
:10C6F000067A002083F0C80CCDED0C7ACDED0B6AE4
:10C700008DED0D7A0E900F9010908CEA0C1E0DF1AD
:10C71000280A5FFA8EFE0DE0AA2100207323002074
:10C72000E4790020B02100203477002088C3E43A67
:10C7300050230020C3F3072CBAE80F008CEA1E1C1C
:10C740004CEA0E2C8CEACE0C0FFA8CFCA9E80F00F8
:10C750008CF01E0E9AE807008EEA0E17FFB2CCF39B
:10C76000072E8EEA171E4EEA072E89E807008EEA8A
:10C77000C70E1C21FE274FF0050A4FF01E0CC822E1
:10C7800008F10103A770E17084F876A184F807C06E
:10C79000A9F11001A27109F10C0784F80480A4F832
:10C7A00000E084F87E3111F8013B83EA0E0383EA4E
:10C7B0000313DBB21A0982EA1E2242EA032282EA4A
:10C7C000C3031BB21FFA83FEB942A4F800E0EAD10A
:10C7D00083F0270383EA0313DBB21A0982EA1E22DD
:10C7E00082EA032282EAC3031BB21FFA83FCDFF84A
:10C7F000E083A4F800C05FFA83FE4FEA1C2C84F8A3
:10C8000025C084F824E008F5D37904F1220AD8F889
:10C810000000D8F80410D8F80820D8F80C304F469B
:10C820000FC708F11008D045B946F0D1DF4FB8F86E
:10C830000030A9F8003007F1240884F8CAE184F830
:10C84000CBC117F8011F30680DF088FDB845F8D14D
:10C8500094F877A1BAF1000F40F0DE86D44B1B6844
:10C86000052284F877219A0641F10D80D14BDFED46
:10C87000D26ADA891B8907EE902A07EE103AF8EEA1
:10C88000E77AB8EE477A67EEA67A94F87EC1CB4B8A
:10C89000CB4AB3F90410B2F90620CA4FCA48CDED0D
:10C8A0000B7A8CF0220383EA03135FFA83FE4FEACC
:10C8B0001E1383F0590343EA0E23B2F5FA6F83EA9D
:10C8C000CE031BB2A8BF4FF4FA6283EA0318B2F595
:10C8D0007A7F5FFA88F8C3F3072EB8BF4FF47A72F5
:10C8E000A2F57A728EEA181E642303FB02F34EEA65
:10C8F000082E87FB03278EEAC80EDA17C2EBA712B1
:10C9000080FB01300FFA8EF7CB174FF0000BC3EB13
:10C91000A00387F0C8080DF128098DED0C7AADF859
:10C920003A20ADF83830CDF828B0CDF834B0CE4646
:10C9300088EA0818BEE80F005FFA88F8C7F30727EF
:10C9400087EA181747EA082787EAC8089F4FDEF8E2
:10C9500000E084F804C00FC70FFA88F888F04A0393
:10C9600083EA0310C0B2C8F3072383EA10133A46E0
:10C970000CF1010143EA002383EAC00342F810E905
:10C9800000204FF04A084FF0FE0C4FF0140E84F8D0
:10C990007E11C82160712380043784F8078084F8F1
:10C9A00002C084F803E0A171184612F8011B41404F
:10C9B00081EA0111C9B20B0983EA102343EA01237A
:10C9C00083EAC10109B288B2BA422080EDD181F078
:10C9D000140181EA0111C9B24FEA111E8EEA102E2C
:10C9E0008EEA012E8EEAC10E794B0FFA8EFE1FFAE7
:10C9F0008EFC1F464FEA1C2B5FFA8EFE84F81DB09A
:10CA000084F81CE0596838689A68DB68A4F800C0AC
:10CA100007F5D37CACE80F0038697969B7F818805E
:10CA20000497ACE8030004F2A717ACF8008084F880
:10CA3000C3B1B84684F8C2E104F2C31B18F8011F61
:10CA400030680DF08BFCC345F8D1624B624A1B780D
:10CA50001278013B12F00100DBB214BFC02140216B
:10CA6000172B03D85D4A134493F80CA05C4B1A882B
:10CA700093071ABF002341F01001012312F4027F33
:10CA800018BF022312F0100F18BF062312F0200F58
:10CA900018BF1023002841F093804FF0030894F84A
:10CAA0007EC10A938CF0460383EA0313DAB21309BA
:10CAB00083F0920343EA022383EAC2031BB283EAB0
:10CAC0000310C0B2C3F3072282EA101242EA002226
:10CAD00082EAC00212B282F0C80E8EEA0E1E002355
:10CAE0005FFA8EFE0320C2F307228DF82CA08DF88A
:10CAF0002F8082EA1E128DF82D308DF82E108DF8C1
:10CB0000300042EA0E2899E8070088EACE0E0FFAB4
:10CB10008EF8DFF8B8A0E37188EA0819AAE80300E4
:10CB20005FFA89F9C8F3072888EA191848EA092141
:10CB300081EAC90994F808808AF800200FFA89F977
:10CB400088EA090282EA02185FFA88F8C9F3072224
:10CB500082EA181242EA0822607AA17A94F80B90CD
:10CB6000637182EAC80212B2504080EA0010C0B27B
:10CB7000C2F3072282EA101242EA002282EAC002CD
:10CB800012B2514081EA0111C9B2C2F3072282EA0E
:10CB9000111242EA012282EAC10212B289EA0209B2
:10CBA00089EA09195FFA89F91CE000BF4F230020C8
:10CBB00030770020B85A00200AD7233C3477002071
:10CBC0004A8C0020D34D621067666666B021002053
:10CBD000AA210020CC4D0020F04B0020ACFC030823
:10CBE00084770020C2F3072282EA191242EA09225E
:10CBF00094F80C80607BA17B84F804C082EAC902AF
:10CC000012B288EA020888EA08185FFA88F8C2F3C4
:10CC1000072282EA181242EA082282EAC80212B205
:10CC2000504080EA0010C0B2C2F3072282EA10121C
:10CC300042EA002282EAC00212B2514081EA0111A6
:10CC4000C9B2C2F3072282EA111242EA012282EA41
:10CC5000C102E17B94F8109013B281EA030282EAE8
:10CC60000212D2B2C3F3072383EA121343EA022368
:10CC700083EAC2031BB289EA030282EA0212D2B239
:10CC8000C3F3072383EA121343EA022383EAC203AE
:10CC90001BB283F0320282EA0212D2B2C3F307233C
:10CCA00083EA121343EA022383EAC2031BB29AB255
:10CCB0004FF0FE085FFA83FE0920C8210CF1010C39
:10CCC00084F802804FEA1228E070A17184F87EC1D6
:10CCD000228084F8128084F811E0049B1868596857
:10CCE0009A68B3F80CB00AF5CC7CACE807000AF5FA
:10CCF000D47A8CF80290ACF800B084F8B88184F84B
:10CD0000B7E117F8011F30680DF028FBBA45F8D1DC
:10CD1000039BC4F86831FEF764BEDFF824A3B84F64
:10CD2000DFF82093412022F045F9BAF9023087FB61
:10CD30000320DB17C3EBA00080B222F01FF9BAF981
:10CD4000003087FB0320DB17C3EBA00080B222F08A
:10CD500015F9BAF9043087FB0320DB17C3EBA000F9
:10CD600080B222F00BF999F80010D8F800000DF00D
:10CD7000F5FA94F860A11AF0010700F0E183A14BE5
:10CD80001B68980672D5A04BA04F1B78990740F1FD
:10CD9000C9863B7D042B8CBF0323022347200393CA
:10CDA00022F008F9386822F0B5F8786822F0B2F875
:10CDB000B7F80EA0964AD8F80000A2FB0A3ACAF3C8
:10CDC000471A51460DF0CAFA3A8999F800106420C2
:10CDD0008AEA010A00FB02F089F800A022F09AF822
:10CDE000039B3F7DD8F8000043EA8707FFB239462E
:10CDF0000DF0B4FA99F80030D8F800005F403946D9
:10CE000089F800700DF0AAFA94F860A1BAF1000F49
:10CE10002CD1804F4F2022F0CDF8386822F07AF8DC
:10CE2000786822F077F8504622F074F80121D8F89B
:10CE300000000DF093FA744B99F800201B78D8F895
:10CE4000000003F0010782F00102394689F8002052
:10CE50000DF084FA99F80030D8F800007B401946AC
:10CE600089F800300DF07AFA94F860A16A4AC4F8A3
:10CE70005CB10AF10103DBB2A2FB0312D20802EBA0
:10CE80008202A3EB420384F86031FEF78ABD634B54
:10CE9000634918680DF02EFA00232370FEF729BEAF
:10CEA000604F386800283EF469AD4FF0000ADFF8A3
:10CEB00098815D4CAB4655460DF04CFAF8B1F5B98A
:10CEC0004FF00109AA4638680DF040FA83B27E2B74
:10CED00000F01A8398F80120002A49D194F84C11E7
:10CEE000B1B11B2B84F84C2100F0E8820D2B45D00A
:10CEF000386888F801900DF02DFA0028E3D1AA4691
:10CF000050460AAA49495D4622F06EF8FEF736BD42
:10CF10007D2B00F0AE8494F8502122B180F02003E4
:10CF2000DBB284F8501194F84B21062A10D8B4F8DB
:10CF30004E1138681944A4F84E11A118013281F835
:10CF4000543184F84B210DF005FA0028BBD1D6E707
:10CF5000B4F84E2188F8019013449BB21A0A52FA91
:10CF600083F3FF2BA4F84E31386802D1304DA3E78C
:10CF700038680DF0EFF90028A5D1C0E73868A4F8AB
:10CF80004E210DF0E7F900289DD1B8E794F8BC32A6
:10CF9000C4F8B852012B40F2558494F8BD222549BB
:10CFA000981801EB8001013202F001024E6A84F808
:10CFB000BD22BEB1204F0B970DF14809123FA523AA
:10CFC00049F8207D802284F81031152329464846EF
:10CFD00084F8112184F81231B047002840F0B3835F
:10CFE00094F8BC32154A013382FB0312A2EBE372C0
:10CFF00002EB42029B1A84F8BC32FEF702BD00BF6E
:10D00000676666663077002086770020B85A002071
:10D010001F85EB51E4790020CDCCCCCCC478002026
:10D02000EC77002094770020A8210020F222002035
:10D03000FC220020ACFC0308CD220020565555559B
:10D04000347700201C770020040000208F4A904B8A
:10D0500092F80BE0029AD4F8381110681B888D4AB8
:10D06000401A4FF47A71DFB201FB0EF11B0A977779
:10D07000177588424FF00007D37753759770177173
:10D0800080F0CD83844985480B688968DFF828E201
:10D09000834F9EF800E097F8149080FB03C8DB17DD
:10D0A00080FB010CC817C3EBA80111770912C0EB74
:10D0B000AC005177F4214FEA202C7A4B82F8200003
:10D0C000917601203021D07682F8221075207821C7
:10D0D0001EF0020F82F821C083F81A9082F8230014
:10D0E00082F8241000F09883D7F800C06E4AD7F871
:10D0F00004E0DFF8C8B1DFF8C88182FB0C014FEA19
:10D10000EC7082FB0EA2C0EBA1504FEAEE71C1EBB6
:10D11000A2520BFB00C10BFB02EB01EB41010BEB3D
:10D120004B0B49004FEA4B0B039288FB012A88FB0B
:10D130000B284FEAA8420692039AB7F80E803F895F
:10D1400002EB820202EB820207F5FA7707924FEABE
:10D15000AA4ACA17BFB20597AAEB02073A464FFA86
:10D1600087FA524F00EB800008EBC80807FB121249
:10D1700000EB8000069F4FEA8808CDF810800AEB8C
:10D18000800A4FEAEB784948A7EB080100FB11B091
:10D1900003900798464FDFF81C81DDF814B083F840
:10D1A00015B049B201EB800106910499B9F1050F60
:10D1B00087FB01074FEADC7C4FEAE179C9EBA7194D
:10D1C00083F809C0039FDFF8FCC0BDF81810CDF844
:10D1D00010904FEADE7E88FB02091FFA8AFA88FB6C
:10D1E000070883F80EE04FEAE770BCF800E0049F00
:10D1F000DFF8D4C083F80AA04FEAE272C2EB6912EA
:10D20000C0EB68104FEA1A294FEA1B284FEA112B8E
:10D210004FEA222A1A73BCF800C083F80B90D97326
:10D2200083F810B04FEA2029C7F307214FEA1E2BDD
:10D2300034BF3222332283F80DA0587483F8129041
:10D2400083F81680DF71197283F813E083F814B045
:10D25000DA7683F81CC0C4F83451FEF721BBDFF83E
:10D260006C90D9F800000DF069F800283EF4A7ABE7
:10D27000D9F8000001210DF05DF80222002387F8A3
:10D28000742088F80030FEF79ABB00BF1C4C0020C9
:10D29000144C0020687800205C7500206766666684
:10D2A000B85A0020947800206BCA5F6B40420F0090
:10D2B000D34D62101F85EB5186770020806967FF90
:10D2C00083DE1B4390770020368C002064480020CA
:10D2D0005E209047D8F8003002209847FF201AF0CF
:10D2E00091FB0378FF2B00F01A8490F901304FEA8C
:10D2F000E3795FFA89F9D8B222F02AFA484622F097
:10D3000027FAD8F800305E209847D8F8003003207C
:10D310009847FF201AF076FB0378FF2B00F0FB8381
:10D32000B0F90830D8B2C3F3072922F011FA484601
:10D3300022F00EFAD34B1B78042B7DD0DFF880B39C
:10D34000B4F82E119BF80020DFF868A391FBF2F3EC
:10D3500002FB13139BB2BAF80010A4F82E314FEA67
:10D3600003191FFA89F9642303FB01235200B3FB5D
:10D37000F2F349EA0329C3F303225E20D8F8003010
:10D380001FFA89F949EA02099847D8F800300620BF
:10D3900098475FFA89F022F0DBF94FEA192022F072
:10D3A000D7F9B949B4F82E214B7ABAF800A0013266
:10D3B000012BA4F82E2100F05E864A7B0AEB8A033B
:10D3C0001FFA83FA002A40F0F683D8F800305E2076
:10D3D0009847D8F800303A209847AC4BA3FB0A395D
:10D3E0004FEA59191FFA89FB5FFA8BF022F0B0F966
:10D3F0004FEA1B2022F0ACF9D8F800305E209847A5
:10D40000D8F800303B209847642303FB19A39BB254
:10D410009F48053380FB0320DB17C3EBA000C0B29D
:10D4200022F096F9002022F093F9DFF8989299F80B
:10D430000630002B40F08A833B689F0600F13A8259
:10D4400094F82C31D8F80020FEF717BADFF878925C
:10D450009FED908A4FF0240A5E2090475046D8F8FE
:10D46000003098478C4BF9EC016A9B8A07EE103A22
:10D47000F8EEE66AB8EEC77A0AF1010AC6EE877AD4
:10D480005FFA8AFA67EE887AFDEEE77ACDED027AE6
:10D49000BDF908B05FFA8BF022F05AF9CBF3072000
:10D4A00022F056F9BAF1270F02D0D8F80020D3E7BE
:10D4B00094F82C31D8F80020FEF7DBB938680CF06E
:10D4C00049FF00287FF414AD386884F84A9188F841
:10D4D00001900CF03FFF00287FF4F5AC0FE5FDF75D
:10D4E00037FB6E4B1B68A0EB030B40F6B8339B4534
:10D4F00000F2B4816A4B1A793A2A00F0CD840023F5
:10D5000088F80030FEF75BBA386884F84AA184F8DE
:10D510004BA184F84C9188F801A00CF01BFF002867
:10D520007FF4D1ACEBE494F8481194F849315D48AC
:10D530004A1CFEF70FBA013B84F86E31FEF76EBC51
:10D54000594B1B88DA0513D4D80600F1FD829906E1
:10D5500000F17C855A0600F1A785180700F1A78520
:10D56000D90700F1DE8513F0020F0CBF04270C274A
:10D570004E4B4F4A1B78D27803F001030AB143F0B7
:10D5800002035320039321F015FD4A4A128802EB4F
:10D59000820202EB8202900080B221F0EFFC0020B8
:10D5A00021F0ECFC444A45491288D8F80000C2EB4F
:10D5B000C212520081FB023111444FEAE27ACAEBF7
:10D5C000612A5FFA8AFA51460CF0C8FE99F80020E9
:10D5D000039BD8F800001F438AEA020A002189F859
:10D5E00000A00CF0BBFE3946D8F800000CF0B6FEE7
:10D5F00099F80030D8F800007B40DBB2194689F872
:10D6000000300CF0ABFE94F860A1FFF7FFBB013ACD
:10D6100084F86F21FEF72ABD0AF1FF3A84F877A15A
:10D62000FFF776BB013F84F87671FFF711B9013B34
:10D6300084F87231FFF71BB80024DFF8908027468A
:10D640004FF0500A02E0DBB283F3118816F804B001
:10D65000601C5946304421F065FB002840F02381CE
:10D660000BF101031C44EFF311838AF31288326E2D
:10D670009442E8DB0022DBB2326683F31188FEF7C6
:10D68000B6BA00BFEC7D00201C4C00201F85EB517A
:10D690006766666600007A443C77002054470020A5
:10D6A0003C4700209877002084770020F04B002032
:10D6B0008C790020144C0020348C0020030820803A
:10D6C0002A4C0020207700206C770020B9F802084F
:10D6D0004FF0000A5E201F6884F82CA19047D8F80C
:10D6E0000030DFF8309317209847504622F030F88A
:10D6F000BC4BA3FB07239B0BA9FB03125209C2EBF4
:10D700000212A3EB8203D8B222F022F8D8F800303C
:10D710005E209847D8F8003018209847B24BA3FBFA
:10D7200007239B09A9FB03125209C2EB0212A3EBC8
:10D730008203D8B222F00CF8504622F009F8D8F84B
:10D740000020FEF79FB80A9EBE4240F2AA843D46E2
:10D75000002141F2210015F8013B81EA03235A0020
:10D7600013F4004F80EA020192B289B208BF114659
:10D770004A0080EA020311F4004F99B293B218BF35
:10D780000B46590013F4004F80EA010289B292B2AD
:10D7900008BF0A46530012F4004F80EA03019BB20F
:10D7A00089B208BF19464B0011F4004F80EA03020A
:10D7B0009BB292B208BF1A46530012F4004F80EA9F
:10D7C00003019BB289B208BF19464B0011F4004F08
:10D7D00080EA03029BB292B208BF1A46530080EA65
:10D7E000030112F4004F9BB289B208BF1946B5423B
:10D7F000B1D148460DF068FF7C490A9D7C486D1AFE
:10D80000152DA8BF15252A4631F030F8794A94F82D
:10D81000BC321570FFF7E6BB2D22DA761BE5764B9E
:10D8200002991B780968C4F83811013B012B3FF6B7
:10D8300029AC102102239170137123E421F06AFFB7
:10D84000FEF790B86D4A02EB8302566AFFF7B1BB50
:10D8500021F050FF01233B70FEF741B8684AB2F84F
:10D86000623100210133A2F8623188F80010FEF71E
:10D87000A6B8386884F850910CF06CFD00287FF44D
:10D8800022ABFFF73CBBDFED5F7AB0EE677AFEF7C5
:10D89000FCBF0146844607468246049080460590B8
:10D8A0000246FEF7F2BA41463A201AF0B9F90743A8
:10D8B000FFB2D5E6DFF860A19AF80030980700F1D2
:10D8C0005782514F4FF00009CB46D8F800305E2008
:10D8D0009847D8F8003001209847584621F038FF83
:10D8E000484621F035FFD8F800305E209847D8F838
:10D8F000003009209847002021F02AFF002021F065
:10D9000027FF7B8A97F81490B3F5967F0AD994F88D
:10D910002C2102F00F02072A04D842F20F79994510
:10D9200028BF9946D8F80030DFF8F0B05E2098475D
:10D93000D8F80030052098479BF80830002B00F0FD
:10D940009183A9F1200307EE903A9FED307AF8EE2B
:10D95000E77AF6EE006A67EE877ABEEE007AF5EEB9
:10D96000C07AF1EE10FA58BFB0EE667A77EE877A99
:10D97000FDEEE77ACDED027ABDF908905FFA89F005
:10D9800021F0E6FEC9F3072021F0E2FE9AF800201C
:10D99000002392070893099300F1CB8094F830316B
:10D9A000012B00F0C680BBF90030DFED196A07EEED
:10D9B000103ABBF9023007EE903AB8EEC77AF8EEAB
:10D9C000E77A27EE267A67EEA67ABDEEC77AFDEEF5
:10D9D000E77A0AA88DED0A7ACDED0B7A21F0DAFE0E
:10D9E0002EE500BF73B2E745D34D6210B822002088
:10D9F0001C45002031450020EC7D0020ACFC0308D4
:10DA0000A821002000000000B85A0020E4380E3F92
:10DA10000050C34789888888867700201C4C0020E6
:10DA2000C149C24B0093A1F13F07C14BC14A0991C3
:10DA300001F8404C0AA8C04908970DF01DFF089F47
:10DA40007B1C08933C70089B2922591C08911A7072
:10DA5000089BEA22591C08911A70089BC822591C7D
:10DA600008910AA81A702FF075FF00F101080AA9A1
:10DA70004246089830F0FAFE089A02EB0803013398
:10DA8000089302F80840089B5A1C08921C70089BD7
:10DA90005A1C08921C70089B5A1C08921C70089B08
:10DAA0005A1C08921C70089B5A1C08921C70089BF8
:10DAB0005A1C08921C70089B5A1C08921C70089BE8
:10DAC0005A1C08921C70089B5A1C08921C70089BD8
:10DAD0005A1C08921C70089B5A1C08921C70089BC8
:10DAE0005A1C08921C70089B0122991812A80891D0
:10DAF0001A7050F8283DDB1B3B7021F0C3FE8F4BA2
:10DB00003470C3F8B052FDF770BFC4F83C5187F8C9
:10DB10000080FDF7E4BE4FF00009484605E44846A2
:10DB2000FFF7EABB0123FFF739B90CF003FCFDF75F
:10DB3000EBBE97E80C00012108A884F83011089288
:10DB4000099321F027FE7BE4342711E5D8F8003053
:10DB5000DFF818A2DFF810B25E209847D8F800303E
:10DB600028209847DAF800308BFB032BDB17C3EB38
:10DB7000AB0B5FFA8BF021F0EBFDCBF3072021F02C
:10DB8000E7FDD8F800305E209847D8F80030042030
:10DB90009847B9F80830002B40F05B82DAF808307B
:10DBA00083F310095FFA89F021F0D2FDC9F3072051
:10DBB00021F0CEFD40E49BF800309AFBF3FA04E438
:10DBC0005F4AD278002A0CBF4FF004084FF00508D6
:10DBD000FEF765BF0123D9F800003B700CF0B6FBDF
:10DBE0000746D9F800000CF0B1FB7B067DF477AE58
:10DBF0008A2800F085828E287DF471AE9AF8003074
:10DC0000002B7DF488AE4F484F4B03602D2384F8E2
:10DC100040310768FDF767BE434B0B93A3F1400902
:10DC200000222121A3F13D0A03F8402C89F80210BB
:10DC300089F80120CDF828A020F06AFC434B444A23
:10DC40001B88444900280ABF11464FF003084FF0D3
:10DC500004085A0500F12182D80700F12B8203F055
:10DC600002033D4A002B1CBF4FF0030811464246F9
:10DC70003A4830F0FBFD0AEB080312A8384A01339A
:10DC800040F8203D9B1A00220AF8082089F801304C
:10DC900021F0F8FDFDF753BF234A324B0B920DF1F3
:10DCA0004808A2F13D0048F8200D1988DFF8BC9023
:10DCB000A2F1400300204FF00A0E02F8400C0822A7
:10DCC00083F801E040469A700DF0D8FCD9F8003096
:10DCD0002549DA1781FB0313C2EBA30399B240462F
:10DCE0000DF0CCFC0EF088FCD9F808900A9B4FEAA6
:10DCF0001942591C0A911A700A9B4FEA1922591CA1
:10DD00000A911A700A9B5A1C0A9283F800900A9B87
:10DD10005A1C0A921870404621F0B4FDFDF70CBF62
:10DD20004FF00108FEF7BCB9EC770020E6A6002012
:10DD3000882C0408902C04089C2C0408A82100209E
:10DD40008C790020A077002068780020847700205C
:10DD50006C2C0408742C0408842C0408AF77002071
:10DD6000AD770020144C0020676666665C75002065
:10DD7000D24FD8F80030DFF874935E209847D8F877
:10DD8000003011209847FA894FF4F36B0BFB02F235
:10DD900089FB0239D217C2EB69395FFA89F021F0A9
:10DDA000D7FCC9F3072021F0D3FCD8F800305E205F
:10DDB00098471920D8F800309847FB89C04A0BFBD8
:10DDC00003F382FB0301DB17C3EB611382FB032127
:10DDD000DA17C2EB6112642101FB1233D8B221F0D1
:10DDE000B7FC002021F0B4FC9AF80030B7F8089096
:10DDF00099077FF567AD5FFA89FB4FEA192964E55A
:10DE0000DFF8EC929FEDAF8AB9F90230AE4A0B927F
:10DE100007EE903AF8EEE77A0DF1480867EE887A57
:10DE2000A2F14003FDEEE77AA2F13D0148F8201D82
:10DE300002F8400C0822CDED027A5A701E229A7028
:10DE4000BDF8081040460DF019FCB9F9003007EE96
:10DE5000903AF8EEE77A404667EE887AFDEEE77A88
:10DE6000CDED027ABDF808100DF008FCB9F90430C8
:10DE700007EE903AF8EEE77A404667EE887AFDEED4
:10DE8000E77ACDED027ABDF808100DF0F7FB4046B9
:10DE900021F0F8FCFDF74DBE99780393184616F073
:10DEA0008FFF00287FF42BAB8849894F894A8A4C21
:10DEB0000988DFF840929368F9611168B4F862212B
:10DEC000F863C7F86CB0FB64F962D9F80000FA6532
:10DED000FBF794FB834600287DF46CAD5146D9F8DE
:10DEE00000000CF027FA039B94F86421DB7804937C
:10DEF000642A4FF0040387F8743040F01C8194F8D2
:10DF00006531DFF8F4A1072B08BF84F865B194F8F8
:10DF10006521069207EB021BDBF804100591084609
:10DF20002FF018FDDBF8083003935FFA80FB1846EA
:10DF30002FF010FDC3B20BEB0300069A0599059371
:10DF400008308AF8070022F00F008AF80A0002F071
:10DF50000F0203EBCB008AF80D208AF80E005A4618
:10DF60000AF10F0030F082FC059B03990BF10900C8
:10DF70001A460AF10603184430F078FC9AF8073084
:10DF800003F1010BD3B1013B5FFA83FC0CF1080CE8
:10DF9000DFF868E1D4440AF10700002310F8011B00
:10DFA00059408B00CA0883EA410302F018024B4033
:10DFB0004EFA02F253408445DBB2EFD1474A04984F
:10DFC0000BF8023030F000FC94F865310022013388
:10DFD00084F8653184F864219AF802305BB11AF84C
:10DFE0000610D9F800000CF0B9F901369AF80230A1
:10DFF000F6B2B342F3D894F864310322013384F8C3
:10E00000643187F8742088F80020FFF72AB92F4B75
:10E01000334A1B88927903EB830303EB83034FEAB4
:10E0200083081FFA88F8002A00F01581294B1B6825
:10E030000FFA83FA0EF0E0FA40B2FDF72ABE11465D
:10E040009446174692460492FDF71FBF2427FFF718
:10E050008FBA0EF0D1FA21F07BFB002021F078FB83
:10E06000FFF7EAB95FFA89F021F072FB4FEA192055
:10E0700021F06EFB8AE4D8F800305E209847D8F88B
:10E080000030392098475FFA8AF021F061FB4FEAAF
:10E090001A2021F05DFBFFF7C8B94FF003081149C2
:10E0A000E5E50021FFF7A5BB1027FFF761BA2027A0
:10E0B000FFF75EBA0C494FF00408D8E5B85A0020C3
:10E0C0001F85EB5158A08B41EC770020144C0020A9
:10E0D000040000205C750020A8210020FA6C0020BC
:10E0E00020770020782C04087C2C040889B5F814CB
:10E0F0003477002064480020F46C00200007090EEB
:10E10000614B1B689F067DF5EAAB9AF80030002B47
:10E110007DF401AC5D485E4B03602D2384F84031F3
:10E1200077E50827FFF724BA5A4B8046B3F900A0D9
:10E130006420FDF7AEBD97F87530DFF868A1564949
:10E1400005961A0704BF0133DBB2072B28BF012352
:10E150004FEA031B07EB0B02107C00228AF80A200F
:10E1600011F800C05FFA8BF203920AF10D02039ED0
:10E1700007EB0B013043BCF1010F1070C96802F1CD
:10E1800001000ED9ACF10206F6B206F1020E964479
:10E19000024602F8011B72454FEA1121F9D10136FE
:10E1A0003044BB4421F0600201339BF81110DBB214
:10E1B0000A43082B027000F101024FD04FEA031B03
:10E1C00007EB0B00344E007C344916F800C0039E68
:10E1D000511A06F1100E01EB0C0606965FFA8EF648
:10E1E0000396069E132EC2DD059EDFF8BCE0C9B281
:10E1F0008A1DD2B242F040008AF8070002F1010BFA
:10E20000CAB14A1DD2B20832524403920EF1010C37
:10E2100000221CF8010B5040820082EA4002C10833
:10E2200042401F4801F0180140FA01F14A400399A9
:10E230006145D2B2EDD104980BF80E2087F8753005
:10E2400030F0C2FAC8E61146944617469246049248
:10E250009046FDF71ABE4FF0FF33E9E60F49059EE1
:10E26000511AC2E71146FDF710BE11469446FDF75C
:10E270000CBE114694461746FDF707BE114694465C
:10E2800017469246FDF701BE30770020A0770020A8
:10E29000947800205C750020ACFC0308016D002020
:10E2A0000007090EF46C0020FA6C00202DE9F047FD
:10E2B000B0F908500D81EDB2442D92B00C461746CE
:10E2C00000F0C382064642D9812D00F0008200F2A0
:10E2D0009580542D00F0C98040F2E6816E2D00F04B
:10E2E0008282802D40F01D81BD4B93F8009009F192
:10E2F000020919F0FF0900F09580BA4BBA4FBB4EE6
:10E30000DFF824A3994403F101080A2516E0322D11
:10E3100000F0CA82A5F13C00C0B2132840F2CA82C4
:10E3200000232268511C216015702268C14502F14A
:10E3300001012160137075D018F8015B0A2DE6D138
:10E34000BAF80030FF2BA8BFFF23DBB2E9E7052DA9
:10E3500000F069821ED8022D7FD040F29281032DF9
:10E3600000F03882042D40F0DC802A46A049204687
:10E370000DF062F9002120460DF0A6F92268022175
:10E38000531C0125236028462B461170638112B06F
:10E39000BDE8F087242D5ED040F20381282D00F0E7
:10E3A000DE81382D40F0BD800B68924901255A1C52
:10E3B00022601D7023680522581920601A70236896
:10E3C0000A22581920601A70236800225819206008
:10E3D0001A7023680A78581920601A7023684A78DE
:10E3E000581920601A7022688978531923602B46C7
:10E3F00011702846638112B0BDE8F087A02D18D0B7
:10E4000040F21481B82D00F0E381FE2D40F08980A8
:10E41000794D05F1080635F8021B20460DF054F938
:10E42000B542F8D101252B462846638112B0BDE8DC
:10E43000F087724B084619680DF02EF9704B204694
:10E4400019680DF029F96F4B1968204601250DF068
:10E4500023F92B46E8E76C4BF6E704226B4920468C
:10E4600001250DF0E9F82B46C3E70B68684A694FB0
:10E47000581C11212060197023681278591C2160E2
:10E480001A70236897F85520591C21601A70236868
:10E4900097F85420591C21601A70B7F85010204684
:10E4A0000DF012F923680022591C21601A702368AC
:10E4B0002822591C21601A70B7F8521020460DF01E
:10E4C00003F9BD1E07F14E0635F8021F20460DF078
:10E4D000FBF8AE42F8D122684F4B0D21501C206052
:10E4E0005D181170226813F8011F501C9D422060B6
:10E4F0001170F7D123680222591C21601A70B7F8F5
:10E50000561020460DF0E0F8B7F8581020460DF0F0
:10E51000DBF80125B7F85A1020460DF0D5F82B4648
:10E5200067E72146284609F0F5FA00287FF47AAF1C
:10E53000742D00F0BF80772D0CD1336872689A4239
:10E540001BBF5A1C326001461978344A20462DF010
:10E5500081FF67E7F52D01F05782762D00F07D8170
:10E56000392D326800F0178200F2FC81212D01F074
:10E570002B82292D40F04282531C336013780A2BE2
:10E5800001F0D182502B40F0468430460DF042F825
:10E59000234F388030460DF03DF8012578802B461A
:10E5A00027E7202DBDD10B681E4D591C6A782160CC
:10E5B0001A7023682A78591C21601A702368AA7877
:10E5C000591C21601A70298920460DF07DF82368B6
:10E5D0006A79591C21601A702268A979D0E600BFB7
:10E5E000EC6D0020E0FC0308676666666828002082
:10E5F000E6A60020FD530020FC8E0020107AFF1FAD
:10E60000147AFF1F187AFF1F5C550020042D0408A0
:10E61000088F0020807D0020DD7D002031C00308B0
:10E62000502800202077002090280020822D7FF4A1
:10E6300078AF0B68B74AB84D1178B84A581C2060BB
:10E640001970118920460DF03FF8B54B22681B88E0
:10E65000FF2B02F10101A8BFFF2321601370A968FD
:10E6600081F3100189B220460DF02EF8296801F3DC
:10E670000F0189B220460DF027F8AA4B22681978BD
:10E680007EE6012D7FF44DAF0B680022591C2160FE
:10E690001A7023685A1C22601D7022682521531CA1
:10E6A00023602B461170A4E6522D7FF43AAF226806
:10E6B000002165E6336872689A421BBF5A1C3260BB
:10E6C00001461978984A20462DF0C4FEAAE6974BD9
:10E6D0001E78033616F0FF063FF4A4AE944B954F18
:10E6E0001E4403F101094FF00A0820E0B8F1500F71
:10E6F00000F0D880B8F1320F00F0F180A8F13C00B2
:10E70000C0B2132840F2EE800025294623685A1C27
:10E710002260204683F800800CF0D6FF2946204670
:10E720000CF0D2FFB1453FF47DAE19F8018BB8F182
:10E730000A0FDBD1804B9D68196805EB85054FF604
:10E74000FF736D009D42A8BF1D469942A8BF1946A0
:10E7500025EAE57521EAE171ADB289B2D6E70B6829
:10E76000DFF8FC81754E591C022221601A70236863
:10E7700006275A1C22601F7023680A22591C216038
:10E780001A70236801255A1922601D70B8F800100C
:10E7900020460CF099FFB8F8021020460CF094FFC8
:10E7A00023685A1922601F7023685022591921606A
:10E7B0001A7023680022591921601A703188204686
:10E7C0000CF082FF718820460CF07EFF2B4610E68D
:10E7D0005B4B39E60B685A1C0A601D700B685A1CAB
:10E7E0000A601D7063E74E4B0A681B884A4DFF2B79
:10E7F000A8BFFF23511C21601370A96881F3100189
:10E8000089B220460CF060FF4E4B204619880CF070
:10E810005BFF296801F30F0189B2204601250CF046
:10E8200053FF2B46E5E50B22474920460CF004FF39
:10E830000822464920460CF0FFFE012507224449E4
:10E8400020460CF0F9FE2B46D3E5002A3FF4EAAD52
:10E85000404B136001252B46CBE533685A1C3260D0
:10E860001B78002B01F05481102B01F057813A4D99
:10E87000064601462268501C2060137020460CF0AA
:10E880000BFF314620460CF007FFE96820460CF0EC
:10E8900003FF204600210CF017FF002120460CF05A
:10E8A00013FF04E72D4B46E73388FF2BA8BFFF2358
:10E8B000DBB236E519F0A6F800283FF431AD037855
:10E8C0000A2B25D8B0F9023087FB0312DB17C3EB04
:10E8D000A2039BB2FF2BA8BFFF23DBB221E597E881
:10E8E00022002AE719F08EF800283FF40DAF0378D4
:10E8F0000A2B3FF609AFB0F90430B0F9061003EB6C
:10E90000830383F3500521EAE171ADB289B2FDE6DC
:10E910000023E2E72A4C00205C75002020770020CD
:10E92000144C0020EC7D00203DC00308EC6D00205D
:10E93000F0FC0308602800201C280020502800203C
:10E9400024400020348C00200C2D0408182D0408CD
:10E95000242D0408B97801087024002054280020D0
:10E96000F84A0020552D28D0572D47D1531C154665
:10E97000336015F8370B0DF107020133336013F8DC
:10E98000011C02F8011FAB42F7D102A90125FAF7D9
:10E990000BFA2B462DE5531C336013780A2B01F03C
:10E9A000C88030460CF042FE30460CF03FFE012598
:10E9B00030460CF03BFE2B461BE5531C33601778AA
:10E9C000FF2F01F00F81FE2F01F0D48030460CF0B4
:10E9D00021FE96E80C009B1A002B06DD531C3360C9
:10E9E000137813B90C2F41F22981272F00F2E2840A
:10E9F000F74B012523F817002B46FAE471680B3D0D
:10EA00008B1AEF2D00F2D68401A050F825F000BF3C
:10EA100035F60008B5F30008B5F30008B5F30008B3
:10EA2000B5F30008B5F30008B5F30008B5F3000826
:10EA3000B5F30008B5F30008B5F30008B5F3000816
:10EA4000B5F30008B5F30008B5F30008B5F3000806
:10EA5000B5F30008B5F30008B5F30008B5F30008F6
:10EA6000B5F30008B5F30008B5F30008B5F30008E6
:10EA7000DBF50008B5F30008C1F50008B5F30008A0
:10EA80009FF50008B5F30008B5F30008B5F30008DA
:10EA9000C5F60008B5F300086BF60008B5F30008EA
:10EAA000EDF60008B5F3000875F50008B5F30008A9
:10EAB0000FF40008B5F30008BFF30008B5F3000831
:10EAC0006DF30008B5F30008B5F30008B5F30008CE
:10EAD000B5F3000825E40008B5F3000841F3000889
:10EAE000B5F30008B5F3000871F40008B5F30008A9
:10EAF000D5ED0008B5F30008B5F30008B5F300083C
:10EB0000B5F30008B5F30008B5F30008B5F3000845
:10EB1000B5F300088BF40008B5F3000853F10008C2
:10EB2000B5F30008B5F30008DFF20008B5F30008FC
:10EB3000B5F30008B5F30008B5F30008B5F3000815
:10EB4000B5F30008B5F300087BF20008B5F3000840
:10EB50000BF20008B5F300089DF10008B5F30008BA
:10EB6000E5F40008B5F3000819F30008C7F400083D
:10EB700037F10008B5F30008B5F30008B5F3000855
:10EB8000B5F30008B5F30008B5F30008B5F30008C5
:10EB9000B5F30008B5F30008B5F30008B5F30008B5
:10EBA000B5F30008B5F30008B5F30008B5F30008A5
:10EBB000B5F30008B5F30008B5F30008B5F3000895
:10EBC000B5F30008B5F30008B5F30008B5F3000885
:10EBD000B5F30008B5F30008B5F30008B5F3000875
:10EBE000B5F30008B5F30008B5F30008B5F3000865
:10EBF000B5F30008B5F30008B5F30008B5F3000855
:10EC0000B5F30008B5F30008B5F30008B5F3000844
:10EC1000B5F30008B5F30008B5F30008B5F3000834
:10EC2000B5F30008B5F30008B5F30008B5F3000824
:10EC3000B5F30008B5F30008B5F30008B5F3000814
:10EC4000B5F30008B5F30008B5F30008B5F3000804
:10EC5000B5F30008B5F30008B5F30008B5F30008F4
:10EC6000B5F30008B5F30008B5F30008B5F30008E4
:10EC7000B5F30008B5F30008B5F30008B5F30008D4
:10EC8000B5F30008B5F30008B5F30008B5F30008C4
:10EC9000B5F30008B5F30008B5F30008B5F30008B4
:10ECA000B5F30008B5F30008B5F30008B5F30008A4
:10ECB000B5F30008B5F30008B5F30008B5F3000894
:10ECC00099F00008B5F3000883F000080DF1000882
:10ECD000B5F30008B5F30008B5F30008B5F3000874
:10ECE000B5F30008B5F30008B5F30008B5F3000864
:10ECF000B5F30008B5F30008B5F30008B5F3000854
:10ED0000B5F3000829F00008D7EF00089FEF0008CE
:10ED1000B5F3000803EF0008E9EE0008CDEE0008A7
:10ED2000B5F30008B3EE00084FEE000827EE000828
:10ED30001DEE00086BF90008B5F300083DF9000866
:10ED4000B5F30008B5F300081BF90008EDF800085A
:10ED5000D9F80008B1F8000891F800086FF8000829
:10ED600043F80008B5F30008B5F30008B5F3000850
:10ED7000B5F30008B5F30008B5F30008B5F30008D3
:10ED8000B5F30008B5F30008B5F30008B5F30008C3
:10ED9000B5F30008B5F30008B5F30008B5F30008B3
:10EDA00029F80008B5F30008B5F30008CFF700080C
:10EDB000B5F30008B5F30008B5F3000869F70008DB
:10EDC000B5F30008B5F30008B5F300081FF7000815
:10EDD000807D0020531C3360BA4B1278BA4F1A70F2
:10EDE00000233B6030460CF0FDFB32683B68B749BE
:10EDF000B74D0343501C3B60306013780B723046B4
:10EE00000CF008FC286030460CF004FC68603046CA
:10EE10000CF000FCA86030460CF0FCFB30460CF017
:10EE2000F9FBFFF7FFBA531C33601078060600F1B8
:10EE3000C287A84B1B78DD073FF5F4AA032828BF3B
:10EE400000200125FAF766FE2B46FFF7D2BA531CC5
:10EE50003360304692F800900CF0C4FB8046304698
:10EE60000CF0C0FB054630460CF0BCFB07463046B4
:10EE70000CF0D0FB30460CF0CDFB30460CF0D6FB4E
:10EE8000B9F1000F00F08287B9F1100F7FF4CAAA20
:10EE9000914BC3F804809D6007B1DF608F49904BB0
:10EEA0000222081F01251A701BF028FD2B46FFF7D0
:10EEB000A0BA884B1B78D8073FF5B4AA0125FBF709
:10EEC000D7F8FAF7F5FE2B46FFF793BA814B1B787C
:10EED000DA073FF5A7AA834A1378012543F0040314
:10EEE00013702B46FFF785BA7A4B1B78D9073FF58D
:10EEF00099AA7D4B4FF4C87201251A802B46FFF763
:10EF000078BA092B40F35682784F1346511C3D685E
:10EF1000316013F8021B297033605378AB70D31C37
:10EF200033609378642B02F10401A8BF64236B71F2
:10EF30003160D378642B02F10501A8BF6423AB7163
:10EF400031601379EB71931D33605379642B02F1B7
:10EF50000701A8BF64232B7231609379EB7002F133
:10EF600008033360D3792B7130460CF053FB726881
:10EF700033686881D11A00290BDD591C386831606B
:10EF8000521A002A1978417203DD9A1C32605B78AC
:10EF9000437001251FF02EFB2B46FFF72ABA544B76
:10EFA0001868D31C014621329D1E356013F8035C9E
:10EFB0000D705D1E356013F8025C4D70336013F800
:10EFC000015C8D7003339A4201F10301ECD11EF014
:10EFD000D3FBFFF727BA531C336013784149002B4A
:10EFE00000F0F4860B7843F00203901C0B70414D47
:10EFF000306053782B7530460CF0F4FA28603046B8
:10F000000CF0F0FA686030460CF004FB28813046C2
:10F010000CF000FB384AE8811378012543F0020325
:10F0200013702B46FFF7E5B9C3F34705122D00F225
:10F03000C181B5B112AB0DF1060903EB4507C84616
:10F04000423F30460CF0E6FA28F8020FB845F8D1F6
:10F050002A4B39F8022F23F8022FC845F9D1112D78
:10F0600009D8274A6B00023B13440021223223F8BF
:10F07000021F9A42FBD1234A01231D461370FFF75A
:10F08000B8B9214F002330463B600CF0ABFA0125A4
:10F0900038602B46FFF7ADB91346511C316013F8A9
:10F0A000025B3360D31C507833609178002D00F000
:10F0B0009286012D7FF4B6A926F0D6FF2B46FFF7E6
:10F0C00098B900BFCC4D00205C550020049500206D
:10F0D000EC3D0020F04B002070240020782400201C
:10F0E0000E7A00208677002006B400208C7700205E
:10F0F00088770020B85A00200C7A0020264600208D
:10F10000284600204C46002024400020531CC448C0
:10F11000336001781378002940F09D850422027045
:10F12000C04A9B001380FBF713FDBF4B01251862FB
:10F130002B46FFF75EB9531C33601378002B00F0A9
:10F14000E2854FF40040012509F0BEFD2B46FFF794
:10F1500050B9531C33601778112F00F22B81931C88
:10F160003360B24D537805F8173030460CF052FA40
:10F1700040F6CA039842A8BF184640F2EE239842D0
:10F1800005EB4701B8BF18460125A0F2EE222B4639
:10F19000192092FBF0F24A70FFF72BB9531C336031
:10F1A000A34DA44F13787B713046D5F800800CF046
:10F1B00031FAA8F820003046D5F800800CF02AFA81
:10F1C00072683368A8F81E00D11A072900F35F851A
:10F1D000D11A032900F34F85D21A002A05DD591CE4
:10F1E0002A6831601B7882F82630FAF7B9FC2AF0D9
:10F1F000C1FC914B1B68002B00F06385286801253A
:10F200001DF0EEFE2B46FFF7F4B81346511C31609B
:10F21000884F13F8021BB9703360884953780B701C
:10F22000D31C3360864D93782B71131D3360D378D4
:10F23000092BA8BF09233046AB700CF0EBF93368FB
:10F2400072682880D11A012905DD30460CF0E2F9F8
:10F2500033687268E8819A4240F03E85FAF780FC94
:10F26000336872689A423FF4DDA85A1C32601B78FA
:10F27000EB7001252B46FFF7BCB8724B1B68002BC7
:10F280003FF4D0A81BF026FCFF283FF4CBA8304663
:10F290000CF0C0F93F2840F228856B4F00253D70E7
:10F2A00033687268B880D21A012A7FF7BBA81A4661
:10F2B000591C316012F8021BB97012A8326000228A
:10F2C0005D7800F8402D1BF0D7FB9DF80830AB426D
:10F2D0003FF4A8A828461BF0F3FBFFF7A3B85B4B4D
:10F2E0001B78012B3FF69EA81046531C3360584FE5
:10F2F00010F8023BBB703060D31C50783360CB1ADF
:10F30000012B917840F3088530460CF083F90125F4
:10F3100038802B46FFF76DB81346511C31604D49BC
:10F3200013F8020BC87033604B4953784B71D31CF0
:10F3300033604A4B9278DA7001252B46FFF759B8B3
:10F340001346501C3060464813F8025B85703360EA
:10F35000557845708B423FF465A8D31C3360324B1F
:10F3600092781A7501252B46FFF743B80721B3FBA6
:10F37000F1F1C1EBC1055B1B1CD1C9B201F1FF3832
:10F380005FFA88F800293FF44DA8DFF8D8A008F10B
:10F3900001081D46531C336092F90020314B0027B1
:10F3A00093F90210914203F1080300F0F68301374C
:10F3B000052FF5D14FF0FF352B46FFF71AB8531C38
:10F3C000336013780E2BF5D8911C31605578032DDE
:10F3D000F0D82548062101FB03F14318D71C5D71C5
:10F3E000376095784554111D3160D1785970511DA1
:10F3F000316011799970911D31605179D970D11DA9
:10F40000316092791A7101252B46FEF7F2BF531C29
:10F410003360164B12785A7501252B46FEF7E9BF6B
:10F42000084D0020348C002070240020D448002097
:10F430008877002048A90020C84D0020FC4A002001
:10F4400010570020F44B0020F84B002054550020AA
:10F45000888C0020084B00204C790020184B00209D
:10F46000284B0020309500203040002004950020DB
:10F47000B14B02F108010132326012F8010C03F8BD
:10F48000010F9142F7D1FEF7CDBF1346511C3160F9
:10F49000AA4D13F8021B2971336053786B71304603
:10F4A0000CF0B8F8336828805A1C32601B78AB71B6
:10F4B00030460CF0AFF8336868805A1C32601B7815
:10F4C000EB71FEF7AFBF9E4B1B7813F001017FF489
:10F4D00071AF531C33601078012526F0FFFC2B46DA
:10F4E000FEF787BF30460CF095F830460CF092F8E6
:10F4F00030460CF08FF830460CF098F83368914D98
:10F500001946581C2A68306011F8020B82F82C004A
:10F510003160597882F83610D91C31609B7882F8B6
:10F52000373030460CF082F830460CF07FF8304629
:10F530000CF07CF830462F680CF06CF87887304679
:10F540002F680CF067F8336872683887D11A012980
:10F550000ADD591C2A6831601B7882F82E3030464B
:10F560000CF064F833687268D31A032B00F37883C5
:10F5700028682CE5511C316015781F2D3FF61AAF15
:10F58000052B7FF417AF30460CF02CF86E4B43F888
:10F590002500012521F0ECFA2B46FEF72ABF304664
:10F5A0000CF038F8694F386030460CF033F878606A
:10F5B00030460CF02FF80125B8602B46FEF719BF36
:10F5C000634F00233B6030460CF00CF83B6801258C
:10F5D00003433B602B46FEF70CBF531C336015788A
:10F5E000132D3FF6E7AE931C3360507801922CF058
:10F5F0006BFF00283FF4DEAE019A564B017803F80A
:10F600002510D11C316003EB850391785970111DD1
:10F610003160D1789970511D31601279DA70002013
:10F620001EF028FF4C4B80F00100012518702B467E
:10F63000FEF7DFBE494A102B4FF0000128BF102310
:10F64000116051609160D1601174002B3EF4EAAEFC
:10F650003168013A0B440131316011F8010C02F8B4
:10F66000010F9942F7D1FEF7DDBE531C3C4D3360CC
:10F6700013782B7230460BF0CDFFA88330460BF089
:10F68000C9FF288330460BF0C5FF32686883531CDE
:10F6900033601278EA747268D31A032B00F357832D
:10F6A0003368D11A052900F34283D21A002A7EF763
:10F6B000B9AE5A1C32601B7885F8213001252B46E3
:10F6C000FEF797BE531C3360264815780570C91A9B
:10F6D00000297EF7A7AE931C33605378003318BF20
:10F6E0000123012543702B46FEF783BE164D05F11D
:10F6F000400730460BF08EFF3368A5F88000591C98
:10F700001A46316012F8021B85F8821032605B786D
:10F7100085F883300435BD42EBD1FEF783BE084B3C
:10F720001B78DB073FF546AE0125FAF70FFAFAF72B
:10F73000BFFA2B46FEF75DBE039500208C740020B7
:10F74000F04B0020887700200C7E0020EC3D00204C
:10F750005C550020C8470020291B0020388C002061
:10F7600004950020CC4D002030460BF053FF336849
:10F77000ADF808001A46591C316012F8021B3260BD
:10F780008DF80A105A788DF80B20DA1C32609A78BE
:10F790008DF80C201A1D3260DA788DF80D205A1D74
:10F7A00032601B798DF80E3002A80023ADF81030BE
:10F7B0000BF088FEC24AC34B1268801A4FF0010555
:10F7C00061F10001C3E906012B46FEF712BE531C8E
:10F7D000336013780F2B3FF6EDAD911C3160C3EB16
:10F7E000C303B9495078C854D01C30600B44917899
:10F7F0005970111D3160D1789970511D31601179A6
:10F80000D970911D316051791971D11D3160917993
:10F81000597102F108013160D2799A7101251DF008
:10F820004BFB2B46FEF7E5BD30460BF0F3FEA74F32
:10F83000F88130460BF0EEFE0125B8812B46FEF72D
:10F84000D8BD1146531C3360A14B11F8020B187040
:10F85000316051785970D11C316091789970111DC7
:10F860003160D278DA7001252B46FEF7C2BD3046F2
:10F870000BF0D0FE974F388230460BF0CBFE7882EB
:10F8800030460BF0C7FE0125B8822B46FEF7B1BD0E
:10F890001346511C316013F8020B3360D31C5178AE
:10F8A0003360927823F06EFE00287EF4BBAD81E5D4
:10F8B0001346511C3160884913F8020B08703360FD
:10F8C000824953788B70D31C3360844B92789A7042
:10F8D00001252B46FEF78DBD814B824918684E22CB
:10F8E00001252EF0C3FF2B46FEF783BD1146531CA6
:10F8F00033607D4B11F8020B1870316051785970EC
:10F90000D11C316092789A7030460BF083FE774BB1
:10F910000125D8802B46FEF76CBD30460BF07AFEF1
:10F92000724F388030460BF075FE788030460BF011
:10F9300071FE0125B8802B46FEF75BBDDFF8C48160
:10F9400098F80030002B3EF46DAD694F002530462D
:10F950000BF060FE1EF066F898F80030A7EC010A84
:10F9600001359D42F3DBFEF75DBD0D2B7FF422AD2B
:10F97000531C33601578072D3FF61CADDFF88881E6
:10F9800030460C270BF046FE07FB05F708EB070592
:10F99000A88030460BF03EFEE88030460BF03AFE81
:10F9A000336828811A46591C316012F8021BA9726B
:10F9B00032605B78EB7230460BF014FE012548F89C
:10F9C00007002B46FEF715BD1346511C3160494D0B
:10F9D00013F8021B6970336053782B70D31C3360AB
:10F9E0009378AB7030460BF015FE33682881591CB4
:10F9F0001A46316012F8021B697132605B78AB7194
:10FA000001252B46FEF7F5BC336872689A4240F038
:10FA10009F802C4BFF221A704FF00009364D25F0C5
:10FA2000E1F949462022354885F8009030F0B1F8D8
:10FA30008DF808909DF80830072B00F20A81DFF856
:10FA4000CC802E4E4A469DF8083003EB430308EB6A
:10FA5000C3035B7CE3B19DF8083003EB430308EB81
:10FA6000C30320215B699BB19DF8083003EB43037E
:10FA700008EBC303586946F822000AF0ADFF2B7863
:10FA800056F823000BF066F82A780132D2B22A70B9
:10FA90009DF808300133DBB28DF808309DF808304E
:10FAA000072BD0D92368591C21601A70002F3EF40F
:10FAB000B9AC134B3B6001252B46FEF79ABC00BF47
:10FAC000E8B3002070240020383F0020084B0020BD
:10FAD0001C7B00201057002048A90020184B002054
:10FAE00088770020FC250408004B00207474002057
:10FAF00064430020207700204D410020383E002044
:10FB000005EA0108EC6D0020783E002088B2002054
:10FB1000B44AB54D92E84200FEF7ACBEB24D6968FA
:10FB2000AE68FEF7A7BE30460BF074FDAF4FFEF790
:10FB300030BD931C3360AE4B51781970D11C3160CD
:10FB400091785970111D3160D2789A70FEF76ABCB5
:10FB50005A1C326013F8022BA3493360FF2A0A7043
:10FB60003FF45AAF22680125531923602B461070C9
:10FB7000FEF73FBC931C33605578022D3FF61AAC5C
:10FB800030460BF047FD9B4B03EB45034FF0FF3531
:10FB9000A3F856002B46FEF72CBC0AEBC7093046EB
:10FBA00089F802200BF036FD33682AF837001A4630
:10FBB000591C316012F8021B89F8031032605A7820
:10FBC00089F80420DA1C32609A7889F806201A1D18
:10FBD00032600135DB7889F80530A8457FF4DAAB6F
:10FBE000FEF720BC931C3360834B51781970D31CF3
:10FBF0003360804F937887F85530131D3360D37886
:10FC000087F8543030460BF005FDA7F85000304619
:10FC10000BF000FD30460BF0FDFC96E80C009B1A43
:10FC2000012BA7F852007EF7FDAB30460BF0F2FC3B
:10FC30000125A7F85A002B46FEF7DBBB6D4B0030C1
:10FC40001F4418BF0120012587F85E002B46FEF7F0
:10FC5000D0BB4A4626E704297EF4E4ABFFF760BA3E
:10FC600030462F680BF0D6FC788630462E680BF0B5
:10FC7000D1FCB0867CE430460BF0CCFCF8813046F9
:10FC80000BF0C8FC336872683882FFF7A5BA3046BB
:10FC90000BF0C0FC788130460BF0BCFCB8813046DC
:10FCA000D5F800800BF0B6FCA8F822003046D5F855
:10FCB00000800BF0AFFC33687268A8F82400FFF7EF
:10FCC00087BA4E484E494F4A4F4B036001250B609F
:10FCD00013602B46FEF78DBB5A1C32601B78003335
:10FCE00018BF0123FB71FFF7B9BAC50800F007037D
:10FCF00001350133EDB2454F284619467B7017F0A8
:10FD000025FEFFF7CCBA424A1368012523F40043CD
:10FD100013602B46FEF76DBB3E4B1A88012512FB84
:10FD200000F22B4692FBF1F23A80FEF762BB5A1CBE
:10FD300032601B78EB7230460BF054FC3368E8609D
:10FD40005A1C32601B782B7433687268ADE43046FD
:10FD50000BF060FCA88430460BF05CFC33687268E2
:10FD6000E884D11A03297FF79CAC1A46591C3160EC
:10FD700012F8021BA97732605B7885F82030304694
:10FD80000BF048FC3368726868848AE4154B1020D5
:10FD9000C3F800805D6008F067FF1F4A137843F0E6
:10FDA00001031370002F3EF43DAB0F4B0125DF60C4
:10FDB0002B46FEF71EBB00F07F00032828BF002063
:10FDC000012526F06DF92B46FEF713BB0B7803F0E7
:10FDD000FD03FFF70AB901251DF052FB2B46FEF784
:10FDE00008BB00BFE479002070240020F84A0020FE
:10FDF000FD530020807D0020088F0020186F002018
:10FE00006C6F00206C73002049A10108F84B0020A2
:10FE10008077002052490020867700202DE9F04F9E
:10FE20002DED068BA04BA14A1C7897B000F59C41A4
:10FE3000203181460B911160002C00F0E9869C4A2C
:10FE40001268904240F285809A4A069216689A4952
:10FE50009A4A0591013C1C70994B049206F4805615
:10FE60000893002E40F08380964B1B78022B01F004
:10FE70002C81042B01F0C581012B01F07981924B7B
:10FE80009945089B9B7800F29285002B40F0938562
:10FE90008E4B0793069B1E6816F4805740F08686AB
:10FEA000DFF85892049BB3F90610059B5D8BA942BD
:10FEB000B4BF00250125DFF83C82D8F8003013F0EC
:10FEC00080535ED0079A127812F001025FD0059835
:10FED000408C884241F39E82002D5ED17C4C94F888
:10FEE0008C10002959D17B487B49006890F82D007F
:10FEF00000240C604C608C60784900284ED108705A
:10FF0000002A4FD0F1064DD5754A1278D20649D451
:10FF1000002F47D1002B45D1740243D4714B1B787D
:10FF2000002B02F03782704B9B78002D42F0AB82A1
:10FF30003BB16E4A6E4B12681B689B1A002BC2F2D3
:10FF400090821020624C2CF0A9F8012384F88D30A7
:10FF500028E0584B06931E68584B574A049306F402
:10FF60008056574B05920893002E3FF47DAF002139
:10FF700060480CF08DF800287FF476AF24F06EFF17
:10FF800072E770029ED4079A127802F00102504C78
:10FF9000002184F88C10002DA5D050490120087054
:10FFA000002AAFD1544B1A78002A40F0B38005994B
:10FFB000049C488BB4F90070898BB4F90240B842B4
:10FFC000B4BF8026002646F04003B942D8BF33466E
:10FFD0009B0843F080068442C8BF3346049F43F029
:10FFE00040068C42B8BF33469B08B7F90440B7F9C6
:10FFF000066043F080078442C8BF3B4643F0400799
:020000040801F1
:100000008C42B8BF3B469B0843F08007304C864289
:10001000C8BF3B4643F0400794F88EE08E42B8BF1D
:100020003B469E4501F0AA84A4F8902084F89220D3
:100030002C4984F88E300E78002E01F073835F2BEC
:1000400001F01F846F2B01F03A84079B1B78DB07BC
:1000500060D494F8921000295CD1B4F99030322B1E
:1000600058DD94F88E200120572A84F8920001F080
:10007000D187069B1B685D0741F1C0825A2A41F077
:10008000BD8294F89430002B42F0948194F896301D
:1000900083F0010384F89630002B42F0D6810C20C7
:1000A0002BF0FCFF01F001BC60470020244600203B
:1000B0005C47002048B10020049500204A8C0020B5
:1000C0008C790020084D0020404B4C00F04B002064
:1000D000A024002088770020804D002020270020C9
:1000E00086770020291B0020284B0020E8B3002041
:1000F000B88E0020D44A0020C755002018480020A0
:100100000F202BF0CBFFB4F8903084F89250FA3BDC
:10011000A4F89030069B1B68854A864E09925907C1
:1001200000F1CA86844B0C930DF1500B1D46002341
:10013000CBF804300A96149340F6330A192740F29C
:100140008334049E02E004354D4522D0A978EB7833
:10015000994217FB0140F6D295F801E00EF1040E2A
:1001600017FB034136F91E305345A8BF5346B3F57C
:10017000617FB8BF4FF461739842E4DA9942E2DBE1
:1001800029782729DFD8584604350BF071FF4D45F3
:10019000DCD16A4B0A9E1B789BE8030088E80300C9
:1001A000002B40F0FF85664B1B78002B00F072851A
:1001B000012164480BF06CFF002840F0E582089BA9
:1001C000DB78002B40F0E082DFF8949133881CB29A
:1001D00024F00104A7B2BB42378001F020805A4CC2
:1001E0004FF002080E204FF0140B4FF0FF0A84F876
:1001F000008084F801B084F802A02BF04FFF414644
:10020000504837880BF044FF002841F0D88227F08F
:1002100002039BB2BB4233800AD04B4B0220142115
:10022000FF2218700E2059709A702BF037FF378814
:10023000464B474A197850680A93BC0708BF81F0BB
:100240000201C1F340010B920AF08AFC24213D48CF
:100250000BF01EFF30B9079A1378590744BF23F0FB
:1002600004031370D9F8003013F00A0F1DD00521D4
:1002700034480BF00DFF002801F0A280348862079B
:1002800041F15D822F4806210BF002FF002801F0AA
:100290008480630641F15B8207212A480BF0F8FE57
:1002A000002840F0DD87D9F800309F0600F1F28584
:1002B000B6F80080274F23480C210BF0E9FE0028F8
:1002C00000F0498348F480734345338009D01E4BC6
:1002D000022214211A700E20FF2259709A702BF0FE
:1002E000DDFE1D4B1B78082B00F041830E2B00F028
:1002F0003E83069B1C68600569D5184B1B79002B53
:1003000000F02D8214210F480BF0C2FE002840F0AF
:100310002B821FF011FB01200CF0FAFD002854D0B5
:10032000DFF840A000244FF0CC0BA9461FE000BF2F
:100330008C77002084770020C847002034570020A5
:100340008C440020D44A002058410020B0B3002043
:10035000B4B300202C4C0020CC4D00201C4C0020BD
:10036000307700202C290020DCB2022C2CD80BFB8B
:1003700004F8631C5AF80850002DF5D1032290F9B7
:10038000023002950192C278E24951F8222000928F
:1003900018462A462B4601210CF03AFC034604EB92
:1003A000440000EB00100D9353B129460AEB800086
:1003B000CC222FF0EEFB0D9B4AF808300134E4B25A
:1003C00029F096F90028D0D14D46069B1C68079B62
:1003D00093F800A0D04B1AF0010A00F035820122F8
:1003E0001A70099B04991B68B1F906105A89CB4809
:1003F0004FF0010E914280F800E080F20B82C84B72
:100400004FF07E521A60C74A059B0498B3F81880D3
:10041000B0F900E092F90430107892F801C0002B96
:10042000AEEB080314BF01224FF0FF32002BB8BF20
:100430005B42B3F5FA7FA8BF4FF4FA73984280F29B
:10044000E6811B1A07EE903AF8EEE77AC645C7ED4B
:10045000007A03DAF1EE677AC7ED007A049BB3F90C
:1004600002E0AEEB0803002BB8BF5B42B3F5FA7FA6
:10047000A8BF4FF4FA73984280F2C6811B1A07EEA8
:10048000903AF8EEE77AF045C7ED017A03DDF1EE38
:10049000677AC7ED017A049BB3F90400A0EB080367
:1004A000002BB8BF5B42B3F5FA7FA8BF4FF4FA73D5
:1004B0006345CCBFA3EB0C03002302FB03F307EE61
:1004C000903AF8EEE77A4045C7ED027ABCBFF1EE0C
:1004D000677AC7ED027A14F4805400F07281B1F5A6
:1004E000FA6F914BA8BF4FF4FA61B1F57A7F1A7891
:1004F000B8BF4FF47A71A1F57A71002A41F02F81CB
:100500008A4ADFF840E282FB0130CB17C3EB60136D
:10051000581C6FF0630C3EF910003EF913E00CFB21
:100520000313A0EB0E0003FB00F382FB0312DB17A7
:10053000C3EB62139E440FFA8EFE07EE90EAB8EE0C
:10054000E78A87ED038A002C40F0448433885A06FA
:1005500040F1FA807649774A91ED018AD2ED019A0D
:1005600092ED026A91ED034A92ED030A91ED029A2F
:1005700092ED007AD1ED005AD7ED011A97ED002ADD
:100580006D4A6E4938EE445A79EEC63A77EE007AF3
:1005900065EE233A75EEC96A75EE890A37EE401AA0
:1005A00066EEA76AB0EE633AA0EE813A13F0030359
:1005B000B0EE665A78EE044A79EE867AA0EE815A59
:1005C000F0EE638AA4EEA73AD4EEA78AA4EEE75A27
:1005D00033EE263AF0EE687AF0EE674AF6EE008ADD
:1005E00035EE88AAE0EEC14A28EEC33A35EE635AEA
:1005F00077EE293A77EEE67AAAEE233A25EE285AE4
:1006000076EE403A34EE49AAE0EE817A74EEA64ADC
:10061000AAEE235A34EE094A37EE697A64EEA84A04
:1006200063EE036AE4EE074A75EEC85A36EE006AD6
:1006300067EEA87AB0EE667A95EE057AE5EE056A81
:10064000E5EE867AB1EE648AF0EE665AF0EE476A1D
:10065000B1EE674AE8EE246A63EE270A67EEA43A31
:10066000E4EE275AB1EE450AB0EE609AB0EE631A96
:10067000A4EE277A23EE244AE7EEA76AA5EE249A91
:10068000A0EE031AE8EE245AB0EE448A31EEA16AD5
:10069000E0EE240AA5EE278A66EEA16A72EE028ACF
:1006A000E5EE033A61EE211A26EE096AA4EEA47A79
:1006B000A0EE274A0CBFD7ED022ADFED212A82EDFA
:1006C000005AA2EE256AE8EEA06AE2EE081A73EE7E
:1006D000A33A27EE227A34EE044AF0EE005AE3EE13
:1006E000A26AA4EE226AA1EEA57AC7ED016AC1ED65
:1006F000376A81ED366A87ED006A81ED387A82EDDE
:10070000013AC2ED027AC2ED034AEBB987ED027AF3
:100710001AE000BF74260408F14B0020582700207F
:10072000D0260020004B0020C02800201F85EB5160
:100730007C070020CC02002004030020A02400201D
:100740000000000094740020BAF1000F40F02281F4
:100750002BF0EEFE17B0BDEC068BBDE8F08F079BCB
:100760001B78D9077FF5D5AD4FF40F701BF06EFBEA
:1007700000283FF42AAE0CF035FA4FF40F701BF04E
:1007800011FB0028F7D120E6DFF88C93D9F8003070
:1007900099077FF51BAD3788FA073FF538AD47F06D
:1007A00001039F4233803FF432ADC54B0222142136
:1007B0001A700E20FF2259709A702BF06FFC378848
:1007C00025E5059B5A8B9142C0F27C84B1F5FA6F06
:1007D000D4BFC2EB0101C2F5FA614FF47A7303FB97
:1007E00001F1B8480378C2F5FA62B1FBF2F1002BCF
:1007F0003FF486AE4378B44A01FB03F182FB012348
:10080000C917C1EB63117BE6DFEDB07A3BE6DFEDA4
:10081000AF7A1BE6B1F5FA6F80F24D84187A8B1A25
:1008200003FB00F3C2F5FA6293FBF2F3C3F1640336
:1008300007EE903AF8EEE77A9FEDA57AA54B67EEC2
:10084000877AC3ED007ADEE51B780693002B7FF4F0
:10085000C8ADA14A1268002A3FF4C3AD9F4A07926F
:1008600012F8030CDFF8B4B21146A2F103091DF02F
:1008700025FE9BF80080079A002800F03386069B2F
:10088000B8F1000F59D109F1080199F805001DF0E0
:1008900015FE002841F06385914999F80A001DF082
:1008A0000DFE002800F03386B8F1020F41F05385A9
:1008B0008C4999F80F001DF001FE002841F0478592
:1008C000894999F814001DF0F9FD002800F03386DD
:1008D000B8F1040F41F03785844999F819001DF0EB
:1008E000EDFD002841F02B85814999F81E001DF08F
:1008F000E5FD002800F03386B8F1060F41F01B85B6
:100900007C4999F823001DF0D9FD002841F03A8573
:10091000794999F828001DF0D1FD002800F03386B0
:10092000B8F1080F41F02A85744999F82D001DF09F
:10093000C5FD00283FF455AD09231A4602EB82029B
:1009400091446F4A99F8010099F802108BF8003031
:100950001070517045E528F480739BB24345338095
:100960007FF4B5AC674B1B78082B7FF4BFAC3288A3
:1009700022F040039BB29A4233803FF4BAAC504B12
:10098000022214211A700E20FF2259709A702BF047
:1009900085FBAEE40A9B19780B9B01F001011868F6
:1009A0000AF0DEF817B0BDEC068BBDE8F08F13B986
:1009B000089A01239370544B089A1D7892F82140AD
:1009C00007931B201DF0B2FD012C05F001088146A4
:1009D00000F0728705F00205089A4C4E92F820301C
:1009E000DFF83CA14A4F09959346052B00F2DE87BC
:1009F000DFE813F0C100B7000600FF000101F400BA
:100A0000012C04BF05238BF82030B8F1000F12D061
:100A1000059B3088B3F918100022134661F30F02CA
:100A200060F31F4261F30F03049861F31F430360F7
:100A3000032342600993374DDBF814102A68914272
:100A400080F0608647F230510322CBF81C108BF8FF
:100A50002020022008F038F924F000FA2968DBF899
:100A60001C200A440421CBF818208BF82010012CFC
:100A700040F0E2872A68DBF81810914280F09687F0
:100A80009AF8000020B91DF051FD002840F08E8733
:100A90003A6822F002023A602A687388642101FBF6
:100AA00003234FF480600022CBF810308BF8202015
:100AB0008BF8032008F0D8F89BF8203095E700BFAA
:100AC00058410020C02800201F85EB510000000085
:100AD0000AD7233CD0260020F44B00201A410020E6
:100AE00024410020294100202E41002033410020D4
:100AF000384100203D410020424100204741002074
:100B0000F84B0020CC4D0020F04B00208C740020CE
:100B100080770020E8B30020307700207A000020A2
:100B2000291B00201DF008FD012807D1AE4D728859
:100B30002B68642101FB0233CBF81030B9F1000FB0
:100B400002D0B379002B4BD1012C00F02F87A64D9A
:100B5000DBF810102A689142C0F07B8701238BF8E4
:100B60002030012C3AD0F379012B46D01DF064FCE3
:100B70009BF8203039E7B8F1000FD3D1099D4FF42D
:100B80008060B9F1000F00F0688308F085F8089ADA
:100B900000231361002D3FF47DA928462BF07EFA37
:100BA000069B1E6816F480573FF47AA91D218F48D2
:100BB0000BF06EFA00287FF473A98D4B03F15009F6
:100BC00003E00433994500F0F7861A78262AF8D115
:100BD0009978DA789142F4D2FFF764B9824D5BE7F5
:100BE0001DF02AFC03224FF47A738BF82020CBF8F7
:100BF0001C307D4D2DE77C4D39E71DF01DFC032297
:100C000040F6B8338BF82020CBF81C30764D20E727
:100C1000784F3B78002B01F05C82774BDFF8E8815E
:100C2000DFF8E8B1DFF8E8A1059345465E46049099
:100C300099460EE019F804109847032C28DC88B96F
:100C40003B782AF8020F01349C4205F1040580F23A
:100C50005881072CE1B23046DBF80430EADD9847D2
:100C600000B2EDE738F824206B88801A4FF47A71CF
:100C70009B1A01FB00F040F6CA0290FBF3F0084417
:100C8000904240F2EE23A8BF10469842B8BF1846E3
:100C900000B2D5E7DFF87CB1DFF87C91574C98467D
:100CA0000BF15A074FF0010A59461BF8010C1DF0D1
:100CB00005FCF8B19BF804009BF802309BF803E0B8
:100CC00000EB400104EB8101013BD1F8A02003EBD4
:100CD00043034B4493420DD094F8CC2081F89CE020
:100CE0000AFA00F022EA0000C1F8A030C1F8A4809E
:100CF00084F8CC000BF1060BBB45D5D1404B3A4AEA
:100D00001B780A93099BD2F800801B68DFF80CA1BE
:100D10000B934FF0FF394FF0000BDAF80430002B43
:100D200037D01F78002F34D0DAF80820A8EB020261
:100D3000002A11DB314C012194F8CC2001FA0BF18F
:100D400022EA010284F8CC202E4A08F5FA704FF00E
:100D5000FF31CAF8080011600A9AD2B19AF800204F
:100D600059780432D2B2002940F05A830599049888
:100D7000098B30F9122001F1C800824240F32D8620
:100D80001E4C9A7894F8CC3043FA0BF3DB0740F111
:100D9000B2860BF1010BBBF1040F0AF10C0ABCD1B6
:100DA000FFF706BA124B03E00433AB423FF4FBA952
:100DB00019782329F8D19878DA789042F4D20B4840
:100DC0000BF066F900283FF4EEA914202BF066F929
:100DD000FFF7E9B91D2105480BF05AF9002840F04A
:100DE000A6850C9B20E000BFE8B30020D44A002079
:100DF000C84700208C48002004950020A024002033
:100E00008179002078070020A048002010460020AB
:100E10009E2400203140002000FD03083C250020D6
:100E20000433AB423FF492AB19782629F8D1987875
:100E3000DA789042F4D2089BDB78002B7FF486AB03
:100E4000B4480BF025F9DFEDB47A002801F05881A1
:100E500038EE678AB14AB249FDEEC87ACDED047A20
:100E6000BDF910301B0382FB0302DB17C3EBA21298
:100E7000C8F57A731BB203FB02F343F30F33434409
:100E800007EE903AF8EEE77A0123C7ED037A0B708C
:100E9000FFF75CBBA34B1B789C0704D5A24C237DBA
:100EA000042B00F2E185B6F8008018F0300F40F016
:100EB00078839E4FFFF7FFB99D4C94F896305BB155
:100EC000079B1B78DA0707D5049BB3F90620059B1F
:100ED0005B8B9A4200F3FD8511218E480BF0D8F808
:100EE000002800F0828294F89A302BB994F894305C
:100EF00013B93223A4F89830012384F89A30FFF70D
:100F000011B9DDF810908B4A06928449126842F2BA
:100F1000010AA1FB091B12EA0A0A4FEA9B1B00F017
:100F20007682854D8548864C86492E7800782670D5
:100F300008701EB183490E7886F001067C4C0F21A3
:100F400084F82410002B00F00D84059D7E4BB5F82D
:100F500026C0B5F824E0059D109318462D8B007827
:100F60007A4B129594F825500995794D0495A3FB79
:100F700000535B0803EB4303C31ADBB20F90CDF8B9
:100F800034C002F480520C9304F128000BF59673E0
:100F9000CDF8449097F80080DDF82490DFF8C8C1C0
:100FA00009946B4C0E91139200210A930896CDF888
:100FB0001CE0089B002B00F04783099B079D33F939
:100FC00011201FFA82FEAE454FEA410303D30D9D67
:100FD000AE4540F27E835CF82120934580F03E834D
:100FE000E25EBAF1000F40F0538301314145E25215
:100FF00000F10600DDDB0E9A099C564B84F8242094
:101000000F2A49460CBF01220022DDF8449084F8E3
:1010100025101A7000F0AD834F4B4849494ADFF85C
:101020004CB108931C46042001230B70137007F089
:101030004BFEDBF80030A1686268E3605B1A934204
:1010400084BF002384F82130069B3C781E68002C66
:1010500001F07780059A414DB2F824E0178B3C49A6
:1010600016F48056284640F0BC8332460EE04378A2
:1010700003EB830303EB830303F2EE239BB2013202
:10108000944221F8023B00F102000ED015F8123014
:10109000002B00F02283022BE9D001320B8821F8CB
:1010A000023B944200F10200F0D1109A1378013310
:1010B0001370FEF7D6BE1B7AC3F1640307EE903AB5
:1010C000FFF7B8BB2146FFF78CBB059A0499537D07
:1010D000D27D013B31F913301AB1C3F53B630833BC
:1010E0001BB2A3F57A7307EE903A9FED1D7A1D4A65
:1010F000F8EEE77A40F2FF3167EE877AFCEEE77AA6
:10110000CDED077ABDF81C308B4228BF0B4613800B
:10111000FEF7B5BED44A002000007A44D34D6210D9
:101120004C27002086770020B85A00202C4C002045
:10113000A024002048B10020EC45002088000020B9
:1011400081790020890000207D470020ABAAAAAA4F
:101150004A8C0020D84D00208C790020D4480020F3
:101160006F12833F348C002080470020E8B30020BA
:10117000BE4CD4F88830A9EB0303002BFEF67FAEFB
:10118000BB4ABC4B527C059933F812308A7DDFEDA7
:10119000BA6A9FEDBA6AC97D9BB207EE102A07EEC4
:1011A000903AB8EEC77AF8EEE77A27EE267A67EE3D
:1011B000867A0B9AC4F88820C7EE876A40F2FF321D
:1011C000FCEEE67ACDED077ABDF81C30934228BFDD
:1011D000134609B1D31A9BB2A948AA4D0178AA4C6B
:1011E00035F81160226825F81130921B1344013143
:1011F000A64D236001F00F021B0902702B80FEF741
:101200003EBEF9F7A5FCA24BA24A1B68C31A934243
:101210007EF735AE9D4B00221A80FEF730BE0221CC
:101220009D480AF035FF00283EF4F1AF3480BB073B
:101230003EF5FEAF47F00203BB4233803EF4F8AF09
:10124000964B022214211A700E20FF2259709A70B8
:101250002AF024FF3788FEF7EBBF07F005FD96E480
:101260008F4AB2F90030002BB8BF5B42B3F5E17F83
:10127000BFF619A8B2F90230002BB8BF5B42B3F534
:10128000E17FBFF610A8874B93ED057AD3ED077A7F
:10129000D3ED096A93ED030A77EEA67A30EE070ADA
:1012A000F7EE000AB0EE007AE7EEC70A30EE000A69
:1012B0000AF03AFCB6EE008A20EE488A9FED7A0AE0
:1012C00038EE000AFDEEC07A17EE903A2033402B3C
:1012D00040F20D849FED750A754ADFED747A82ED58
:1012E000000ABDEEC87AC2ED017A17EE103A20333B
:1012F000402BC2ED027A49D8DFED6E7AB4EEE78A70
:10130000F1EE10FA41F34280DFED6B6A9FED6B7AEC
:1013100001E0B0EE678AB4EEC78AF1EE10FA78EE1B
:10132000667AF6DC9FED667AF4EEC77AF1EE10FA93
:1013300041F149809FED606ADFED626A01E0F0EE05
:10134000477AF4EEE67AF1EE10FA37EE867AF6D4C2
:10135000DFED557AB4EEE77AF1EE10FA40F39E86AF
:10136000DFED547A37EEC77A27EE076ADFED565A7B
:10137000DFED566ADFED567AE6EE256A67EE065A2D
:10138000E6EE267AA5EEA77AF0EE477A0A20C2EDBD
:10139000037A2AF083FEFEF786BF24F040039BB257
:1013A000A34233803EF478AF3C4B022214211A70E2
:1013B0000E20FF2259709A702AF070FEFEF76CBF63
:1013C000338823F00404A4B2A34234803EF45AAF1D
:1013D000324B022214211A700E20FF2259709A708B
:1013E0002AF05CFE3488FEF74DBF94F89430002B51
:1013F0003EF498AE079B1B7813F001037EF492AE87
:10140000012284F8943084F89520FEF78BBE314990
:101410000E788EE5154C012184F88C10FEF7BDBDC9
:10142000012900F0B285B9F1FF3F104C0BD01B78B9
:101430000C2B08D0284B294A03EB8707284BC3F80D
:1014400000907B6C136094F8CC20012303FA0BF31B
:101450000BF1010B1343BBF1040F84F8CC300AF1FC
:101460000C0A7FF45AACFEF7A3BE00BFA0240020F4
:1014700088B30020A8B300200000C84200008044C8
:10148000094D0020104D00200C4D0020348C002010
:101490009024002060E31600D44A00205841002028
:1014A00034770020DC020020DB0FC93F0000000081
:1014B0007C070020DB0F4940DB0FC940E4CB16411D
:1014C000DB0F49C0E4CB16C192E741B99730083C25
:1014D00015A82ABE8179002000FD0308748C002025
:1014E00078070020511D99F805001CF0E7FF00283F
:1014F0003FF4D2A9B8F1010F40F0318709F10D0195
:1015000099F80A001CF0DAFF002840F02487C1494E
:1015100099F80F001CF0D2FF00283FF4D1A9B8F1D0
:10152000030F40F01487BC4999F814001CF0C6FF63
:10153000002840F00887B94999F819001CF0BEFF4F
:1015400000283FF4D1A9B8F1050F40F0F886B4495E
:1015500099F81E001CF0B2FF002840F0EC86B1495B
:1015600099F823001CF0AAFF00283FF4D1A9B8F194
:10157000070F40F00787AC4999F828001CF09EFF40
:10158000002840F0FB86A94999F82D001CF096FF31
:1015900000283EF426AFB8F1090F3EF422AFFFF762
:1015A000CBB9102007F060FB202007F05DFBA04BBB
:1015B000B6F800809F4F00221A709F499F4AA04CA6
:1015C000A04800230B60A04923604FF0000E036089
:1015D00053609361C2F800E0C2F808E0C2F814E07A
:1015E000C2F81CE0C1F800E04B60C1F808E0C1F8A7
:1015F00014E08B61C1F81CE0FEF75DBE5D2A00F0CF
:101600007F825B2A00F069855E2A00F0E285562A17
:1016100000F0F985972A00F0A686A72A00F0CD856C
:101620008A4E3388980740F09885A2F1B703072BBC
:1016300000F2C482DFE813F09002C202C202C202CA
:101640008202C20274027402079B002B3FD05CF836
:10165000212093454FEA4103FFF4C2AC7C4A7C4D04
:10166000D25C05EB030E002A00F09C80022A47D1D1
:101670009EF8012002EB820202EB820202F2EE22CD
:1016800092B2032933DD12B2BAF1000F3FF4ADACD0
:101690000C9D20F81520B9F1000F03D10F9D022DEC
:1016A0007FF6A3ACB0F802900288B0F804E04A4498
:1016B0009644684A0FFA8EFE82FB0E52664DA2EBEC
:1016C000EE7225F803E012B24FF001098DE41A46DC
:1016D0004B000A9D4CF8215083E4D3B2022B04D96D
:1016E000032B7FF4DAAC7346C9E43B46C7E401251B
:1016F00005FA01FE0E9D25EA0E0512B20E9570E464
:10170000E25ABEE7554A1278002A7FF49BA9B8F145
:10171000000F3FF497A9012C40F048819BF820303E
:10172000FFF763B931464E480AF0B2FC002800F0DA
:10173000DA8084F8936023F087FEFEF786BC44F0DD
:1017400004039C4233807FF443AEFEF79BBD44F01C
:101750004003A34233807FF427AEFEF79DBD5B7844
:10176000FFF749B83F4B404A109201221A703F4B95
:1017700004931B213A480AF08BFC00287FF44CAC00
:101780003B4BDFF8F0B008931946DBF80030CA682D
:101790008B609B1AC82B00F2A484069B1E6806F47B
:1017A000805682E4CAB2022A40F2EC83032AA7D10F
:1017B000129A139D079E002D08BF324661E727F05D
:1017C00001039BB2BB4233803FF431AD0E2084F85D
:1017D000008084F801B084F802A02AF05FFC37880A
:1017E00025E500220FE0437803EB830303EB83033B
:1017F00003F2EE239BB20132A24221F8023B00F138
:1018000002003FF452AC15F81230ABB3022BEAD011
:101810000B88F0E7294100202E41002033410020B1
:10182000384100203D410020424100204741002036
:101830000E7A00202C4C0020F87A0020A87A002094
:10184000F4260020B4270020D07A002084770020DE
:10185000D44800205655555510250020102700204B
:10186000D44A0020D84D00207D4700204A8C00201B
:101870008C790020E8B30020D3B2032BC8D83B46B4
:10188000B9E7B2F5FA7FFEF645AC94F89230002B3A
:101890007EF440AC079B1B78012213EA020584F812
:1018A00092203EF42DAC23F0D9FAB24E069BB24AF8
:1018B0001B680992FEF733BC0025FFF78DB8B2F51F
:1018C000FA7FFEF627AC94F89220002A7EF422AC30
:1018D000079B1B78012184F89210D90700F1D5836A
:1018E00023F0B2FDE1E7079BA44A1B781060D807FC
:1018F0007EF5AFABA24B1B78002B3EF40BAC089BE4
:10190000DB78002B7EF406AC94F893300133DBB225
:10191000032B84F893307EF6FDAB9A4B5B7813B9BA
:10192000002D7EF4F7AB23F099FAFEF78EBB089BEF
:10193000DB78002B7FF455AADFED937A934938EEDC
:10194000678AC8F5FA63FDEEC87A1BB2CDED047A5A
:10195000BDF91020120381FB0201D217C2EBA112C4
:1019600003FB02F343F30F33434407EE903AB8EE20
:10197000E78A0C9B87ED038AFFF756BA844A8349AE
:101980001068B4F99020C66981FB06018911F61729
:10199000701A00F5FF407F3082423EF749AB891B49
:1019A0000A4412B2A4F89020FEF742BB099D002D14
:1019B0003EF470AAFFF7F1B8764A059BD588049AE1
:1019C0001B8BB2F906105A1B91427FDD2B449942C2
:1019D000B4BF00250125FEF76EBAC8398A426E4CA5
:1019E00065DA9A7894F8CC3043FA0BF3D8073FF5D0
:1019F000D0A9524201200D922AF076FC7B1E0D9A4E
:101A0000162B00F2A283DFE813F00A02F101D401E1
:101A1000370223028D016201820268029D02BA012F
:101A2000A0033702BB028D01620182026402B70289
:101A3000490134011B010201AB460899DBF8002083
:101A4000CB69099D13448B61002D3EF423AAFFF757
:101A5000A4B81CF0F1FC032140F6B8328BF820103A
:101A6000CBF81C20FEF7F5BF0A201CF05FFDB6F88E
:101A700000808146002800F0ED8218F0100F00F081
:101A8000D183454C94F8D490B9F1000F7FF411AA9A
:101A9000424F0D202AF002FB012384F8D430B6F81F
:101AA0000080B9F1000F7FF488ADFEF704BC94F814
:101AB000CC30012202FA0BF223EA020308F5FA7293
:101AC00084F8CC30CAF80820FFF763B90125FEF787
:101AD000F2B9002132480AF0DBFA00287FF4FCA9B1
:101AE000322384F89600A4F89830FFF7F5B909F08E
:101AF000A1FFFFF7F1BB002A0CBF012002207AE70B
:101B0000284B002201202849284C0B601A4B0993CE
:101B100022702AF0E9FB069B164E1B68FEF7FFBAFF
:101B2000154A224B09921146214A0A6002225A7034
:101B30001CF060FD069B1B68FEF7F1BA0E4A1B4BBA
:101B4000099211461B4A0A6000225A701CF052FD8D
:101B5000069B1B68FEF7E3BA074A144B099211462D
:101B6000154A0A6001225A701CF044FD069B1B684E
:101B7000FEF7D5BA847700208C770020BC8E002039
:101B800081790020284B002000007A44D34D621058
:101B90006C79002074740020A02400202C4C0020BC
:101BA000D44A00201254002088770020E0A60020AC
:101BB000365500201E5500202A5500209E2A00F090
:101BC0003C849D2A00F03184AE2A00F02684AD2AA0
:101BD00000F01B84EF2A00F01584FD2A00F0008439
:101BE000FB2A00F04984FE2A00F04384F72A00F023
:101BF00055847B2A7FF45AAE4FF4FA61022024F018
:101C00006DF9CE4B0993069B1B68FEF788BAD4F892
:101C1000D000CB4B90F836909B789144B9F1640F8B
:101C2000A8BF4FF0640929EAE97980F83690002BC3
:101C300040F03F841BF0A0FDDAF80430FFF7F7BB5B
:101C4000D4F8D000BE4B90F837909B789144B9F10E
:101C5000FE0FA8BF4FF0FE0929EAE97980F8379016
:101C6000002BE7D0162049461CF0AAFCD4F8D0007F
:101C7000E0E70B99B24B91F801909144B9F5967F4A
:101C8000A8BF4FF4967929EAE97981F801909B7809
:101C9000002B40F00684D4F8D000CBE7D4F8D00075
:101CA000A74B90F802909144B9F1C80FA8BF4FF02C
:101CB000C80929EAE97980F802909B78002BB9D00D
:101CC000142049461CF07CFCD4F8D000B2E7D4F8CC
:101CD000D0009B4B90F8049099789144B9F1C80FCB
:101CE000A8BF4FF0C80929EAE97980F804900029D3
:101CF00040F0E583102F9DD090F801909144B9F108
:101D0000C80FA8BF4FF0C80929EAE97980F8019007
:101D10009B78002B8ED0132049461CF051FCD4F840
:101D2000D00087E7D4F8D000854B90F803909978DD
:101D30009144B9F1C80FA8BF4FF0C80929EAE97961
:101D400080F80390002940F0C5830F2F3FF472AF55
:101D500090F800909144B9F1C80FA8BF4FF0C8099E
:101D600029EAE97980F800909B78002B3FF462AF74
:101D7000122049461CF024FCD4F8D0005AE7D4F8CD
:101D8000D0006F4B90F808909B789144B9F1C80F40
:101D9000A8BF4FF0C80929EAE97980F80890002B1C
:101DA0003FF448AF0B2049461CF00AFCD4F8D000A1
:101DB00040E70B99624B91F804900D939144B9F16F
:101DC000640FA8BF4FF0640929EAE97981F804900B
:101DD0001CF010FC0D9B9B78002B3FF45CAF0320A4
:101DE00049461CF0EDFBD4F8D00023E70B99544B87
:101DF00091F802909144B9F1640FA8BF4FF06409C3
:101E000029EAE97981F802909B78002B3FF443AFEF
:101E1000022049461CF0D4FBD4F8D0000AE70B9905
:101E2000474B91F800909144B9F1FA0FA8BF4FF0D9
:101E3000FA0929EAE97981F800909B78002B3FF4B0
:101E40002AAF012049461CF0BBFBD4F8D000F1E6D4
:101E50000B993B4B91F807909B78914489F30809C3
:101E600081F80790002B3FF416AF052049461CF07F
:101E7000A7FBD4F8D000DDE60B98314B90F8069024
:101E800099789144B9F1640FA8BF4FF0640929EA29
:101E9000E97980F80690002940F0DA820D2F3FF4AE
:101EA000FAAE0B989B7890F805909144B9F1640FC5
:101EB000A8BF4FF0640929EAE97980F80590002B62
:101EC0003FF4E9AE0E2049461CF07AFBD4F8D0006E
:101ED000B0E6D4F8D0001A4B3AE7D4F8D000184B4B
:101EE00090F806909B789144B9F1C80FA8BF4FF0C5
:101EF000C80929EAE97980F80690002B3FF49AAEE8
:101F0000092049461CF05CFBD4F8D00092E6D4F8D6
:101F1000D0000B4B90F8059099789144B9F1C80F17
:101F2000A8BF4FF0C80929EAE97980F8059000298F
:101F300040F0DB82112F7FF4B4AE7BE68C7700207B
:101F4000888C0020D4F8D000C44B90F807909B7880
:101F50009144B9F1C80FA8BF4FF0C80929EAE9793F
:101F600080F80790002B3FF465AE0A2049461CF02C
:101F700027FBD4F8D0005DE6D4F8D000B74BBBE621
:101F8000B64B8EE7129AFFF77CBB049993F8029048
:101F900031F91220B2F5617F4FF4966191FBF9F1AE
:101FA000C0F2898040F633099145A8BF91460C2FB5
:101FB000A9F5617999FBF1F95FFA89F900F00D81D2
:101FC000182F40F083804A46C82AA8BFC822A44CD4
:101FD000D4F8D01091F817E0D0B270453FF427AA9A
:101FE000B2EB0E029D4BC87548BF0732D2109978EC
:101FF000531CDBB239B913B118462AF075F9DAF877
:102000000430FFF714BA494618200D931CF0D8FA93
:102010000D9BF0E7934B94491A684FF47A73B3FB26
:10202000F2F3C3EB431203EB8202069B1B68D20060
:102030001F06A1F8A8207EF56FA88C4A1278960793
:102040007EF56AA88A4A127D042A7EF665A81EF0EB
:1020500019FE2AE418F0100F40F05B810B201CF0F1
:1020600065FA002840F02681824F18F0200F40F0DA
:102070005B817B4C94F8D430002B3FF40AADB9F16E
:10208000000F7FF49AAAFEF716B97B49069B0A60F7
:102090007A4A1B687A4E0992FEF741B8DFED797AE9
:1020A000B4EEE77AF1EE10FA44BFDFED777A37EE5F
:1020B000C77AFFF759B90C2F00F0CC80182F03D145
:1020C0004FF000094A4682E74FF00009644CFFF7E1
:1020D000AEB96E4A0592FEF716BF6D4B0122022083
:1020E00011E56C4A069B1E68136823F00403136015
:1020F000089A012306F4805682F82130FEF7D5BFF6
:1021000038EE678A644B65491870FDEEC87AC8F5E9
:10211000FA63CDED047ABDF91020120381FB0201B0
:10212000D217C2EBA1121BB203FB02F343F30F332E
:10213000434407EE903AF8EEE77AC7ED037AFEF7EC
:1021400005BA06F48056FEF7B0BFD4F8D0001BF0F5
:1021500013FB4FF0FF39FFF776B90023BB2A149326
:1021600000F03B81B72A00F03481BE2A00F02F81B5
:10217000BD2A7FF423AD4FF6FE71494A3F48D58909
:10218000099090892B4401449181D38111F0DCFDA9
:1021900008F07EFF11F0C0FDF7F78AFD01202AF05C
:1021A000A3F8B4F89020069BFA3A00211B68A4F823
:1021B000902084F89210FDF7B2BF2C49069B0A7854
:1021C0001B682F4E42F004020A702C4A0992FDF758
:1021D000A6BF344B0222032095E44C46324A527883
:1021E000A2423FF473AF1D4B0D93204623F058FFDE
:1021F0000D9B9B781BB149460C201CF0E1F9631C38
:10220000DBB2174CF7E611F09FFD08F041FF11F02B
:1022100083FDF7F74DFD01202AF066F894F88E2033
:10222000FFF7F8B9102006F037FD202006F01CFD5E
:102230001E49104F081F18F061FB1D4B02221A7037
:10224000074C94F8D430002B00F01981B6F80080C8
:10225000FFF7B3B90024A146C0E700BF888C002077
:10226000A024002038B100205CA90020867700203F
:10227000B85A00202C4C0020BC8E00208C77002007
:1022800084770020DB0FC9BFDB0F49C00495002015
:1022900060540020807700204C270020D34D62102E
:1022A000084B0020AE540020E0A60020E879002072
:1022B0000E7A0020924B934F5B8997ED007A07EEE0
:1022C000903AF8EEE77AB0EEC77AB4EEE77AF1EE3C
:1022D00010FA7FF5CAAE97ED017AB0EEC77AF4EE48
:1022E000C77AF1EE10FA7FF7C0AE18F0200F7FF436
:1022F000C0AE202006F0D0FC94E80C0082490A60B1
:10230000084641F8043F18F0F9FA804B01221A7090
:1023100096E7102006F0A8FC7C4BB6F8008083F806
:1023200000904FF0010999E6202006F09DFC774BC4
:1023300000221A7084E706231A46FEF7FFBA052327
:102340001A46FEF7FBBA04231A46FEF7F7BA032330
:102350001A46FEF7F3BA02231A46FEF7EFBA012334
:102360001A46FEF7EBBA6A4A069B6A4E1B684FF4A0
:10237000C8711180684A0992FDF7D1BE08231A4638
:10238000FEF7DCBA07231A46FEF7D8BAF0EE487A11
:10239000FEF7C8BF002D3DF4D4AD604C94F88D30ED
:1023A000002B3DF4FFAD29F05DFE002384F88D3055
:1023B000FDF7F8BD584B84F8941084F89500554EFD
:1023C0000993FEF77ABDB0EE677AFEF7C1BF02212E
:1023D000D3E619464FF6FE73CFE619460223CCE644
:1023E0000021012023F07AFDB4F89020069B4A4991
:1023F0001B680991963AA4F89020002284F8922054
:10240000FDF78DBE00210846ECE7FF21002015F006
:1024100064FA94F88E20FFF7DDBB0121002015F04F
:102420005CFA94F88E20FFF7D2BB0021FF2015F054
:1024300054FA94F88E20FFF7C7BB0021012015F055
:102440004CFA94F88E20FFF7BCBB0B20FDF728BE9A
:1024500049460D200E930D921CF0B2F80E9B0D9A7A
:102460001CE52E4C22F0FAFC002384F88D30FDF799
:1024700099BD00210320B5E700210220B2E74FF00B
:102480000109FFF706BB002B87D02549254A0968BB
:102490004FF47A7000FB031313607EE700210420E1
:1024A000A0E7152049461CF08BF8D4F8D000FFF7C0
:1024B000C1BB494617201CF083F8FFF7ECBB102086
:1024C00049460E930D921CF07BF8D4F8D0000E9B79
:1024D0000D9A0FE40F2049460E930D921CF070F8F0
:1024E000D4F8D0000E9B0D9A2FE4112049460E938C
:1024F0000D921CF065F8D4F8D0000E9B0D9A19E5EA
:102500009C7A00202C4C0020742400200E7A00209D
:1025100006B40020847700208C770020A0240020BF
:10252000E8B30020B88E00202DE9F047C74C63685F
:1025300020469847002800F0C380C54B1B78012235
:10254000042B84F83C2000F0BD80B4F91610B4F9D7
:102550001820B4F91A3021636263A363BD4B1B8852
:10256000002B69D0BC4DD4ED0C7AD5ED004A95ED29
:10257000050A95ED015A95ED067AD5ED035A95EDCC
:10258000026AF8EEE76AD5ED047AA4EEA60AA5EE93
:10259000267A67EEC07AA5EEC07AE6EE267A85ED59
:1025A000057AC5ED067A2CF037FBD4ED0D6AD5ED32
:1025B000094A95ED0E0A95ED0A5A95ED0F7AD5ED7B
:1025C0000D7AD5ED0C5A95ED0B6A2063F8EEE66AAC
:1025D000A4EEA60AA5EE267A67EEC07AA5EEC07A2A
:1025E000E6EE267A85ED0E7AC5ED0F7A2CF014FB17
:1025F000D4ED0E6AD5ED124A95ED170A95ED135AF2
:1026000095ED187AD5ED167AD5ED155A95ED146A33
:102610006063F8EEE66AA6EEA40AA6EE857A67EE97
:10262000C07AA0EE657AE6EE867A85ED177AC5ED7A
:10263000187A2CF0F1FAA063884FA17F884816F031
:1026400027FE3B88002B40F08480864ED6F8E4506D
:10265000854B1B685B0743D4B5F90070216B636B36
:10266000A06B824A824E92ED026AD2ED006AD2EDF0
:10267000015AC91B2163B5F90270DB1B6363B5F90D
:1026800004703568C01B07EE900AB8EEE75A07EEF3
:10269000901AB8EEE77A07EE903AF8EEE77A36EE5F
:1026A000056A36EE877A77EEA57A0135A06382ED6A
:1026B000026A82ED007AC2ED017A3560BDE8F087EA
:1026C000BDE8F0876B4BB4F91600B4F91810B4F9F3
:1026D0001A2018802063598061639A80A2633DE7C5
:1026E000B6F89820322A00F08880002A66D196F841
:1026F0009530002BB0D06048D6F800215F4980FBB0
:102700000273D217C2EB23122A80D6F8042180FB71
:102710000273D217C2EB23126A80D6F80831A78A57
:1027200080FB0302DB17C3EB2213DB1BAB80002310
:10273000CB6086F8953011F007FB08F0A9FC11F08A
:10274000EBFAF7F7B5FA012029F0CEFDD6F8E45000
:1027500082E7444E226BD6F8E450B3F5C87F4FF0C1
:10276000000323632B80398818BFD6F8E800B7F838
:10277000008008BF0020B1F5C87F18BFD6F8EC3044
:10278000616B02440B440020B8F5C87F6063C6F853
:10279000E820C6F8EC30688052D0D4F838E0D6F89B
:1027A000F010A0637144B8F1010FA880C6F8F010D2
:1027B00068D008F1FF38A7F8008049E7D6F8000193
:1027C000236B00210344C6F8003121632980D6F829
:1027D0000401636B61630344C6F804316980A36B31
:1027E000D6F80801A1630344012AC6F80831A9807C
:1027F00075D0013AA6F8982079E72B8820491F4820
:10280000276BA6F8F4300023B5F802E0B5F804C051
:10281000C0684B608B602363C6F800712B80616BCE
:10282000C6F8041163636B80A16BC6F80811A3633B
:10283000A6F8F6E0A6F8F8C0C6F8FC00AB80D8E72A
:10284000A36BC6F8F030A063A880B2E73C77002005
:10285000F98E0020185100201C51002006B40020E1
:102860006C770020A024002048B10020E86E0020F2
:10287000E46E0020FC8E00201F85EB51084B0020E9
:10288000A0250020DFF88CC0DFF884E0C8328CFB84
:1028900002A9C833D217C2EBE9128CFB03A9DB17DC
:1028A000C3EBE913C8316B802A808CFB013CA28A00
:1028B000CB17C3EBEC139B1AAB80CEF80C0011F0D6
:1028C00043FA08F0E5FB11F027FAF7F7F1F9404673
:1028D00029F00AFDB7F80080D6F8E45069E70B202C
:1028E00086F89A1086F8942029F0D8FBD6F8E450A0
:1028F000074BB6F8F420B6F8F670B6F8F800D6F83C
:10290000FC102A806F80A880B6F89820D96070E704
:10291000084B00201F85EB512DE9F04F2DED0C8B5E
:10292000DFF8F4B093B0DBF80420049058469047E9
:10293000002800F08C82BBF8A87000218BF85110A1
:10294000002F6DD1BBF93A00DBF82450DBF82810DA
:10295000BBF93860DBF82040BBF93C20DFF8BC90C5
:10296000401B521ACBF830009BF85210CBF83420A1
:10297000341B0BF12C00CBF82C4016F089FCD9F855
:102980000020910041F1CD87DBED0C5A1F4CDBEDAF
:102990000B7A1F4994ED406AD4ED416A94ED427A76
:1029A000D4F80C2109681B4B0293B8EEE58ADBEDE5
:1029B0000D5AF8EEE77AF8EEE58A013277EE867A7C
:1029C00038EE268A78EE878A8A42C4ED407A84ED12
:1029D000418AC4ED428AC4F80C2101F0668393F861
:1029E00000E0BEF1140F02F0A3870023D4F81451C5
:1029F0000393062D01F2B584DFE815F0D816C5164D
:102A000031155D16200C0C16931500BFAC25002067
:102A1000E04D0020F98E00205CA9002048B1002084
:102A2000D84BD9481A6805934FF47A76B6FBF2F280
:102A3000C2EB421602EB8602D600D44BDFF8A48329
:102A400044780293B6B2B7421D78B8F9060003F095
:102A50008A80DBF87C30BBF93810DBF8602003F1AA
:102A6000010E07EE901A0A44BEF1010FCBF87CE08C
:102A7000CBF86020F8EEE77A03F08280DBED1B5A9A
:102A8000DBED1D6A07EE10EA37EEE56AB8EEC75ACD
:102A9000012F86EE057A37EE257A77EEC77A8BED31
:102AA0001C7AE7EE866A8BED1B7AF0EE667ACBED48
:102AB0001E6ACBED1D6A03F08784DBF89030BBF90A
:102AC0003A10DBF8642003F1010E07EE901A0A4475
:102AD000BEF1010FCBF890E0CBF86420F8EEE77A76
:102AE00003F06980DBED205ADBED226A07EE10EA85
:102AF00037EEE56AB8EEC75A012F86EE057A37EE53
:102B0000257A77EEC77A8BED217AE7EE866A8BED30
:102B1000207AF0EE667ACBED236ACBED226A03F0E1
:102B20002B84DBF8A430BBF93C10DBF8682003F100
:102B3000010E07EE901A0A44BEF1010FCBF8A4E093
:102B4000CBF86820F8EEE77A03F05080DBED255AE9
:102B5000DBED276A07EE10EA37EEE56AB8EEC75AF2
:102B6000012F86EE057A37EE257A77EEC77A8BED60
:102B7000267AE6EE276A8BED257AF0EE667ACBEDC3
:102B8000286ACBED276A03F0EA83814CA8F8060097
:102B9000BBF8A820029B013A1D78ABF8A820059944
:102BA0000022072D4A608A60CA6040F05781F7F71B
:102BB000CFFF029BDFF82C821D78049BC01A94F88B
:102BC0002131A8F800000693002B40F04D816E4A99
:102BD0005279002A01F096816E4A1278013AD2B2F7
:102BE000072D84F8212102F00282002308936A4B0A
:102BF000D4F82C21D3F800A0624B0593049B9FEDE1
:102C0000676AD4ED4A9A6649DFF8DC81D1ED006A43
:102C1000C4F82C319A1A07EE902AF8EE677AB7EECC
:102C2000007AC6EE278A08F11C0300250793DFF817
:102C3000BC915C4B5C4F03932E4677EE69BA94EDE2
:102C400049CA9FED5A9ADFED5AAA9FED5ABA9FEDF5
:102C50005AAA6BEEA6BAF4EEC7BAF1EE10FA88BF24
:102C6000F0EE47BA554B98ED008A2B44D3ED007A2D
:102C7000F5EE407AF1EE10FA17D0514B2B4493ED5C
:102C8000007A78EE476AB0EEE66AF4EEC67AF1EEC4
:102C900010FA08D5F5EEC06AF1EE10FACCBF37EEA7
:102CA000878A37EE678A83ED008A464B1A88930736
:102CB0003FD0022E3DD0444B9AF82E1033F91630F7
:102CC00007EE103A079B07EE901A2B44F8EEE76ADE
:102CD000B8EEC77AD3ED007A4B42A6EEA77A700021
:102CE00007EE903AF8EEE77AB4EEE77AF1EE10FAF2
:102CF0000AD407EE901AF8EE677AF4EEC77AF1EE8E
:102D000010FA88BFF0EE477A304B31490344085E31
:102D1000B3F90C30C31A07EE103AB8EEC77AD007F1
:102D2000E7EE497A41F184802A4B93ED008A27EE41
:102D3000888A059B94F864212B4493ED01DA78EEA0
:102D40004DCA002A00F0F180234BD4F86821049981
:102D50001B688A1A9A4240F3E8809AF84830022B9E
:102D600002F09481022E04F0D8841C4B1B68990752
:102D700000F192801A4B87ED00BA1B689342C0F2B3
:102D8000C48035E038B1002048A90020F98E002029
:102D9000AC250020FC4A00208877002000247449DC
:102DA000C0730020744D0020804D0020CDCCCC3D60
:102DB000AE47813F000000000000C842B47300200D
:102DC000E826002084770020F4260020084B00200D
:102DD000347700209C730020C873002030770020D7
:102DE000C4730020FC8E0020DC2600208C4D0020C7
:102DF000F7EE007AF4EEE79AF1EE10FA40F19580E2
:102E000005991F4BD1ED017A93ED007AF0EEE77A48
:102E1000F4EEC77AF1EE10FA40F18780D1ED027A34
:102E2000F0EEE77AB4EEE77AF1EE10FA7DDDD1ED5F
:102E3000037AF0EEE77AB4EEE77AF1EE10FA74DD99
:102E4000104B1B689B0760D50F49104B44E0104B9B
:102E5000104C1D780293072D3FF4A9AE94F8213150
:102E60000693002B3FF4B3AE5F1E84F82171012D51
:102E700001F0C98213B0BDEC0C8BBDE8F08F00BF30
:102E8000D07300203077002034770020084B0020DA
:102E9000F98E0020AC250020D24BD349DFF8C4E3E3
:102EA00031F916C09EED008ADFF8BCE387ED00BA69
:102EB00003EB460028EE098AB0F90C00A0EB0C00E9
:102EC00007EE900AF8EEE77ADEF8000027EE888A2F
:102ED000904278EE4DCA8BDAB3F90C20B1F900E0DC
:102EE000C248AEEB020E00688EEAEE72A2EBEE7202
:102EF00082421ADAB3F90E30B1F90220D21A82EA0C
:102F0000E273A3EBE27398420FDDB94B1A880023FA
:102F100084F86431002A43F0EF85B64AB64B117845
:102F2000186881F0010107F01BFEB44B2B4493EDB0
:102F3000000A039B2CEE000A022E20EE2C0AA3ECC2
:102F4000010A039304F02084AD4BD7ED006A93EDA2
:102F5000007AAC4BD3ED007AAB4B93ED006AAB4BF0
:102F600067EE277A2B4427EEAB7AD3ED007A67EE33
:102F7000277AF0EE665AECEEA75AB1EE467AB4EE36
:102F8000E57AF1EE10FA08DCB4EEE56AF1EE10FA3B
:102F90008CBFB0EE657AB0EE467A94ED4A6AF7EEF1
:102FA000007AB4EEE76AF1EE10FAACBF0123002319
:102FB00043B1F0EEE66AF0EEC77AF4EEE67AF1EEAF
:102FC00010FA01D587ED007A022E04F04183904A71
:102FD000904B52F826001B68B0EE4D0A98478E4A77
:102FE0008E4B52F826001B6898479AF8373023B169
:102FF0008B4B1B88002B00F08887B0EE4B8A894BE7
:1030000038EE400A2B4493ED008A83ED000A9AF8CB
:10301000483030EE480A20EE288A002B33D0824B0D
:103020001B7813F0010300F0C886F7EE007AF4EE87
:10303000E79AF1EE10FA94F86431C1F21F85002B83
:1030400001F00880D4F86831049AD31A774A1268DC
:103050009A4218DD764BD3ED007AF0EEECCAF4EE2E
:10306000E7CAF1EE10FA42F12280614B1A88002380
:1030700084F86431002A00F0AC866E494A6912B1C6
:103080000A6813604B746C4B94F874212B4493EDD5
:10309000000A2CEE000A20EE088A89ED008A32B977
:1030A000039B87ED00BA03ED01BA89ED00BA013642
:1030B000032E08F1040809F1040907F1040705F1DA
:1030C00004057FF4CFAD029B1A78072A01F0DB8458
:1030D000012A01F079870023039394F87C21002AC8
:1030E00041F0C481DFF88491544BD9F8002019686D
:1030F000D60491F82C0000F12387DFF874A1504A20
:10310000BAF81A30D2ED005A4E4A4F4DD2ED004A6D
:10311000D5ED036A4D4AC4ED635A07EE103A4C4BA5
:1031200092ED005AD3ED007AD3ED013A93ED026AA5
:10313000C4ED615AB8EEC77A34EEE54A012236EEA4
:10314000C77A84ED604AC4ED644A84F89421C7EEDE
:10315000055A0A8D534206EE903A3E4BDFED3E4A49
:1031600093ED005A3D4B93ED004AB7EE007AF4EE32
:10317000C75A35EE045AF1EE10FA88BFF0EE475AFE
:1031800035EE275AF8EEE66AF4EEE45AF1EE10FA5C
:1031900007EE902AB4EEE65AB8BFF0EE645AF1EEAC
:1031A00010FAC4ED675AB8EE677A01F14B83B4EEBA
:1031B000C75AF1EE10FA88BFB0EE475A254BDFED43
:1031C000284AD3ED017A254B93ED014A77EE847AB4
:1031D00025EE245A77EEA37AF4EEE76AF1EE10FAC0
:1031E00051DC47E0084B002034770020CC730020EE
:1031F000C0B30020C2B30020C4B30020707300200D
:10320000146F00207C000020E47300207C730020F9
:103210001C6F0020186F0020706F00206C6F002062
:103220008477002018270020F04B0020C87300206E
:10323000D4730020C8B30020887300208877002052
:103240007C490020F44A00202C4C00207C74002093
:10325000804D0020744D0020000000008C4D0020A7
:103260006F12833A9C730020C473002048B1002081
:1032700004950020B4EEE77AF1EE10FA8CBFF0EE80
:10328000676AF0EE476AED4B4A8DD3ED027A9FED07
:10329000EC7A534204EE103A76EE277AB8EEC44A3E
:1032A00066EE876AF4EEC47AF1EE10FA0AD407EEFD
:1032B000102AB8EE474AB4EEE74AF1EE10FA88BF9A
:1032C000B0EE674ADF4ADFEDDE7A527824EE274A15
:1032D0000AB9B1EE444A002841F01A86B7EE003A26
:1032E000D94E3278002A02F0AE86D8499FEDD86ACE
:1032F000D1ED024A91ED017AD1ED037A66EEA44A4E
:10330000E5EE074AE4EE274A63EE244AF4EEC64AA5
:10331000F1EE10FAB4BFF0EE463AF0EE643A98BF20
:10332000B0EE646A012ACDED0A4A02F0D986D1EDE9
:10333000067AD1ED052A91ED077A66EEA77AE5EED9
:10334000227AE4EE077A23EE277AB4EEC67AF1EE1B
:1033500010FAB4EEE37A8CBFF0EE467AF0EE477ADC
:10336000F1EE10FA98BFB0EE676AB4BFF0EE637A80
:10337000F0EE477A022A8DED0B7A00F0DE8091EDB7
:103380000A7AD1ED092AD1ED0B3A26EE877AA5EE1D
:10339000227AA4EE237A23EE077AB4EEC67AF1EE0F
:1033A00010FAB4EEE77A8CBFF0EE463AF0EE473A08
:1033B000F1EE10FA98BFB0EE636AA8BFF0EE477A5C
:1033C000032A8DED0C7A00F0B88091ED0E7AD1EDE4
:1033D0000D2AD1ED0F3A26EE877AA5EE227AA4EED9
:1033E000237A23EE077AB4EEC67AF1EE10FAB4EE41
:1033F000E77A8CBFF0EE463AF0EE473AF1EE10FA7B
:1034000098BFB0EE636AA8BFF0EE477A042A8DED4C
:103410000D7A00F09280D1ED123AD1ED112A91EDA2
:10342000137A66EEA33AE5EE223AE4EE073A63EE4B
:10343000233AF4EEC63AF1EE10FAF4EEE73A8CBF16
:10344000B0EE467AB0EE637AF1EE10FA98BFB0EEC5
:10345000476AA8BFF0EE637A052ACDED0E3A6CD02C
:10346000D1ED163AD1ED152A91ED177A66EEA33A11
:10347000E5EE223AE4EE073A63EE233AF4EEC63A7A
:10348000F1EE10FAF4EEE73A8CBFB0EE467AB0EE09
:10349000637AF1EE10FA98BFB0EE476AA8BFF0EE7B
:1034A000637A062ACDED0F3A47D0D1ED1A3AD1ED25
:1034B000192A91ED1B7A66EEA33AE5EE223AE4EE84
:1034C000073A63EE233AF4EEC63AF1EE10FAF4EE60
:1034D000E73A8CBFB0EE467AB0EE637AF1EE10FABE
:1034E00098BFB0EE476AA8BFF0EE637A072ACDED29
:1034F000103A22D091ED1E7AD1ED1D2AD1ED1F3A5E
:1035000026EE877AA5EE227AA3EE847A27EE037A56
:10351000B4EEC67AF1EE10FAB4EEE77A8CBFF0EEB4
:10352000466AF0EE476AF1EE10FA8DED117A98BF17
:10353000B0EE666AA8BFF0EE477A77EEC67AF7EE8D
:10354000006AF4EEE67AF1EE10FAC4ED4A7A43F33B
:103550000C8686EEA77A022ADDED0B7A67EE244A06
:1035600067EE877ACDED0A4ACDED0B7A2DD0DDEDF1
:103570000C7A67EE877A032ACDED0C7A25D0DDED43
:103580000D7A67EE877A042ACDED0D7A1DD0DDED38
:103590000E7A67EE877A052ACDED0E7A15D0DDED2D
:1035A0000F7A67EE877A062ACDED0F7A0DD0DDED22
:1035B000107A67EE877A072ACDED107A05D0DDED17
:1035C000117A27EE877A8DED117A2249096811F078
:1035D000805801F00882F6EE005AC4ED675A002ABE
:1035E00002F02B851C4B94ED646A1C491C4F1D781E
:1035F000DFF874E094F9943194ED635AB7F90670EA
:10360000C878D9F80010DEED004A0597BDEEC66A0D
:1036100007EE103ABAF81A70124B079716EE10EA36
:10362000BDEEC56A05F0010C01F4805701F01005EC
:1036300001F4800108911B7818E000BF744D002050
:103640006F12833ACC4D0020EC6D0020EC7300200B
:1036500000000000D44A0020F04B00208C790020AC
:103660004A8C002034570020E8730020D4ED606AB3
:10367000D4ED617AB8EEC77A16EE101A002840F041
:103680004987002D41F01383D34D9DED0A5A95EDE6
:10369000006AD24825EE866AA5EE076AB0EE675A40
:1036A000A6EE265ABDEEC56A16EE108A16EE107A00
:1036B000F045A8BF77464145C8BF0F4606EE107AD1
:1036C000B8EEC66A012A80ED006A00F0DC8095ED54
:1036D000046A9DED0B5A25EE866AA5EE076AB0EEE8
:1036E000675AA6EE265ABDEEC56A16EE108A16EE89
:1036F000107AF045A8BF77464145C8BF0F4606EE91
:10370000107AB8EEC66A022A80ED016A00F0BB802A
:1037100095ED086A9DED0C5A25EE866AA5EE076ABE
:10372000B0EE675AA6EE265ABDEEC56A16EE108AAE
:1037300016EE107AF045A8BF77464145C8BF0F4640
:1037400006EE107AB8EEC66A032A80ED026A00F02F
:103750009A8095ED0C6A9DED0D5A25EE866AA5EED0
:10376000076AB0EE675AA6EE265ABDEEC56A16EE97
:10377000108A16EE107AF045A8BF77464145C8BFBB
:103780000F4606EE107AB8EEC66A042A80ED036A88
:1037900079D095ED106A9DED0E5A25EE866AA5EE5C
:1037A000076AB0EE675AA6EE265ABDEEC56A16EE57
:1037B000108A16EE107AF045A8BF77464145C8BF7B
:1037C0000F4606EE107AB8EEC66A052A80ED046A46
:1037D00059D095ED146A9DED0F5A25EE866AA5EE37
:1037E000076AB0EE675AA6EE265ABDEEC56A16EE17
:1037F000108A16EE107AF045A8BF77464145C8BF3B
:103800000F4606EE107AB8EEC66A062A80ED056A03
:1038100039D095ED186A9DED105A25EE866AA5EE11
:10382000076AB0EE675AA6EE265ABDEEC56A16EED6
:10383000108A16EE107AF045A8BF77464145C8BFFA
:103840000F4606EE107AB8EEC66A072A80ED066AC1
:1038500019D095ED1C6A9DED115A65EE865AE7EE7A
:10386000055AE6EEA57AFDEEE77A17EE905AAE45D8
:10387000A8BFAE46A942D8BF714607EE901AF8EE2F
:10388000E77AC0ED077ABCF1000F00F05087544A88
:103890001268002A40F05887524A127892B1307864
:1038A00068B14E4FDFF85C810025E8B2D8F80030EF
:1038B000B7EC010A9847307801358542F5DB4A4A72
:1038C00012689047029B1A78072A01F0F2804FF0A5
:1038D0000008D9F80020530501F12780434B1B78DD
:1038E000BBB1434ABAF81A30B2F906209A4210DC4A
:1038F000404B1B78012B01F08F83192B01F08C8337
:103900000E2B06D0082B04D03B4D0023AB60C4F82F
:10391000383194F8A65125B1384B1B889E0741F0E9
:103920003D8394F8AC31002B40F0A0879AF81E60DC
:10393000002E00F04784022E01F01F83032E41F079
:1039400018839AF82020C2EB421102EB8102D200C8
:1039500092B29AF81F700237FFB2002B00F09C85DC
:10396000002A00F0998526490E68B2FBF6F216B2DD
:10397000A4F8DC61002F03F0CF8007EE906AF8EE28
:10398000E77AF7EE006A86EEA77A1B4D012FD4ED99
:103990007C6AD5ED007A77EEE67A67EE877AC4ED39
:1039A000787A3BD0D5ED017AD4ED7D6A77EEE67A70
:1039B000022F67EE877AC4ED797A2FD0D5ED027A9F
:1039C000D4ED7E6A77EEE67A032F67EE877AC4ED50
:1039D0007A7A23D018E000BFEC730020A84D0020B5
:1039E000106F00205C5A002030570020291B002057
:1039F0004A8C0020CC4D00202C4C002084770020E5
:103A0000C84D002028570020D5ED037AD4ED7F6AF9
:103A100077EEE67A67EE877AC4ED7B7A029A1278BF
:103A2000092A03F0C881002E40F3D2839FB394ED9E
:103A30007C7AD4ED787A77EE877A012FC4ED7C7AA0
:103A4000C5ED007A21D094ED7D7AD4ED797A77EEC8
:103A5000877A022FC4ED7D7AC5ED017A15D094EDF9
:103A60007E7AD4ED7A7A77EE877A032FC4ED7E7A68
:103A7000C5ED027A09D0D4ED7F7A94ED7B7A77EEAA
:103A8000877AC4ED7F7AC5ED037A013F022FB8BF74
:103A90000227FAB20692002B069F18BF0227D24BCC
:103AA000DFEDD26A1A68029B91781878137807EED6
:103AB000903AF8EEE77AB0EE007A67EEA67AF4EE86
:103AC000C77AF1EE10FA40F3A886DFEDC96A37EE47
:103AD000C77AB0EE676AA7EE266AF0EE466A95ED01
:103AE000007A9FEDC46A27EE066AF0EEC65A84EDAE
:103AF000536AC4ED565A99B107EE101AB8EEC75A78
:103B00009FEDBA7A66EE064A25EE075AB7EE007ABE
:103B100037EE457A64EEA54AA4EE857A26EE076A6A
:103B20009FEDB57A537926EE877A27EE067ACBB1E8
:103B3000DFEDAE6A9FEDB16A65EEA65A06EE903AE9
:103B4000F8EEE66A65EEA65AF4EEC65AF1EE10FA01
:103B500001F3B581B7EE006A76EE655AC6EE256AC6
:103B600027EE267A0C289FEDA68ADFEDA66A00F0E4
:103B70006087B4EEC87AF1EE10FA98BFB0EE478ACB
:103B8000B4EEE68AF1EE10FAB8BFB0EE668A84EDC4
:103B90004C8A002F00F0DC80B0EE007AF4EEC77A99
:103BA000F1EE10FA05DD37EEC77ADFED916AE7EE48
:103BB000267A95ED017ADFED8F6A27EE267AF0EE10
:103BC000C75A84ED547AC4ED575A99B106EE901A4B
:103BD0009FED866AF8EEE66A27EE075A66EE866A79
:103BE000B7EE006A36EE666A25EE255AA5EE266A1D
:103BF00027EE067ADFED806A937967EEA67A67EEA4
:103C0000877AABB107EE103AB8EEC77A9FED776AC4
:103C1000DFED7A6A27EE257A27EE067AB4EEE67AA9
:103C2000F1EE10FA41F34F81DFED776A67EEA67A85
:103C30000C2800F0DF86DFED726A9FED727AF4EEF9
:103C4000E67AF1EE10FA88BFF0EE667AF4EEC77A03
:103C5000F1EE10FAB8BFF0EE477A012FC4ED4D7ABD
:103C600076DD5378DFED616A07EE903AF8EEE77A99
:103C7000B0EE007A67EEA67A537AF4EEC77AF1EEE8
:103C800010FA05DD37EEC77ADFED596AE7EE267ADE
:103C900095ED027ADFED576A27EE267AF0EEC75AE5
:103CA00084ED557AC4ED585A9BB106EE903A9FEDDB
:103CB0004F6AF8EEE66A27EE075A66EE866AB7EEB6
:103CC000006A36EE666A25EE255AA6EE856A27EE6C
:103CD000067ADFED496AD37967EEA67A67EE877ACE
:103CE000FBB107EE103AB8EEC77A9FED406ADFED00
:103CF000436A27EE257A27EE067AB4EEE67AF1EEED
:103D000010FA01F3EE80B5EEC07AF1EE10FA02F18E
:103D10008883B7EE006A36EE477AC6EE076A67EE2A
:103D2000A67A0C2800F0A286DFED356A9FED357A81
:103D3000F4EEE67AF1EE10FA88BFF0EE667AF4EE71
:103D4000C77AF1EE10FAB8BFF0EE477AC4ED4E7ABA
:103D5000092800F03B869AF82150002D40F0F085AC
:103D6000002384F8AC31294B1B68980609D5284BF1
:103D70001B8803F0300323B1264B1B78D90702F1CF
:103D8000E7801EF057FE002840F04A83224B1B7844
:103D900023B9224B9B78002B41F0FB80029B1D78BE
:103DA000072D7FF464A8F6F7D3FE1D4B029AA0EB13
:103DB00008001578D880FFF75AB894F86421002AD3
:103DC0003FF461A9174A84F864311288002A7FF40D
:103DD00054A9154A154B1178186881F0010106F0B5
:103DE000BFFEFFF750B900BF8C7700200AD7233CF5
:103DF000D7A368416F12033B00004843A4707D3F86
:103E000000C0F94400C0F9C40000C8423077002067
:103E100084770020867700208C440020888C002046
:103E2000FC8E0020C0B30020C2B30020C4B3002029
:103E300094ED567AB1F90000D4ED576AB1F902E079
:103E4000E44AF4EEC76A80EAE0738EEAEE71A3EB0F
:103E5000E073F1EE10FAA1EBEE71B4BFB0EE476A79
:103E6000B0EE666A8B42B8BF0B4607EE103A137885
:103E7000B8EEC77A27EE097A002B40F0BC80D64B0B
:103E8000D3ED005AF4EEEA5AF1EE10FA41F17C80DB
:103E9000B7EE005A75EE654ADFEDD06A9FEDD05A55
:103EA000D04B36EEC77A24EE855AD3ED006AE7EEA2
:103EB000055A65EEA65AF5EEC05AF1EE10FA40F238
:103EC0008E85CAEE256AB7EE007AF0EE475AE6EE26
:103ED000665AF0EE656AF4EEC76AF1EE10FA88BF32
:103EE000F0EE476AF5EEC06AF1EE10FAB8BFF0EEF8
:103EF0004B6ABD4B93ED007A67EE877AA7EEA68AF0
:103F0000FEF717BF0122FEF76BBEB84BB84A2B4431
:103F100093ED007AD2ED007AB64B67EE277AF7EE92
:103F2000006AF4EEE67AF1EE10FA93ED007A88BFBB
:103F3000F0EE667A67EE877A27EE888AFFF75FB839
:103F4000AD4BDFF8F0A21A78D5075CBFBAF818209D
:103F5000A4F88821A94AAA4D1288D5ED037A07EE64
:103F6000102AB8EEC77AF4EEC77AF1EE10FA41F2F1
:103F7000AC87A44D2B8807EE103AB8EEC77AF4EE62
:103F8000C77AF1EE10FAC1F253809F4A9F4D92ED2D
:103F9000006AD5ED006A94F99421C4ED636A76EE67
:103FA000665A012AC4ED616AC4ED605A84ED646A00
:103FB00001F0D385049BC4F89831002537EEC77A09
:103FC000FCEEE77A924E84ED677A17EE902AA4F819
:103FD0008821012296ED005A84F894218D4A954259
:103FE00041F2A3878C4BD3ED007AD3ED013A93EDE8
:103FF000026AFFF7ACB87B4B93ED005AB5EEC05A9E
:10400000F1EE10FA40F3EB84844BD3ED006AF5EE49
:10401000C06AF1EE10FA40F3E28436EEC77A66EE3B
:104020004A5A87EE266AC5EE856AB7EE007AB4EE84
:10403000C76AF1EE10FA88BFB0EE476AB5EEC06A03
:10404000F1EE10FA76EE876AB8BFB0EE4B6A66EE14
:10405000266A40E7724AD2ED007AB0EEC87AB4EE32
:10406000E77AF1EE10FA7FF70EA86E4AD2ED007AE9
:10407000B0EEEC7AB4EEE77AF1EE10FA7FF703A82F
:10408000694AD8ED007A92ED007AF0EEE77AF4EE24
:10409000C77AF1EE10FA7EF5F6AF01220499C4F862
:1040A000681184F86421FEF7D1BF07EE102A197851
:1040B000DFF88481C4F80C71B8EEC77AF7EE006AB5
:1040C000132986EE879AB8F90400B4F810619BEDC5
:1040D000070A01F0CE84554A554992ED001AD2EDF7
:1040E000053A92ED122A92ED173AD2ED091AD2ED65
:1040F0000E4A92ED016A92ED064A92ED0A7AD2EDED
:104100000F5AD2ED132AD2ED186A92ED045AD2ED6D
:10411000030A67EE897A69EE288A29EE088AE1EEB9
:10412000273A01EB86070025A2EE283AC4F8005191
:10413000C4F80451E1EE884AA6EE274AE7EE085A91
:1041400092ED167A92ED0D6A92ED021AD2ED0C1AEA
:10415000C7ED003AE2EEA86A25EE635A27EE437AED
:1041600092ED0B2AD2ED152AC7ED204AA0EEE34AC4
:1041700026EE646AD2ED143A82ED054AA1EE275A82
:10418000F0EE477AE1EEE45AA2EE086AE2EEC36A84
:10419000E3EEA87A82ED065AC2ED0E5A82ED0F6A5E
:1041A00087ED403AC2ED176AC2ED187AC4F808519B
:1041B000721C02F01F02A4F81021A8F80400029B50
:1041C000FEF70DBCA4F8DC61002B3FF4CCAD0C4D28
:1041D000022764E4A8730020B07300200000344379
:1041E000610BB63BA4730020A073002004270020BD
:1041F0009873002094730020F04B002080740020FE
:104200002C4C002082740020F44A00206C740020A2
:10421000887400208FD00300804D0020AC730020F4
:10422000D8730020D4730020DC730020705000206D
:10423000044E002004950020FC8E00209C4A11783A
:10424000D4F818719B4B9FED9C7AFE009A1982ED71
:10425000007A002979D09948B0EE476AF0EE476AB3
:104260000022F0EC017A013267EEA77A05EE902A7F
:10427000B4EEE77AF1EE10FAF8EEE55AB8BFB0EE18
:10428000677A914276EEA76AA7EEA56AE9D1F5EEC4
:10429000C06A9A19F1EE10FA82ED007A55DDC6EE89
:1042A000265A874A87490988F7EE007A75EEE75A59
:1042B000D2ED007A65EEA77AFDEEE77A17EE902A46
:1042C000812A42F3BA808A42A8BF0A4607EE902AA2
:1042D000F8EEE77A7C4AF01902EB800292ED057A5B
:1042E000D2ED003A92ED066A92ED014AD2ED046AEF
:1042F000D2ED034A92ED025AA3EEA77AA4EE276A02
:1043000066EEC76AA7EE646ABDEEC77AE5EE276A75
:1043100017EE100A812882ED056AC2ED066A42F3A3
:1043200089808142A8BF014607EE901AF8EEE77A2D
:10433000FCEEE77ACDED057ABDF8142099198A8054
:104340001FB9BEF1130F02F01887BEF1150F41F02F
:10435000D8801E44DFF89081B28828F81720D4F85E
:1043600014515A4A013582FB05325119EA17C2EB42
:10437000A102C2EBC202AD1AC4F814515448D4F8D9
:104380001C11049B534D02682D78C4F81C31591A36
:104390000A440260002D40F0DB8107EE901A4E4E79
:1043A000DFF864914D4FB8EEE78A06F2447506F5E2
:1043B000F668F6EC017A9BED070ADBF86C37F8EE4D
:1043C000E77A284627EE800A9847A5F1E000DBF857
:1043D0008C369847A5F17000DBF8FC369847D6F884
:1043E0005006DBF8AC309847D7ED007AA9EC010A0B
:1043F000E0EE087A2435A845E7EC017AD9D1029B92
:104400001D78FEF728BD364B364A19681288364BA0
:10441000C96919805A8013B0BDEC0C8BBDE8F08FD0
:10442000324C1EF0C3F96378022B00F0E585032BB4
:104430007FF4ACAC41F2B813E35C002B41F00A838B
:1044400041F2A403E35C002B41F00E8341F2E80348
:10445000E35C002B41F0038341F22C13E35C002B5F
:104460003FF494AC224824F023F88FE4214B224EF1
:104470001A7812F0010F327840F04883002A00F0D9
:10448000418592001D491E48DFF88090DFF880A02A
:104490002AF0ECF9FFF7FBB9B4F8DC61013E36B263
:1044A000002EA4F8DC617FF78FAE164DFFF7BEBA81
:1044B000E64D0020DC50002000000000AC2500206C
:1044C000E84D0020E44D0020045000209324499240
:1044D000D46E0020D94D002088A90020D86E00207D
:1044E0006C79002090440020FC8E0020D05A0020DF
:1044F000FC6B0020F04B0020EC6D0020644300209A
:10450000A84D00202C4C00203CB1002048B10020D8
:1045100004950020002D00F0B986BCF1000F42F098
:104520000583CA4D002B42F0998195ED006A9DEDFF
:104530000A5AC74825EE866AFDEEE44AA5EE076AE8
:10454000B0EE675AA6EE265A14EE901ABDEEC56A72
:1045500016EE10CA16EE107AF445A8BF77466145EC
:10456000C8BF0F4606EE107AB8EEC66A012A80ED83
:10457000006A00F0DF8095ED046A9DED0B5A25EE90
:10458000866AA5EE076AB0EE675AA6EE265ABDEE19
:10459000C56A16EE10CA16EE107AF445A8BF774623
:1045A0008C45B8BF0F4606EE107AB8EEC66A022AEE
:1045B00080ED016A00F0BE8095ED086A9DED0C5A11
:1045C00025EE866AA5EE076AB0EE675AA6EE265A71
:1045D000BDEEC56A16EE10CA16EE107AF445A8BFF5
:1045E00077468C45B8BF0F4606EE107AB8EEC66A1D
:1045F000032A80ED026A00F09D8095ED0C6A9DED26
:104600000D5A25EE866AA5EE076AB0EE675AA6EE49
:10461000265ABDEEC56A16EE10CA16EE107AF4459B
:10462000A8BF77468C45B8BF0F4606EE107AB8EEA5
:10463000C66A042A80ED036A7CD095ED106A9DED70
:104640000E5A25EE866AA5EE076AB0EE675AA6EE08
:10465000265ABDEEC56A16EE10CA16EE107AF4455B
:10466000A8BF77468C45B8BF0F4606EE107AB8EE65
:10467000C66A052A80ED046A5CD095ED146A9DED4A
:104680000F5A25EE866AA5EE076AB0EE675AA6EEC7
:10469000265ABDEEC56A16EE10CA16EE107AF4451B
:1046A000A8BF77468C45B8BF0F4606EE107AB8EE25
:1046B000C66A062A80ED056A3CD095ED186A9DED24
:1046C000105A25EE866AA5EE076AB0EE675AA6EE86
:1046D000265ABDEEC56A16EE10CA16EE107AF445DB
:1046E000A8BF77468C45B8BF0F4606EE107AB8EEE5
:1046F000C66A072A80ED066A1CD095ED1C6A9DEDFE
:10470000115A65EE865AE7EE055AE6EEA57AFDEEF9
:10471000E77A17EE905AAE45A8BFAE46A942D8BF79
:10472000714607EE901AF8EEE77AC0ED077A002A94
:104730003FF4ADA89200474945482AF097F8464A09
:104740001268002A3FF4A8A80BF03EFEFFF7A4B8B9
:1047500007EE901A414D424BDFF80881DFF808A1BF
:104760000394F8EEE78A05F2D46600271C46CDF8DC
:104770001880029BDBED077A1B78172B51D095ED43
:10478000007AB8EEC78A082B28EE278A07D1B0EE48
:10479000480A05932AF040FA059BA8F80000D9F8CA
:1047A000002092000BD5002F02F09C87B0EE480A43
:1047B000DBF86C3706F170009847B0EE408AB0EE37
:1047C000480ADBF88C36A6F170009847DBF8FC3617
:1047D00030469847029B1B78032BB0EE408A2CD0C2
:1047E000D5F85406DBF8AC30B0EE480A9847DAED5D
:1047F000007AA4EC010AE0EE287A0137032F06F1D3
:10480000240608F1020805F10405EAEC017AB0D1AA
:10481000029B039C1D78FEF71EBBF0EE676AFFF754
:104820005EB995ED007A0BEB4702B8EEC78A128F9E
:10483000A8F8002028EE278AB1E72AF0EDF9A8F8B9
:104840000000CDE7B0EE665AFEF7B8BCEC7300206E
:10485000A84D002064430020106F002088A900208C
:104860003CB10020FC8E0020D86E002099499A4A65
:10487000D1F8EC10126844F620608142A8BF0146CE
:10488000B1F57A7FB8BF4FF47A7189B212F0100F88
:10489000A4F8AE11D9F8002000F0C583D20441F18C
:1048A000D0858E4A17687E8E76088D4D8D48D4F857
:1048B000B021D5ED037AA0FB01018809642191FBA9
:1048C000F0F11429BDEEE77A04EB4205A8BF1421EC
:1048D00001328A42C4F8B02117EE10EAA4BF0022C8
:1048E000C4F8B02104EB4202A5F8B4E1B2F9B42156
:1048F00007EE102AB8EEC77A77EEC77AFDEEE77AB0
:10490000CDED037ABDF90C1081EAE172A2EBE17200
:10491000B24201F35B8774494FF07E520A60FFF7A1
:1049200005B8724B0293724C28E5DBF80830002B77
:104930003EF4D4AF6F49A1F14C009847FEF7CEBFCB
:104940001E21654807F0A4FB00283FF409AA6A4B22
:104950001B885E063FF504AA94F80032AB4242F091
:104960004982614BD4ED817AD3ED016A94ED4E5AC0
:10497000DFED625A9FED626A27EEC57A68EE277A0C
:10498000A8EE267AE5EE267AB4EEE57AF1EE10FA94
:1049900088BFB0EE657AB4EEC67AF1EE10FAF4EEA6
:1049A000E57AB8BFB0EE467AF1EE10FA88BFF0EEC5
:1049B000657AF4EEC67AF1EE10FAB8BFF0EE467AF8
:1049C00084ED4C7AC4ED4E7AFFF7CAB9FDEEC87A91
:1049D0004C4A17EE903A9680D380FFF7BCB9DFEDD2
:1049E0004A6AFFF786BAD9F8001049023EF5F3ADDE
:1049F000FEF7F5BD9FED417ADFED416A4149F4EEE6
:104A0000C77AF1EE10FA98BFB0EE677AFDEEE77A5A
:104A1000B4EEE67AF1EE10FA17EE903AB8BFB0EEC7
:104A2000667A012F84ED4D7A4B803FF71AA9FFF784
:104A300092B9B4EEC87AF1EE10FA98BFB0EE478A98
:104A4000BDEEC77AB4EEE68ADFF8B8E0F1EE10FA10
:104A500017EE103AB8BFB0EE668A84ED4C8AAEF815
:104A60000030002F7FF498A8FFF775B9BDEEE77A04
:104A7000244B17EE102A9A80FFF756B9002B3EF40C
:104A800002ABFEF7DFBAF6F763F8029BDFF874803B
:104A90001A78089B012AA0EB0300A8F8020000F096
:104AA0009582072A7EF417ABF6F752F80390FEF7CB
:104AB00014BBF6F74DF8029B12491A78039B072A9C
:104AC000A0EB030088807EF402AFF6F741F8804641
:104AD000FEF7FFBE14030020D44A00208877002090
:104AE0002C4C0020D34D62107C000020F98E002059
:104AF000AC250020A8A900208477002000C0F9443C
:104B000000C0F9C4FC8E002000000000002A00F064
:104B1000F981D4ED573A94ED564AD4ED617AF349D0
:104B200094ED607A91ED005AD4ED545A94ED536AA5
:104B3000EF4DF048F4EEC43AF3EE046AF1EE10FAE9
:104B400077EEA64A00F1C28295ED026A26EE656A0A
:104B5000B0EE674AA6EE074AB4EEE44A34EE666A5F
:104B6000F1EE10FA48BFB0EE456A012A80ED006A06
:104B700000F0C88195ED066A26EE656AB0EE674AD8
:104B8000A6EE074AB4EEE44A34EE666AF1EE10FA95
:104B900048BFB0EE456A022A80ED016A00F0B2819A
:104BA00095ED0A6A26EE656AB0EE674AA6EE074AF8
:104BB000B4EEE44A34EE666AF1EE10FA48BFB0EEA5
:104BC000456A032A80ED026A00F09C8195ED0E6A29
:104BD00026EE656AB0EE674AA6EE074AB4EEE44AEE
:104BE00034EE666AF1EE10FA48BFB0EE456A042A68
:104BF00080ED036A00F0868195ED126A26EE656A03
:104C0000B0EE674AA6EE074AB4EEE44A34EE666AAE
:104C1000F1EE10FA48BFB0EE456A052A80ED046A4D
:104C200000F0708195ED166A26EE656AB0EE674A6F
:104C3000A6EE074AB4EEE44A74EE666AF1EE10FAA4
:104C400048BFF0EE456A062AC0ED056A00F05A81B9
:104C5000D5ED1A6A66EEE56AB0EE674AA6EE874AB7
:104C6000B3EE046AB4EEE44A74EE466AF1EE10FA6A
:104C700048BFF0EE456A072AC0ED066A00F042819F
:104C8000D5ED1E6ADFF87492DFF874A266EEE55A7D
:104C9000E5EE877AF4EEE74A77EEC67AF1EE10FA9F
:104CA000C8BFF0EE457AC0ED077AFEF7F0BD904D33
:104CB0009DED0A5A95ED006ABCF1000F41F04C825F
:104CC00025EE866A8B48A5EE076AB0EE675AA6EE17
:104CD000265ABDEEC56A16EE10CA16EE107AF445D5
:104CE000A8BF77466145C8BF0F4606EE107AB8EEFA
:104CF000C66A012A80ED006A3FF41CAD95ED046A96
:104D00009DED0B5A25EE866AA5EE076AB0EE675A4E
:104D1000A6EE265ABDEEC56A16EE10CA16EE107A39
:104D2000F445A8BF77466145C8BF0F4606EE107A26
:104D3000B8EEC66A022A80ED016A3FF4FBAC95ED3D
:104D4000086A9DED0C5A25EE866AA5EE076AB0EE5C
:104D5000675AA6EE265ABDEEC56A16EE10CA16EEC2
:104D6000107AF445A8BF77466145C8BF0F4606EEE6
:104D7000107AB8EEC66A032A80ED026A3FF4DAAC14
:104D800095ED0C6A9DED0D5A25EE866AA5EE076A33
:104D9000B0EE675AA6EE265ABDEEC56A16EE10CAE8
:104DA00016EE107AF445A8BF77466145C8BF0F4696
:104DB00006EE107AB8EEC66A042A80ED036A3FF464
:104DC000B9AC95ED106A9DED0E5A25EE866AA5EEFA
:104DD000076AB0EE675AA6EE265ABDEEC56A16EE11
:104DE00010CA16EE107AF445A8BF77466145C8BFD1
:104DF0000F4606EE107AB8EEC66A052A80ED046A00
:104E00003FF498AC95ED146A9DED0F5A25EE866A35
:104E1000A5EE076AB0EE675AA6EE265ABDEEC56A41
:104E200016EE10CA16EE107AF445A8BF7746614513
:104E3000C8BF0F4606EE107AB8EEC66A062A80EDA5
:104E4000056A3FF477AC95ED186A9DED105A25EE92
:104E5000866AA5EE076AB0EE675AA6EE265ABDEE40
:104E6000C56A16EE10CA16EE107AF445A8BF77464A
:104E70006145C8BF0F4606EE107AB8EEC66A072A2B
:104E800080ED066A3FF456AC95ED1C6A9DED115A13
:104E900065EE865AE7EE055AE6EEA57AFDEEE77A6C
:104EA00017EE905AAE45A8BFAE46A942C8BF8E467F
:104EB00007EE90EAF8EEE77AC0ED077A37E4DFED27
:104EC0000E6AFEF74DBEB5EEC07AF1EE10FA01F1B2
:104ED000A482B7EE006A36EE477AC6EE076AFEF79E
:104EE000A5BEDFED056AFEF71ABF00BFE87300201C
:104EF000EC730020A84D00200000C84248B10020FB
:104F000004950020DFF87893DFF878A3FEF7BFBCA4
:104F1000C8494A79002A3EF4E1A9C74A1278002A12
:104F20003EF4DCA90B78C549DFEDC54A07EE903A9F
:104F30000B88B8EE677A07EE902A06EE103AF8EE84
:104F4000E77AB8EE466A67EE277AB7EE007A87EE20
:104F5000863AB4EEE43AF1EE10FA88BFB0EE643A65
:104F6000B4EEC73AF1EE10FAB8BFB0EE473AFEF72A
:104F7000B7B9B44A5288FEF7ECBCB4F8AE2102F5DA
:104F80007A7292B2FEF7E5BCAF4BD3ED005AFEF752
:104F900092BF049810F08AFCFEF700BFAB4B9FED68
:104FA000AC7AD3ED087AF4EEC77AF1EE10FA00F29B
:104FB000F5849FEDA87AA84DD5ED037A77EE877A30
:104FC000C5ED037AFEF7ADBCDFF8BC82F5F7C0FD96
:104FD000A249D4F8782109680390821A511AC4F8BA
:104FE0007801A8F80420A8F80610FEF776B8F5F7BF
:104FF000AFFD0890FDF7FBBDA3784FF0010A072B2A
:105000003EF6C4AEDFE813F042063E0723072F0743
:105010005A060C0716073A07914B9B7B002B3EF470
:1050200073ACFEF776BCD0003FF538ACFEF77EBC23
:10503000B4F88851954240F2FC8494F8A051002DB8
:1050400041F02480874A884E92ED007AD6ED007AAE
:1050500094F99421C4ED637A77EE676A012AC4ED6E
:10506000617AC4ED606A84ED647A02F07880049B12
:10507000C4F898317D4A9FED777A92ED005A84ED1D
:10508000677A012284F89421FEF7A8BF784B1B8829
:10509000002B40F0E385774A774B1178186805F0CC
:1050A0005FFDD4F86821049B9A1AFDF75BBE734B31
:1050B000D8ED007A93ED007AF0EEE77AF4EEC77A55
:1050C000F1EE10FA7DF7DFAFFDF7CFBFD5ED015A56
:1050D00065EEC65AB0EE674AA5EE874AB4EEE44ADA
:1050E00074EE665AF1EE10FA48BFF0EE455A012A06
:1050F000C0ED005A3FF406AFD5ED055A65EEC65A2D
:10510000B0EE674AA5EE874AB4EEE44A74EE665AFA
:10511000F1EE10FA48BFF0EE455A022AC0ED015AEE
:105120003FF4F0AED5ED095A65EEC65AB0EE674AC7
:10513000A5EE874AB4EEE44A74EE665AF1EE10FA30
:1051400048BFF0EE455A032AC0ED025A3FF4DAAEEA
:10515000D5ED0D5A65EEC65AB0EE674AA5EE874A00
:10516000B4EEE44A74EE665AF1EE10FA48BFF0EE7F
:10517000455A042AC0ED035A3FF4C4AED5ED115A86
:1051800065EEC65AB0EE674AA5EE874AB4EEE44A29
:1051900074EE665AF1EE10FA48BFF0EE455A052A51
:1051A000C0ED045A3FF4AEAED5ED155A65EEC65AC1
:1051B000B0EE674AA5EE874AB4EEE44A74EE666A3A
:1051C000F1EE10FA48BFF0EE456A062AC0ED056A16
:1051D0003FF498AED5ED196A66EEC66AB0EE674A3E
:1051E000A6EE874AF3EE045AB4EEE44A74EE656A1A
:1051F000F1EE10FA48BFF0EE456A072AC0ED066AE4
:105200003FF480AED5ED1D6ADFF87490DFF874A02E
:1052100026EEC66AE6EE077AF4EEE47A77EEE57AF1
:10522000F1EE10FAB8BFF0EE457AC0ED077AFEF75E
:105230002EBB00BF207700202A4C0020144C0020F9
:10524000713DAA3F10460020A4730020AC6E0020E0
:105250008FC2753C000000002C4C0020C84D00207F
:10526000F0A60020F44A00206C740020887400200E
:10527000C0B30020C2B30020C4B30020DC73002000
:1052800048B1002004950020FC8E0020D84D002B52
:1052900041F0EE8095ED006A9DED0A5AD54825EE65
:1052A000866AFDEEE44AA5EE076AB0EE675AA6EEFE
:1052B000265A14EE901ABDEEC56A16EE108A16EE46
:1052C000107AF045A8BF77464145C8BF0F4606EEA5
:1052D000107AB8EEC66A012A80ED006A3EF4D3AABD
:1052E00095ED046A9DED0B5A25EE866AA5EE076AD8
:1052F000B0EE675AA6EE265ABDEEC56A16EE108AC3
:1053000016EE107AF045A8BF77468845B8BF0F461D
:1053100006EE107AB8EEC66A022A80ED016A3EF403
:10532000B2AA95ED086A9DED0C5A25EE866AA5EEA7
:10533000076AB0EE675AA6EE265ABDEEC56A16EEAB
:10534000108A16EE107AF045A8BF77468845B8BF98
:105350000F4606EE107AB8EEC66A032A80ED026A9E
:105360003EF491AA95ED0C6A9DED0D5A25EE866AE4
:10537000A5EE076AB0EE675AA6EE265ABDEEC56ADC
:1053800016EE108A16EE107AF045A8BF77468845CB
:10539000B8BF0F4606EE107AB8EEC66A042A80ED52
:1053A000036A3EF470AA95ED106A9DED0E5A25EE43
:1053B000866AA5EE076AB0EE675AA6EE265ABDEEDB
:1053C000C56A16EE108A16EE107AF045A8BF774629
:1053D0008845B8BF0F4606EE107AB8EEC66A052AB1
:1053E00080ED046A3EF44FAA95ED146A9DED0F5AC4
:1053F00025EE866AA5EE076AB0EE675AA6EE265A33
:10540000BDEEC56A16EE108A16EE107AF045A8BFFA
:1054100077468845B8BF0F4606EE107AB8EEC66AE2
:10542000062A80ED056A3EF42EAA95ED186A9DEDD8
:10543000105A25EE866AA5EE076AB0EE675AA6EE08
:10544000265ABDEEC56A16EE108A16EE107AF045A1
:10545000A8BF77468845B8BF0F46FEF7F2B9664E3B
:10546000D4ED017A94ED006A3188726977EEA77AFB
:10547000F0EE006AB0EE677AA6EE267A4E1E04EBD6
:10548000C601D6EE267A08391032F6EE003A27EE3B
:10549000237A67EEA37A84ED207AC4ED217A574C03
:1054A000274604F1800091ED027A91ED036AD7ED71
:1054B000036AD7ED027A52ED014A12ED025A37EE35
:1054C000674A76EEC65A77EE277AE4EE845A013EB2
:1054D000A1F10801E5EE047A07F1080702F10802DC
:1054E00036EE267A00F10800E4EE877AE5EE475AB8
:1054F00067EEA37A25EEA37AC0ED007A80ED017AFB
:10550000D1D1BEF1140F7EF42CAFF5F721FB039B34
:10551000DFF8FC80C01AA8F80200D4F81451FEF796
:1055200020BFD4F818A1B4F81031C3F120025FFAFB
:1055300082FC334A03EB4A1702EB87075FEA9C02BF
:1055400001F02C86013216012E482F4907EB060880
:1055500007F1100212ED024A12ED035A12ED016A30
:1055600012ED047A50ED024A50ED035A50ED016AF3
:1055700050ED047A64EE244A65EE255A66EE266AFA
:1055800067EE277A1032904541ED024A41ED035A09
:1055900041ED016A41ED047A00F1100001F11001C2
:1055A000D8D11A48A6F110010F4400EB010821449C
:1055B0001CF0030209D0B7EC017AF8EC017A67EE2F
:1055C000277A013AE1EC017AF5D1002B41F0AD8068
:1055D000BEF1140F7EF4C5AEF5F7BAFA039BDFF8FF
:1055E0003080D4F81451C01AA8F80200FEF7B9BEF2
:1055F000EC730020A84D0020EC4D0020AC250020CD
:10560000044E0020944F0020BC250020844F002031
:10561000FC8E0020D4F81851CF49D048D04BEA0076
:10562000114415448A88196800EE102A643AC82A81
:10563000A8BFC822782AB8BF782207EE902AB8EE11
:10564000C07AF8EEE77A00EB850577EE670A77EE29
:10565000876A67EE877A20EEA67AB8EE400AC7EE30
:10566000870A2846D5F814A0D5F81880EF692E6A65
:1056700021F0F2FC029BC5F814A093F800E0C5F8F5
:105680001880BEF1140FEF612E6201F0EC85D4F8A2
:105690001821B449D4F81451013281FB023AAAEB23
:1056A000E27A0AEB4A0AA2EB0A0A0135C4F818A109
:1056B000C4F8145137E7AC4E31785FEA910C01F031
:1056C000A186AA4F0CF101035B0107EB030807F168
:1056D0002002A7F1700012ED076A52ED056A12ED83
:1056E000037A52ED017A52ED025A12ED084A52ED58
:1056F000064A12ED045A26EE066A66EEA66A27EE00
:10570000077A67EEA77AA4EE046A20329045E4EEA9
:10571000A46A00F11000A5EE057AE5EEA57AF1EE97
:10572000C65AB1EEE66AF1EEC76AB1EEE77A40ED2D
:10573000085A00ED076A40ED066A00ED057ACAD105
:10574000A3F120023A4404EB0C1711F0030018BF38
:1057500008320FD052ED017A12ED027A67EEA77A85
:105760000138E7EE077A02F10802B1EEE77AA7EC1A
:10577000017AEFD1BEF1140F01F058850135C4F85C
:105780001451FEF75DBD7A4E7A48B268B18928F0AF
:1057900077F8029B93F800E0BEF1140F01F05685F4
:1057A000D4F814510135C4F8145159E6704E3188BB
:1057B00073684FEA51084FEA88005FEAD10C04EBA6
:1057C000000204EB810500F0A18000F110010CF152
:1057D000010C694F02EB0C1C2944103203F1100E2E
:1057E00005F1100050ED032A50ED043A17ED043A8C
:1057F00017ED032A50ED026A10ED016A17ED021A47
:1058000057ED010A11ED044A11ED035A52ED044A15
:1058100052ED035A12ED027A52ED017A51ED021A5D
:1058200011ED010A73EE238A32EE228A47ED048AD3
:1058300007ED038A71EE268A30EE868A47ED028AEA
:1058400007ED018A74EE848A35EE858A42ED048A7A
:1058500002ED038A77EE218A37EE808A42ED028AD2
:1058600002ED018A73EE633A75EE655A1EED035A36
:1058700032EE623A74EE644A25EE638A1EED044A03
:1058800023EE052A64EE652AA3EE048A10329445BD
:1058900024EE843AA3EE842A07F110070EF1100ECD
:1058A000A5EE853A00F1100001F11001E4EE852A21
:1058B00000ED078A00ED082A01ED073A41ED082ABC
:1058C0005EED055A1EED065A71EE666A30EEC66A46
:1058D00031EEC77A70EE677A26EE253A65EEE63A43
:1058E00025EE674A67EE054AE6EE053AA6EE853AEA
:1058F000A7EE254AE7EEA54A00ED063A40ED053A47
:1059000001ED064A41ED054A7FF46CAF1FFA88F8B5
:105910001A464146174820F093FE726841462846D1
:1059200020F08EFE029B1A78142A7FF4F6ADECE587
:10593000F5F70EF9029B039093F800E0BEF1140F07
:1059400005BFDFF83880D4F81451D4F81451A8F802
:105950000050FDF74EB800BFDC500020CCB0002056
:1059600038B1002056555555E64D00202C26002014
:10597000EC4D0020AC250020BC250020FC8E002032
:10598000306E99BC2716983DA40DC93F843459BE8A
:10599000DB0F4940D06D393A00000000F0EEE76AB5
:1059A000B7EE005A35EE665A1FED0B4A5FED0B5A03
:1059B0001FED0A6A1FED0C7A94ED6A0AF1EEC54AF2
:1059C000E6EE845AF5EEC07AA6EEA56AF1EE10FA7C
:1059D000A6EE867A48BF5FED127A27EE247A48BF9A
:1059E00037EEC77A27EE000A29F016F9B0F5617F85
:1059F00000F3068707EE900AF8EEE76A5FED1B7A80
:105A000066EEA76A07EE905ABDEEE67AF8EEE77A00
:105A100017EE103A2033402B41F2F9841FED220A91
:105A200029F0FAF800B207EE900AB8EEE77AFFF72D
:105A3000C2BAD34A02F1500503E00432AA4200F090
:105A400025831378262BF8D19678D3789E42F4D20A
:105A5000FFF7F3BACB4822F02BFDFEF7F1BCCA48A2
:105A600022F026FDFEF7F8BCC84822F021FDFEF723
:105A7000EDBCC74DC74F95ED004A95ED057AD5EDC4
:105A8000014A95ED066AD5ED046A95ED035AD5ED08
:105A9000025A67EE897A07EB8602A4EE277AA4EE13
:105AA000A76A66EEC76AA5EE476AE5EEA76A20EE2A
:105AB000070A85ED056AC5ED066A82ED007A29EED2
:105AC000088A29F0A9F869EE288AD5ED0E5AD5ED95
:105AD000176A95ED091AD5ED121A95ED0F5A95ED45
:105AE000187A95ED0A2AD5ED132A95ED0D6AD5EDB4
:105AF000167A95ED0C3AD5ED0B3A95ED154AD5EDA4
:105B0000144AE1EE085A002207EB8601E8EEA16A8A
:105B100000B2C4F80021A2EE085AC4F80421C4F867
:105B20000821A8EEA27A26EE656A67EEE67AA3EE71
:105B3000655AA3EE886AA6EEC47AE8EEA47A85EDEB
:105B40000E5AC1ED205A85ED0F6AC1ED406A85ED10
:105B5000177AC5ED187AFEF72BBBD4F89851049B41
:105B60005D1BFEF72BBABBF93820CBF8201007EEEF
:105B7000902A0121F8EEE77ACBF86020CBF87C1070
:105B80000022012FCBED1C7ACBED1B7ACBF87420D1
:105B900001F0E182B7427CF490AFBBF93A20CBF838
:105BA000642007EE902A00210122F8EEE77ACBF874
:105BB0002410CBF890200022012FCBED217ACBEDE1
:105BC000207ACBF8882001F0C282B7427CF4A9AFDA
:105BD000BBF93C20CBF8682007EE902A0021012277
:105BE000F8EEE77ACBF82810CBF8A4200022012F9A
:105BF000CBED267ACBED257ACBF89C207CF4C5AF93
:105C00009FED658A032D3BD04CB107EE904AF8EE2C
:105C1000E77AF4EEC87AF1EE10FA01F14A845F4AAD
:105C20005F4C1168DBF86820A8F8060094F82001A2
:105C300002EB560292FBF6F60022CBF828608A624D
:105C40000A63CA6228B1574A126832F480637CF44E
:105C50009FAF012026F022FAFCF79ABF52494B6908
:105C6000002B3DF47FA85148514B008893FBF0F086
:105C70000B684FF0010E186081F811E0FDF772B863
:105C8000B0EE480A28F0C8FF00B2BDE700230AAD15
:105C90002946184609221CF065FB01287EF476A8E7
:105CA0000A9B93F8FE21552A01F07D8241F2B4123D
:105CB00002210123A1546370FEF768B82278237D86
:105CC0003C4EDFF8FC90032A14BF4FF48077802706
:105CD000002B40D0012BFBD1374B6268196830682C
:105CE00000234FEA412E4FF0FF31B1FBFEF112EBE2
:105CF000010B43F1000C0021614500F1020008BFD7
:105D0000584538BF83465A462C4902201CF06AFC8D
:105D1000032801F2408201A353F820F08D3D0108D1
:105D20002D5D01088D3D01082D5D01086268A368A5
:105D30002569991AA94284BFE2602161032841D0F4
:105D40000133B3FBF7F207FB12320AB13B449B1A53
:105D500000226360227532684946023200201CF03E
:105D600041FC032801F2178201A353F820F000BF81
:105D70008D3D0108BF5E01088D3D0108C55D01082C
:105D8000C8470020886C0020B86B0020746B00208E
:105D900070500020044E0020000000006C790020AC
:105DA000AC25002080770020C8B30020E0B300209D
:105DB00020A10700D86C0020E06C0020D85A0020F9
:105DC000D45A002023690622652BA27032D922788A
:105DD000032A14BF6FF0FF026FF07F02A3F1650387
:105DE00003EA020303F1010314BF4FF4807280221F
:105DF0009A4223611ED23268E66802329F199742A6
:105E000081F01B84BF4A6660D16FA760490203FB23
:105E100001F30521166042F81C3C42F8183CA170C1
:105E2000A268B949012025F021FA012841F09B839D
:105E30000623A3700021B54824F038FE012841F064
:105E40009283A3780133DBB2A370FFF7D8B8B04BCD
:105E500000930320A07030230522AE49AB4825F003
:105E6000D9FBFDF793BF41F27013E35C002B3DF4C7
:105E70008DAFA64822F01CFBFDF788BF032363709B
:105E8000FDF784BF0AAD41F2FC162946A059002354
:105E900009221CF067FA01287DF478AF00230A9AE2
:105EA0002370B2F80B30B3F5007F01F0668341F246
:105EB000B41203210123A1546370FDF767BF636827
:105EC00084F814A00133A36006E7934A934DD2ED02
:105ED000006A934A95ED006A1278C4ED636A84ED16
:105EE000646A002A00F0A18276EE665A94F9942141
:105EF000C4ED605A0132C4ED616A00F00786049B6C
:105F0000C4F89831002537EE677AFCEEE77A854EC3
:105F100084ED677A17EE902AA4F88821FF2296ED87
:105F2000005A84F89421FEF759B8DFED7F7A7F4B51
:105F300094ED677AC3ED007AC3ED017AC3ED027A7E
:105F40007B4BB0EE676AF0EE673A1968FDF7FFB871
:105F5000784B794AB3F90430DFED787A82FB03128B
:105F6000DB17C3EBA2031BB208EE103AB8EEC88AE7
:105F700028EE278AB0EE480A05F0BEFEF0EE408A11
:105F8000B0EE480A05F03EFE6D4BDD78002D00F0C6
:105F9000AD836C49B4F90A22B1F9023044F2506081
:105FA0009B1A834240F3F186A3F50C43A03B6E425B
:105FB0009E4200F3E786AB42A8BF2B46B1F9001022
:105FC000B4F9080213440A1A44F250611BB28A421F
:105FD000A4F80A3240F3E186A2F50C42A03A9642B8
:105FE00003DC9542A8BF15462E46821912B207EE71
:105FF000902A07EE103AF8EEE77AB8EEC77A67EE25
:10600000E86A9FED516AA4F80822E0EE076A60EEA4
:10601000277AE8EE877A26EE867A67EE867ABDEEF4
:10602000C77AFDEEE77A17EE102A17EE903AA4F839
:106030004821A4F84A31FDF7A4BE444B1D7805F071
:10604000010CFDF720BC4249DFED427A0968C4ED3E
:106050004A7A11F0805840F0C783D9F8001011F443
:10606000800800F0F4814FF00008B6EE007A67EE89
:10607000877AF4EEE57AF1EE10FAC8BFF0EE675ACF
:1060800040F3B283C4ED675AFDF7A9BA224A234D03
:10609000D2ED007A224A95ED007A1278C4ED637A47
:1060A00084ED647A002A00F03B8377EE676A94F906
:1060B0009421C4ED606A0132C4ED617A00F0758606
:1060C000049BC4F8983100259FED177A154E84ED96
:1060D000677AFF2296ED005A84F89421FDF77EBF7F
:1060E00073EEC67AB7EE007AF4EEC77AF1EE10FAE4
:1060F000C4ED4A7A41F3398084EEA77A8DED0A7AAD
:10610000FDF763BA646C0020D45A0020406C002074
:1061100005A80308402E04087C4900207074002064
:10612000345700208474002000000000804D0020BF
:1061300088770020347700206766666635FA8E3CE3
:106140009C7A0020F87A0020CDCCCC3DF04B00208A
:10615000D44A002000000080002F00F0DF8625EEEA
:10616000866AC048A5EE076AB0EE675AA6EE265AC0
:10617000BDEEC56A16EE10CA16EE107AF445A8BF39
:1061800077466145C8BF0F4606EE107AB8EEC66A7C
:10619000012A80ED006A3DF47AAB95ED046A9DED2D
:1061A0000B5A25EE866AA5EE076AB0EE675AA6EE90
:1061B000265ABDEEC56A16EE10CA16EE107AF445E0
:1061C000A8BF77466145C8BF0F4606EE107AB8EE05
:1061D000C66A022A80ED016A3DF459AB95ED086A62
:1061E0009DED0C5A25EE866AA5EE076AB0EE675A59
:1061F000A6EE265ABDEEC56A16EE10CA16EE107A45
:10620000F445A8BF77466145C8BF0F4606EE107A31
:10621000B8EEC66A032A80ED026A3DF438AB95ED0C
:106220000C6A9DED0D5A25EE866AA5EE076AB0EE62
:10623000675AA6EE265ABDEEC56A16EE10CA16EECD
:10624000107AF445A8BF77466145C8BF0F4606EEF1
:10625000107AB8EEC66A042A80ED036A3DF417ABE3
:1062600095ED106A9DED0E5A25EE866AA5EE076A39
:10627000B0EE675AA6EE265ABDEEC56A16EE10CAF3
:1062800016EE107AF445A8BF77466145C8BF0F46A1
:1062900006EE107AB8EEC66A052A80ED046A3DF46F
:1062A000F6AA95ED146A9DED0F5A25EE866AA5EEC5
:1062B000076AB0EE675AA6EE265ABDEEC56A16EE1C
:1062C00010CA16EE107AF445A8BF77466145C8BFDC
:1062D0000F4606EE107AB8EEC66A062A80ED056A09
:1062E0003DF4D5AA95ED186A9DED105A25EE866A03
:1062F000A5EE076AB0EE675AA6EE265ABDEEC56A4D
:1063000016EE10CA16EE107AF445A8BF774661451E
:10631000C8BF0F4606EE107AB8EEC66A072A80EDAF
:10632000066A3DF4B4AA95ED1C6A9DED115A65EE1E
:10633000865AE5EE075AE6EEA57AFDEEE77A17EE05
:10634000902A9645A8BF96468A42A8BF714607EE96
:10635000901AF8EEE77AC0ED077AFDF798BABEF129
:10636000010F7FF74DAC07EE103AB8EEC77AC7EED3
:10637000876AB1EEE68A45E4BEF1010F40F3E78695
:1063800007EE103AB8EEC77AC7EE876AB1EEE68A32
:10639000032D13D04CB107EE904AF8EEE77AF4EEF5
:1063A000C87AF1EE10FA01F18480DBF8642002EB88
:1063B000560292FBF6F2CBF8242006E4B0EE480A2F
:1063C00028F02AFC00B2E5E7BEF1010F40F3C386D6
:1063D00007EE103AB8EEC77AC7EE876AB1EEE68AE2
:1063E000032D14D04CB107EE904AF8EEE77AF4EEA4
:1063F000C87AF1EE10FA01F15C80DBF8602002EB64
:10640000560292FBF6F2CBF82020FFF7C3BBB0EEAA
:10641000480A28F001FC00B2E4E7F7EE006AFDF755
:1064200005BCF7EE006AFDF77ABC76EEC65AF0EED0
:10643000466A5BE58222FDF781BFDFED0B7AFDF74F
:1064400049BF0A4A1768B7F93260FEF72EBAB6EEAE
:10645000007AF4EEC75AF1EE10FA3FF706AEFDF7F8
:10646000BEB800BFA84D002000000243887700207E
:1064700095ED006A9DED0A4AEE4825EE866AFDEE2E
:10648000E43AA4EE076AB0EE674AA6EE264A13EE97
:10649000901AB4EEC45AF1EE10FAB0EE446A88BF16
:1064A000B0EE646ABDEEC66A16EE108A16EE107A79
:1064B000F045A8BF77464145C8BF0F4606EE107AA3
:1064C000B8EEC66A012A80ED006A3DF4DCA995EDBC
:1064D000046A9DED0B4A25EE866AA4EE076AB0EECB
:1064E000674AA6EE264AB4EEC45AF1EE10FAB0EEB0
:1064F000446A88BFB0EE646ABDEEC66A16EE108AC2
:1065000016EE107AF045A8BF77468845B8BF0F460B
:1065100006EE107AB8EEC66A022A80ED016A3DF4F2
:10652000B2A995ED086A9DED0C4A25EE866AA4EEA7
:10653000076AB0EE674AA6EE264AB4EEC45AF1EEF8
:1065400010FAB0EE446A88BFB0EE646ABDEEC66A67
:1065500016EE108A16EE107AF045A8BF77468845E9
:10656000B8BF0F4606EE107AB8EEC66A032A80ED71
:10657000026A3DF488A995ED0C6A9DED0D4A25EE61
:10658000866AA4EE076AB0EE674AA6EE264AB4EE23
:10659000C45AF1EE10FAB0EE446A88BFB0EE646AF5
:1065A000BDEEC66A16EE108A16EE107AF045A8BF48
:1065B00077468845B8BF0F4606EE107AB8EEC66A31
:1065C000042A80ED036A3DF45EA995ED106A9DED05
:1065D0000E4A25EE866AA4EE076AB0EE674AA6EE7A
:1065E000264AB4EEC45AF1EE10FAB0EE446A88BFFF
:1065F000B0EE646ABDEEC66A16EE108A16EE107A28
:10660000F045A8BF77468845B8BF0F4606EE107A1A
:10661000B8EEC66A052A80ED046A3DF434A995ED0A
:10662000146A9DED0F4A25EE866AA4EE076AB0EE65
:10663000674AA6EE264AB4EEC45AF1EE10FAB0EE5E
:10664000446A88BFB0EE646ABDEEC66A16EE108A70
:1066500016EE107AF045A8BF77468845B8BF0F46BA
:1066600006EE107AB8EEC66A062A80ED056A3DF499
:106670000AA995ED186A9DED104A25EE866AA4EEEA
:10668000076AB0EE674AA6EE264AB4EEC45AF1EEA7
:1066900010FAB0EE446A88BFB0EE646ABDEEC66A16
:1066A00016EE108A16EE107AF045A8BF7746884598
:1066B000B8BF0F4606EE107AB8EEC66A072A80ED1C
:1066C000066A3DF4E0A895ED1C6A9DED114A65EE61
:1066D000865AE7EE045AE6EEA57AB4EEE75AF1EEF2
:1066E00010FAC8BFF0EE647AFDF7BDB8524B9FEDCB
:1066F000536AB3F90020B3F9023007EE902A06EE90
:10670000903AF8EEE77AF8EEE66A27EEE87A60EE7D
:10671000277AA0EE267AE8EEA67A27EE067A7CE4BF
:1067200077EEC76AF0EE477AC1E4454A4FEA8C0734
:1067300002EBCA1A9A083844274436D001324FEA8D
:10674000021C0AEB0C080AF1100200F1100607F116
:10675000100112ED024A12ED035A12ED016A12ED18
:10676000047A56ED024A56ED035A56ED016A56ED8B
:10677000047A64EE244A65EE255A66EE266A67EED0
:10678000277A1032904541ED024A41ED035A41ED1E
:10679000016A41ED047A06F1100601F11001D8D129
:1067A000ACF1100292441044174413F0030C3EF471
:1067B0000FAFBAEC017AF0EC017A67EE277ABCF100
:1067C000010CE7EC017AF4D1FEF702BFBA8E9FED1F
:1067D0001D7A07EE902AF8EEE77A1B4A67EE877A71
:1067E000C2ED007AFDF7A2B8B7EE007A77EE677ACD
:1067F000F4EEE75AF1EE10FA88BFF0EE675A41E482
:1068000007EE905ADFED116AF8EEE77A66EEA65AC7
:106810009FED0F5A9FED0F6A9FED0F7AA5EE856AE7
:1068200026EEA55AA5EE867AE5EE076A26EEA70AB9
:10683000FFF7F6B8A84D0020F87A0020CDCCCC3D6B
:10684000044E00206F12833A7C00002084F9223F1E
:1068500092E741B99730083C15A82ABE95ED006A29
:106860009DED0A4AAE4825EE866AFDEEE43AA4EEB6
:10687000076AB0EE674AA6EE264A13EE907AB4EEA7
:10688000C45AF1EE10FAB0EE446A88BFB0EE646A02
:10689000BDEEC66A16EE10CA16EE101AF445A8BF71
:1068A00071466745C8BF394606EE101AB8EEC66A8B
:1068B000012A80ED006A3DF43DAF95ED046A9DED3F
:1068C0000B4A25EE866AA4EE076AB0EE674AA6EE8A
:1068D000264AB4EEC45AF1EE10FAB0EE446A88BF0C
:1068E000B0EE646ABDEEC66A16EE10CA16EE101A55
:1068F000F445A8BF7146BC45B8BF394606EE101A2C
:10690000B8EEC66A022A80ED016A3DF413AF95ED38
:10691000086A9DED0C4A25EE866AA4EE076AB0EE81
:10692000674AA6EE264AB4EEC45AF1EE10FAB0EE6B
:10693000446A88BFB0EE646ABDEEC66A16EE10CA3D
:1069400016EE101AF445A8BF7146BC45B8BF3946CB
:1069500006EE101AB8EEC66A032A80ED026A3DF40C
:10696000E9AE95ED0C6A9DED0D4A25EE866AA4EE22
:10697000076AB0EE674AA6EE264AB4EEC45AF1EEB4
:1069800010FAB0EE446A88BFB0EE646ABDEEC66A23
:1069900016EE10CA16EE101AF445A8BF7146BC4593
:1069A000B8BF394606EE101AB8EEC66A042A80ED62
:1069B000036A3DF4BFAE95ED106A9DED0E4A25EEDB
:1069C000866AA4EE076AB0EE674AA6EE264AB4EEDF
:1069D000C45AF1EE10FAB0EE446A88BFB0EE646AB1
:1069E000BDEEC66A16EE10CA16EE101AF445A8BF20
:1069F0007146BC45B8BF394606EE101AB8EEC66AF5
:106A0000052A80ED046A3DF495AE95ED146A9DED7E
:106A10000F4A25EE866AA4EE076AB0EE674AA6EE34
:106A2000264AB4EEC45AF1EE10FAB0EE446A88BFBA
:106A3000B0EE646ABDEEC66A16EE10CA16EE101A03
:106A4000F445A8BF7146BC45B8BF394606EE101ADA
:106A5000B8EEC66A062A80ED056A3DF46BAE95ED88
:106A6000186A9DED104A25EE866AA4EE076AB0EE1C
:106A7000674AA6EE264AB4EEC45AF1EE10FAB0EE1A
:106A8000446A88BFB0EE646ABDEEC66A16EE10CAEC
:106A900016EE101AF445A8BF7146BC45B8BF39467A
:106AA00006EE101AB8EEC66A072A80ED066A3DF4B3
:106AB00041AE95ED1C6A9DED114A65EE865AE7EEF2
:106AC000045AE6EEA57AB4EEE75AF1EE10FAC8BF22
:106AD000F0EE647AFDEEE77A17EE901A8E45A8BFC5
:106AE0008E468F42D8BF774607EE907AF8EEE77A67
:106AF000C0ED077AFDF71BBE0A494A69002A3CF43B
:106B000014AA0A6813604B74FCF70FBAD4F89851B2
:106B1000049B5D1BFFF7F7B9034DFCF77FBF00BF78
:106B2000A84D0020C8B300202C4C0020002F00F0FE
:106B3000B583E84D9DED0A4A95ED006A25EE866A1B
:106B4000A4EE076AB0EE674AA6EE264AB0EE446AA3
:106B500033B1B4EE445AF1EE10FAC8BFB0EE646A35
:106B6000FDEEE44ABDEEC66A14EE907A16EE101AF7
:106B70008F4214EE90CA00F3F2847145A8BF7146AB
:106B800006EE101AD448B8EEC66A012A80ED006AF3
:106B90003CF47DAE95ED046ADDED0B4A25EE866A88
:106BA000A4EE876AF0EE674AE6EE264AB0EE646A23
:106BB000002B00F0CA84B4EEE45AF1EE10FA40F370
:106BC000C48439467145A8BF714606EE101AB8EE66
:106BD000C66A022A80ED016A3CF459AE95ED086A56
:106BE000DDED0C4A25EE866AA4EE876AF0EE674A70
:106BF000E6EE264AB0EE646A002B00F09C84B4EE08
:106C0000E45AF1EE10FA40F3968439467145A8BF74
:106C1000714606EE101AB8EEC66A032A80ED026AC3
:106C20003CF435AE95ED0C6ADDED0D4A25EE866A35
:106C3000A4EE876AF0EE674AE6EE264AB0EE646A92
:106C4000002B00F06E84B4EEE45AF1EE10FA40F33B
:106C5000688439467145A8BF714606EE101AB8EE31
:106C6000C66A042A80ED036A3CF411AE95ED106A01
:106C7000DDED0E4A25EE866AA4EE876AF0EE674ADD
:106C8000E6EE264AB0EE646A002B00F04084B4EED3
:106C9000E45AF1EE10FA40F33A8439467145A8BF40
:106CA000714606EE101AB8EEC66A052A80ED046A2F
:106CB0003CF4EDAD95ED146ADDED0F4A25EE866AE4
:106CC000A4EE876AF0EE674AE6EE264AB0EE646A02
:106CD000002B00F01284B4EEE45AF1EE10FA40F307
:106CE0000C8439467145A8BF714606EE101AB8EEFD
:106CF000C66A062A80ED056A3CF4C9AD95ED186AAE
:106D0000DDED104A25EE866AA4EE876AF0EE674A4A
:106D1000E6EE264AB0EE646A002B00F0E583B4EE9E
:106D2000E45AF1EE10FA40F3DF8339467145A8BF0B
:106D3000714606EE101AB8EEC66A072A80ED066A9A
:106D40003CF4A5AD95ED1C6ADDED114A65EE865A61
:106D5000E4EE875AE5EEA67A002B00F0BD83F4EE50
:106D6000C57AF1EE10FA40F1B7833A467245A8BFF2
:106D70007246944607EE90CAF8EEE77AC0ED077ABD
:106D8000FCF785BD3346FFF719B954488342BCBFB1
:106D900003F50C43A033FFF70AB950498A42BCBF40
:106DA00002F50C42A032FFF71AB9D4F89851049BAF
:106DB0005D1BFFF789B995ED000A039327F02CFFBF
:106DC000474A4849D2F8EC20DFF84CE181FB023118
:106DD000D217C2EBA11207EE902AF8EEE77AAEF8CE
:106DE0000000FDEEE77A039B17EE902AAEF8022032
:106DF000FCF719BE07EE905ADFED3B6A9FED3B7A38
:106E000084F80052F8EEE77A67EEA67A77EE876AA2
:106E1000BDEEE66A16EE103A2033402B40F2AC820B
:106E2000DFED336A334BBDEEE77AC3ED016A17EE4F
:106E3000103A2033402B00F29C829FED2F7AF4EE23
:106E4000C77AF1EE10FA40F3FD83DFED2C5A9FED87
:106E50002C6A01E0F0EE477AF4EEC67AF1EE10FA11
:106E600037EEE57AF6DCDFED277AB4EEE77AF1EE7D
:106E700010FA40F1EA83DFED215A9FED236A01E029
:106E8000B0EE677AB4EEC67AF1EE10FA77EE257AB4
:106E9000F6D49FED167AF4EEC77AF1EE10FA40F3CD
:106EA000FC829FED157A77EE677A67EEA75A9FED21
:106EB000175A9FED176A9FED177AA5EE856A27EEA0
:106EC000A55AA5EE867AE5EE077AC4ED817AFDF73C
:106ED0004DBD00BFEC730020A84D0020B0B9FFFFEE
:106EE00014030020D34D621035FA8E3CDB0FC93FEE
:106EF000000000007C000020DB0F4940DB0FC94090
:106F0000E4CB1641DB0F49C0E4CB16C192E741B98F
:106F10009730083C15A82ABEFC8E002025EE866A14
:106F2000A5EE076AB0EE675AA6EE265ABDEEC56A10
:106F300016EE100A814200F3AF817045A8BF70467B
:106F400006EE100AB8EEC66AB8F1000F00F0A6838C
:106F5000D948012A80ED006A3CF499AC95ED046AA9
:106F60009DED0B5A25EE866AA5EE076AB0EE675ACC
:106F7000A6EE265ABDEEC56A16EE107AB94200F3A7
:106F800089817745A8BF774606EE107AB8EEC66AC3
:106F9000B8F1000F00F07783022A80ED016A3CF41B
:106FA00076AC95ED086A9DED0C5A25EE866AA5EE45
:106FB000076AB0EE675AA6EE265ABDEEC56A16EE0F
:106FC000107AB94200F364817745A8BF774606EE90
:106FD000107AB8EEC66AB8F1000F00F07583032A84
:106FE00080ED026A3CF453AC95ED0C6A9DED0D5AB0
:106FF00025EE866AA5EE076AB0EE675AA6EE265A17
:10700000BDEEC56A16EE107AB94200F33F817745AE
:10701000A8BF774606EE107AB8EEC66AB8F1000F40
:1070200000F04783042A80ED036A3CF430AC95ED10
:10703000106A9DED0E5A25EE866AA5EE076AB0EE3F
:10704000675AA6EE265ABDEEC56A16EE107AB94208
:1070500000F31A817745A8BF774606EE107AB8EE9E
:10706000C66AB8F1000F00F0E883052A80ED046AD3
:107070003CF40DAC95ED146A9DED0F5A25EE866A31
:10708000A5EE076AB0EE675AA6EE265ABDEEC56AAF
:1070900016EE107AB94200F3F5807745A8BF77461F
:1070A00006EE107AB8EEC66AB8F1000F00F0BA83A7
:1070B000062A80ED056A3CF4EAAB95ED186A9DED71
:1070C000105A25EE866AA5EE076AB0EE675AA6EE5C
:1070D000265ABDEEC56A16EE107AB94200F3D0808A
:1070E0007745A8BF774606EE107AB8EEC66AB8F1C3
:1070F000000F00F0BD82072A80ED066A3CF4C7ABA2
:1071000095ED1C6A9DED115A65EE865AE5EE075A1B
:10711000E6EEA57AFDEEE77A17EE902A914203DCBF
:107120007245A8BF7246114607EE901AF8EEE77A4C
:10713000B8F1000F7FF422AE089B002B7FF41EAE47
:10714000059B079A9342B8BFF0EE647A16E69FED6E
:10715000618AFFF71DB99FED5F8AFFF741B9D4F847
:107160009851049B5D1BFDF785BF5449096811F0D8
:1071700080587EF47AAFFEF770BF9FED510ADFF8BA
:10718000508125EE800A27F047FDD4F81451A8F865
:107190000600FDF7E6B8237DFEF79ABD49484A4947
:1071A0008046FEF705BA93F8FF21AA2A7EF47EAD49
:1071B000D3F8C61149B193F8C221A2F10B000128FE
:1071C0002DD902F0F702062A29D0D3F8D61149B1F9
:1071D00093F8D221A2F10B00012820D902F0F70286
:1071E000062A1CD0D3F8E61149B193F8E221A2F1A6
:1071F0000B00012813D902F0F702062A0FD0D3F8AA
:10720000F61100293EF452AD93F8F231A3F10B02CE
:10721000012A04D903F0F703062B7EF447AD41F2AF
:10722000FC120123A150A370FEF72DBEF3F790FCD2
:10723000029BDFF89C8093F800E0039B3178D4F840
:107240001451C01AA8F80400FEF798BAF3F780FCAE
:10725000029BDFF87C8093F800E0039BC01AA8F83B
:107260000200FEF79DBAF3F773FC029BDFF8608023
:1072700093F800E0039BC01AA8F80200FEF707BAD3
:107280000F4630E70F460BE70F46E6E60F46C1E62E
:107290000F469CE60F4677E6084651E60AA9BDEE82
:1072A000E46A01EB820294460848034D09941A46A9
:1072B00016EE107A434627E0A84D0020D44A00205D
:1072C0000000C842844F0020AC250020EC73002051
:1072D000FC8E002000000000E4CB1641DB0F49C00B
:1072E000DB0FC940E4CB16C1DB0FC93FDB0F4940C0
:1072F00092E741B99730083C15A82ABE6145A5EC34
:10730000016A00F1100031D090ED006AB1EC014A41
:1073100025EE866AA7EE046AB0EE674AA6EE864AB4
:10732000B0EE446A32B1B4EE445AF1EE10FAC8BF7E
:10733000B0EE646ABDEEC66A16EE108A474506EEE8
:10734000107A04DCF045A8BFF04606EE108AB8EECD
:10735000C66A002BD2D1089C002CCFD1059CA04638
:10736000079CA045B8BFB0EE646AC7E7099CFCF76C
:107370008EBA5FED287AA8E5F4EEC77AF1EE10FA3E
:1073800040F370815FED2A5A1FED2D6A01E0F0EEA7
:10739000476AF4EEC66AF1EE10FA36EEE57AF6DCEC
:1073A0005FED326AB4EEE67AF1EE10FA40F1578101
:1073B0005FED355A1FED356A01E0B0EE667AB4EE46
:1073C000C67AF1EE10FA77EE256AF6D41FED3A7A16
:1073D000F4EEC76AF1EE10FA72DD1FED3C7A77EE3B
:1073E000666A66EEA65A1FED3E5A1FED3E6A1FED15
:1073F0003E7AA5EE856A26EEA55AA5EE867AE5EEDA
:10740000076A0FE5D24F07F18002FEF79EB99FEDA4
:10741000D17AF4EEC76AF1EE10FA40F32681DFED7F
:10742000CE5A9FEDCE6A01E0F0EE476AF4EEC66AEE
:10743000F1EE10FA36EEE57AF6DCDFEDC96AB4EE6D
:10744000E67AF1EE10FA40F14A81DFEDC35A9FED82
:10745000C56A01E0B0EE667AB4EEC67AF1EE10FAD3
:1074600077EE256AF6D49FEDC07AF4EEC76AF1EEA6
:1074700010FA05DD9FEDB77A77EE666AFFF7C6B9B9
:107480009FEDBA7AF4EEC76AF1EE10FA44BF9FEDB1
:10749000B47A77EE666AFFF7B9B99FEDB47AF4EE85
:1074A000C77AF1EE10FA44BF9FEDAD7A77EE677AB6
:1074B000FBE4A8F80600ABF8A860A54CFBF76FBB8F
:1074C0009FEDAA7AF4EEC76AF1EE10FA44BF9FED81
:1074D000A47A77EE666A84E7FDEEE77A17EE902AE3
:1074E000BA42FFF647AC41E4BDEEC66A16EE101A8A
:1074F000B942BFF61BAC39461BE4BDEEC66A16EEB8
:10750000101AB942BFF6EEAB3946FFF7EEBBBDEE3F
:10751000C66A16EE101AB942BFF6C0AB3946FFF77D
:10752000C0BBBDEEC66A16EE101AB942BFF692ABEA
:107530003946FFF792BBBDEEC66A16EE101AB94285
:10754000BFF664AB3946FFF764BBBDEEC66A16EE04
:10755000101AB942BFF636AB3946FFF736BB14EE08
:10756000901AFFF70DBB02287CF410AC41F2B41264
:107570000123A3546370FCF709BC137C022B7EF437
:1075800096AC92F8FE31552B7EF491AC92F8FF3117
:10759000AA2B7EF48CACD589A659754B2E441E605F
:1075A000577B41F210217B1E7F2B67503EF67FAC4C
:1075B0007B4237EA03037EF47AAC7B0241F2182166
:1075C000013B6350D08A00B9506A6A4941F20423F2
:1075D000E050B2F811305B0103F2FF135B120B6055
:1075E000B2F8131001B9116A40001D440544491B4B
:1075F00041F2082E40F6F475B1FBF7F1A94244F8C8
:107600000E1040F20B814FF6F475A94240F2028150
:1076100003212170D26A58493344184441F20C25A1
:1076200041F21C2309786051E25009B927F0ECF8C7
:10763000A3780133A370FCF7A9BB23F001F92369F8
:10764000FEF7E0BBB0EE677A0DE4F0EE477A20E497
:1076500094F87431002B7BF436ADFBF721BDF0EECE
:10766000476AB3E6B0EE667A9AE6B0EE667AE4E68A
:10767000089B002B7FF43FAD059B079FBB42B8BF23
:10768000B0EE646A37E5089B002B7FF485AC059B60
:10769000079FBB42B8BFB0EE646A7DE4089B002B35
:1076A0007FF456AC059B07988342B8BFB0EE646A7E
:1076B0004EE4089B002B7FF4B5AC059B079FBB42B3
:1076C000B8BFB0EE646AADE4089B002B7FF487ACD2
:1076D000059B079FBB42B8BFB0EE646A7FE4F0EE43
:1076E000476AC0E6132B05D1B0EE480A27F094FA9A
:1076F000069B1880B0EE480ADBF86C371F489847A5
:10770000029B1B78132BB0EE408A7DF458A827F01B
:1077100083FA069B5880FDF752B8194BD3ED007AD7
:10772000B1EE677AF4EEC7CAF1EE10FA6FD4F4EE58
:10773000E7CAF1EE10FA88BFF0EE67CA114B87ED89
:1077400000BA1B689342BBF653ABFBF779BB00BF93
:10775000AC250020DB0F4940DB0FC940E4CB1641CC
:10776000DB0F49C0E4CB16C1DB0FC93FDB0FC9BF3C
:10777000D06C0020F06C0020B06C0020CCB0002059
:10778000E0730020C4730020314A324B10681B683C
:107790009847314BD7ED006A93ED007A2F4BD3ED2C
:1077A000007A2F4B93ED006A2E4B83ED020A2E4B8D
:1077B00067EE277A2B4427EEAB7AD3ED007A67EE9B
:1077C000277AF0EE665AECEEA75AB1EE467AF4EE5E
:1077D000C75AF1EE10FA08D4F4EEC65AF1EE10FAD8
:1077E0008CBFB0EE467AB0EE657A204B1B78012B49
